:020000040800F2
:1000000000040020A51F0008F71F0008F71F0008C4
:10001000F71F0008F71F0008F71F00080000000086
:10002000000000000000000000000000F71F0008B2
:10003000F71F000800000000F71F0008E9FD010895
:1000400075FF010877FF010879FF01087DFF0108AE
:100050009DFF01089FFF0108A1FF0108C5FF0108DE
:10006000E9FF01080D0002083100020855000208EE
:1000700057000208590002085B0002085D000208F0
:100080005F0002086100020863000208F71F000811
:10009000F71F0008F71F0008F71F00086500020897
:1000A000B1000208B3000208B5000208B700020858
:1000B000B9000208BD000208E9000208590102085F
:1000C0005B0102085D0102085F010208610102088C
:1000D00065010208D5020208FD0102089903020821
:1000E0005D0402082105020823050208250502080F
:1000F00029050208910502089305020895050208E2
:1001000097050208990502089B0502089D0502084B
:10011000A10502087506020877060208790602089A
:100120008507020887070208890702088B0702086B
:1001300000000000000000000000000000000000BF
:1001400000000000000000000000000000000000AF
:10015000000000000000000000000000000000009F
:10016000000000000000000000000000000000008F
:10017000000000000000000000000000000000007F
:10018000000000000000000000000000000000006F
:10019000000000000000000000000000000000005F
:1001A000000000000000000000000000000000004F
:1001B000000000000000000000000000000000003F
:1001C000000000000000000000000000000000002F
:1001D000000000000000000000000000000000001F
:0401E0005FF8E0F1F3
:1001E800032A70B404460D4626D941EA000313F0E9
:1001F800030F13D020782B78984208BF294606D0E1
:100208001EE014F8010F11F8013F984218D1012A95
:1002180002F1FF32F5D1002070BC70470B4604464E
:1002280051F8045B50F8046BAE4204D1043A04461A
:10023800032A0B46F2D81D461046002ADAD1EBE70E
:10024800C01AE9E7032A2DE9F00109D82AB10023E9
:10025800CC5CC45401339342FAD1BDE8F001704735
:100268000B468218014603E02478013301F8014B5C
:1002780011F0030F1C46F7D113F003055DD06E4251
:10028800C5F1040CED009B594FEACC0C08E004348E
:10029800A7593B4607FA0CF748EA070741F8047BD9
:1002A800571A23FA05F8032FF1DC03E014F8013B91
:1002B80001F8013B8A42F9D8CFE753F8404C41F89E
:1002C800404C53F83C4C41F83C4C53F8384C41F8FE
:1002D800384C53F8344C41F8344C53F8304C41F80E
:1002E800304C53F82C4C41F82C4C53F8284C41F81E
:1002F800284C53F8244C41F8244C53F8204C41F82E
:10030800204C53F81C4C41F81C4C53F8184C41F83D
:10031800184C53F8144C41F8144C53F8104C41F84D
:10032800104C53F80C4C41F80C4C53F8084C41F85D
:10033800084C53F8044C41F8044C561A1D460C4618
:10034800403340313F2EB8DC2B460FE053F8101CE9
:1003580044F8101C53F80C1C44F80C1C53F8081CE7
:1003680044F8081C53F8041C44F8041C161B2146C6
:100378001D46103410330F2EE8DC2B4602E02468AB
:1003880041F8044B551A1C46032D03F10403F6DC0F
:1003980090E700BF032AC9B270B408D82AB103464F
:1003A800121803F8011B9342FBD170BC70478218E6
:1003B800044601E004F8011B14F0030FFAD14FF0D2
:1003C800013303FB01F31FE044F8403C44F83C3C94
:1003D80044F8383C44F8343C44F8303C44F82C3C6D
:1003E80044F8283C44F8243C44F8203C44F81C3C9D
:1003F80044F8183C44F8143C44F8103C44F80C3CCD
:1004080044F8083C44F8043C161B254640343F2E6B
:10041800DADC2C4607E044F8103C44F80C3C44F87D
:10042800083C44F8043C161B254610340F2EF2DC19
:1004380001E045F8043B541B032CFADC01E005F805
:10044800011B9542FBD3B0E710F0030F38B5044603
:1004580012D10368A3F1013222EA030313F0803FAB
:100468000AD1031D184653F8042BA2F1013525EAD9
:10047800020212F0803FF5D003782BB1431C1846D6
:1004880013F8012B002AFAD100F076F9204638BD7E
:10049800C9B2F0B4002950D010F0030F10D003787F
:1004A800002B79D0994246D0431C05E013F8012B64
:1004B800002A3FD091423ED013F0030F1846F5D1E1
:1004C800036841EA01270646A3F1013247EA0747D4
:1004D80022EA030212F0803F1DD187EA0303A3F149
:1004E800013222EA030313F0803F14D1043002E002
:1004F80012F0803F0FD1064650F8043BA3F10135B6
:1005080087EA030225EA0303A2F1013413F0803FCE
:1005180024EA0202ECD033783046002B3CD09942D2
:1005280009D0731C01E0914205D0184613F8012B3D
:10053800002AF8D11046F0BC704710F0030F0CD019
:100548000378002BF7D0431C03E013F8012B002A93
:10055800F1D013F0030F1846F7D102680346A2F151
:10056800013121EA020212F0803F0AD10430034629
:1005780050F8042BA2F1013121EA020212F0803F67
:10058800F5D01A781846002AD5D00133184613F842
:10059800012B002AFAD1CEE71846CCE780EA0102FF
:1005A80012F0030F3AD110F0030220F0030021F0FB
:1005B800030150F804CB08BF51F8043B0DD082F07A
:1005C80003024FEAC2026FF07F4323FA02F251F8A6
:1005D800043B4CEA020C43EA020300BFACF10132CF
:1005E8009C4501BF22EA0C0212F0803F50F804CB70
:1005F80051F8043BF2D04FEA0C604FEA1C2C01285A
:1006080028BFB0EB036F08BF1B0AF4D003F0FF0349
:100618004FEA1060A0EB0300704700BF10F0030F13
:100628000AD010F8012B11F8013B012A28BF9A4281
:10063800F4D0A2EB030070474DF8045D4DF8044D6B
:100648004FF0010242EA022242EA024201F0030CA0
:1006580021F0030150F8044B51F8045BBCF1020F80
:1006680026D04BD824F07F4CBCEB152FA4EB02030B
:1006780023EA04030DD113EAC21308BF51F8045B3F
:100688000AD18CEA040CBCEB056F0CD150F8044B72
:10069800E8E74FEA15255CE033F07F4352D10D7847
:1006A8004FEA146C55E04FEA146C05F0FF0550E072
:1006B8004FEA044CA4EB02034FEA1C4C23EA040360
:1006C800BCEB154F17D113EAC21308BF51F8045BEE
:1006D80007D18CEA040CBCEB054F08D150F8044B49
:1006E800E6E71B042ED10D884FEA144C31E04FEA9F
:1006F80005454FEA144C4FEA15452AE004F0FF0C73
:10070800BCEB156FA4EB020323EA04030DD113EA33
:10071800C21308BF51F8045B0AD18CEA040CBCEB85
:10072800052F0AD150F8044BE8E74FEA156510E0A9
:1007380014F0FF0F06D051F8045B4FEA142C25F093
:100748007F4506E04FF000005DF8044B5DF8045B60
:1007580070470CF0FF0205F0FF00012828BF904207
:1007680004BF4FEA1C2C2D0AF3D0A2EB00005DF861
:10077800044B5DF8045B704780EA0102844612F07E
:10078800030F4FD111F0030F32D14DF8044D11F082
:10079800040F51F8043B0BD0A3F101329A4312F035
:1007A800803F04BF4CF8043B51F8043B16D100BF0E
:1007B80051F8044BA3F101329A4312F0803FA4F19F
:1007C80001320BD14CF8043BA24312F0803F04BF26
:1007D80051F8043B4CF8044BEAD023460CF8013B93
:1007E80013F0FF0F4FEA3323F8D15DF8044B70473D
:1007F80011F0010F06D011F8012B0CF8012B002A7B
:1008080008BF704711F0020FBFD031F8022B12F069
:10081800FF0F16BF2CF8022B8CF8002012F47F4F24
:10082800B3D1704711F8012B0CF8012B002AF9D12C
:10083800704700BF20F0030110F00300C0F1000072
:1008480051F8043B00F1040C4FEACC0C6FF00002A5
:100858001CBF22FA0CF213434FF0010C4CEA0C2C8B
:100868004CEA0C4CA3EB0C0222EA030212EACC126B
:1008780004BF51F8043B0430F4D013F0FF0F1FBF3E
:10088800013013F47F4F013013F47F0F18BF01308C
:10089800704700BFF0B4002A46D041EA000313F0C5
:1008A80003032CD1032A07460E4643D904680D6872
:1008B800AC423FD1043A37D0A4F1013525EA04040B
:1008C80014F0803F18BF18462CD1041D0D1D0EE0F2
:1008D80054F8043B55F8041BA3F101308B4220EA7D
:1008E800030027D1043A1FD010F0803F1ED1032AFD
:1008F80027462E46ECD820462946002A1DD00478E3
:10090800013A0D78AC420CD172B18CB1002302E0EF
:1009180093420BD064B1013310F8014FCD5CAC4267
:10092800F6D0601BF0BC70471046FBE70020F9E7E3
:100938002046F7E738463146E1E724782D78F0E796
:1009480041EA000313F0030F0B4670B414BF0024F0
:100958000124032A94BF002404F001040546D4B9F5
:10096800BAB10E782B46013A03F8016B56B1AC1CAC
:100978007AB111F8015F2346013A04F8015C0134A9
:10098800002DF5D12AB19A18002103F8011B9342D2
:10099800FBD170BC7047194653F8044BA4F10136DB
:1009A80026EA040616F0803FDAD1043A45F8044BEB
:1009B800032A1946EFD8D3E701232DE9F0071D468E
:1009C80000264FF0FF37AC1900EB070C8C420DD214
:1009D8001CF805C010F80480E0452ED201252646F3
:1009E800E31BAC198C4200EB070CF1D34FF0010963
:1009F80000264D464FF0FF3C1360AC1900EB0C0885
:100A0800A1420ED918F8058010F804A0C2451AD9D9
:100A180001252646CCEB0409AC19A14200EB0C08D1
:100A2800F0D80CF101000137B8423CBF994638466E
:100A3800C2F80090BDE8F00770470BD00123374695
:100A48001D46F618BFE709D04FF00109B4464D46D8
:100A58004E44D2E79D4205D00135B4E74D4505D057
:100A68000135CAE72B4626460125ACE7A9462646A6
:100A78000125C2E72DE9F04FADF5826D81B014462E
:100A8800074610460DF580628B460C3219461D4606
:100A9800FFF792FF03AE04A901F57E72331F0090A1
:100AA80043F8045F9342FBD14DB1681E0023E25C1A
:100AB800C11A013303AEAB4246F82210F7D1DDF874
:100AC8000C142046009A6118FFF78AFB002877D19A
:100AD8000099814605F1FF380646C1F101020192ED
:100AE8005A46AB4609EB0B0501F1FF3AB81800214D
:100AF800AA1A00F0E5F900284FD1002D00F0C080B7
:100B08007B1903A913F8013C51F82330002B4CD171
:100B1800009B9E4228BF334698450FD903EB090135
:100B2800E05C7A18795C884205D038E012F8011F39
:100B3800E05C884233D101339845F7D8009A964251
:100B480080F0A48007EB090214F80A10534612F843
:100B58000A20914204BF0AEB0901791807D095E0F1
:100B680014F802C011F8010D844503D113465A1E2A
:100B7800B342F5D101369E4200F28D80DDF80C6457
:100B88002A46B144C6EB0B0609EB0B05B818002141
:100B9800AA1A00F095F90028AFD0002071E0019A58
:100BA8000026914499442A46EEE7002EFAD0DDF853
:100BB8000C2493423CBFC2EB0B0306469944F2E770
:100BC800009E4FF000080099AB1BB34238BF334674
:100BD800C1F101026E1E019201F1FF3A5A4689469F
:100BE800AB460133CDF80C3408EB0B05B8180021DF
:100BF800AA1A00F065F90028CFD1002D40D07B1942
:100C080003A913F8013C51F82330002B30D1B1452A
:100C180013D208EB090314F80910FA18FB5C99427F
:100C280018BF4B4627D14B4604E012F8011FE05C81
:100C3800884220D10133B342F7D3BAF1FF3F53467C
:100C48002CD007EB080C14F80A101CF80A20914263
:100C58000CD10AEB0802BA1804E0E05C12F8011D96
:100C6800884203D1013BF8D260460AE0DDF80C3433
:100C780098442A46B8E701992A4688449844B3E735
:100C8800284605B00DF5806DBDE8F08F009B013654
:100C98009E427FF673AF07EB0900F2E707EB080CFB
:100CA8006046EEE72DE9F04F8346037885B00C46A1
:100CB800002B00F0F9800A78A2B106460131012024
:100CC80002E011F8012B8AB1934214BF002000F012
:100CD800010016F8013F0D46002BF2D12B782BB1FD
:100CE8004FF0000B584605B0BDE8F08F0028F9D149
:100CF8000BF101002178FFF7CBFB2D1BA5F10102B9
:100D0800534243EB0203002808BF43F001030746A0
:100D180083B90BEB0508404594BFC0EB08084FF0BA
:100D280001081F2D08D9414622462B46FFF7A2FE8F
:100D38008346D7E78346D5E7294603AA2046FFF727
:100D48003BFE03996118814620464A46FFF748FA58
:100D580000284FD109F1FF33C9F10102064601927B
:100D680082464246C84699460AEB050BB818002148
:100D7800C2EB0B0200F0A4F80028B1D1BBF1000FC0
:100D8800B0D046452CBF334643469D420FD903EBAE
:100D98000A01E05C7A18795C884205D075E012F89F
:100DA800011FE05C884270D101339D42F7D1B04504
:100DB8007DD907EB0A0214F809104B4612F80920EE
:100DC800914202BF09EB0A01AC46791806D06EE0E1
:100DD800A55C11F8010D854203D113465A1EB34292
:100DE800F6D1654601369E4267D8039E5A46B244FC
:100DF800AE1BB9E7C9F10101C9EB0503424600265C
:100E080009F1FF3A88464B4538BF4B4601330393F7
:100E180006EB050BB8180021C2EB0B0200F050F8E6
:100E280000287FF45DAFBBF1000F3FF45BAF4D4589
:100E380012D906EB090314F80910FA18FB5C994259
:100E480008BF4B4605D026E012F8011FE05C884237
:100E580022D101339D42F7D1BAF1FF3F534628D042
:100E680007EB060C14F80A101CF80A20914217D157
:100E78000AEB0602BA1804E0E05C12F8011D884289
:100E88000ED1013BF8D2E3462CE7019A00269244A2
:100E98005A469A4468E74B4646445A46F618B7E716
:100EA800039B5A46F618B3E70D46012016E743465A
:100EB80098E707EB060CE34614E707EB0A0B11E784
:100EC80010F0030F034670B4C9B211D0002A22D023
:100ED80003788B421DD0013A013005E0DAB110F8F1
:100EE800014B013A8C4218D010F0030F0346F5D19C
:100EF800032A14D87AB1187888420ED0541E5D1C83
:100F080003E015F8016B8E4203D0013C2846F8D265
:100F1800002070BC70471046FBE71846F9E741EA25
:100F2800012646EA0646184653F8044B86EA0404A6
:100F3800A4F1013525EA040414F0803F03D1043AF2
:100F48001846032AEFD80346D4E700BF0000000084
:100F5800C1F30A5C0246ACF57E7C2DE9F84FACF192
:100F68000704132C0B4606460F468946804627DCA5
:100F7800002C52DB4FF6FF7CC0F20F0C4CFA04FA3F
:100F88000AEA0105054317D037A3D3E9002300F087
:100F980075F80022002300F0B3FC002856D0002F7B
:100FA80005DD4FF4801353FA04F407EB040929EA2A
:100FB8000A0900264B46324610461946BDE8F88F06
:100FC800332C07DDB4F5806FF6D100F057F80246F0
:100FD8000B46F1E74FF0FF3BACF11B0C2BFA0CFB77
:100FE8001BEA000FE8D020A3D3E9002300F046F85D
:100FF8000022002300F084FC40B3002F0ADD142CEB
:1010080006D00126C4F13404A64016EB080601D325
:1010180007F1010926EA0B0619E013A3D3E9002317
:1010280000F02CF80022002300F06AFC78B1002FB1
:1010380013DB46EA07054FF000094D45C3F6F07982
:101048000CBF2E46002608BFA94600E0B9464B460D
:10105800324610461946BDE8F88F00264FF0004981
:10106800F5E700BFAFF300809C7500883CE4377E4D
:1010780081F0004102E000BF83F0004330B54FEA41
:1010880041044FEA430594EA050F08BF90EA020FAE
:101098001FBF54EA000C55EA020C7FEA645C7FEA41
:1010A800655C00F0E2804FEA5454D4EB5555B8BF64
:1010B8006D420CDD2C4480EA020281EA030382EAD5
:1010C800000083EA010180EA020281EA0303362D67
:1010D80088BF30BD11F0004F4FEA01314FF4801C3A
:1010E8004CEA113102D0404261EB410113F0004F4C
:1010F8004FEA03334CEA133302D0524263EB430303
:1011080094EA050F00F0A780A4F10104D5F1200EA0
:101118000DDB02FA0EFC22FA05F2801841F10001FB
:1011280003FA0EF2801843FA05F359410EE0A5F1CF
:1011380020050EF1200E012A03FA0EFC28BF4CF000
:10114800020C43FA05F3C01851EBE37101F00045B6
:1011580007D54FF0000EDCF1000C7EEB00006EEBC3
:101168000101B1F5801F1BD3B1F5001F0CD349084D
:101178005FEA30004FEA3C0C04F101044FEA4452A4
:1011880012F5800F80F09A80BCF1004F08BF5FEA2B
:10119800500C50F1000041EB045141EA050130BD0B
:1011A8005FEA4C0C404141EB010111F4801FA4F1AE
:1011B8000104E9D191F0000F04BF01460020B1FA03
:1011C80081F308BF2033A3F10B03B3F120020CDA3B
:1011D8000C3208DD02F1140CC2F10C0201FA0CF019
:1011E80021FA02F10CE002F11402D8BFC2F1200C7E
:1011F80001FA02F120FA0CFCDCBF41EA0C01904034
:10120800E41AA2BF01EB0451294330BD6FEA04047C
:101218001F3C1CDA0C340EDC04F11404C4F1200267
:1012280020FA04F001FA02F340EA030021FA04F379
:1012380045EA030130BDC4F10C04C4F1200220FAD0
:1012480002F001FA04F340EA0300294630BD21FA0E
:1012580004F0294630BD94F0000F83F4801306BFD4
:1012680081F480110134013D4EE77FEA645C18BFC8
:101278007FEA655C29D094EA050F08BF90EA020F5F
:1012880005D054EA000C04BF1946104630BD91EA57
:10129800030F1EBF0021002030BD5FEA545C05D15A
:1012A8004000494128BF41F0004130BD14F5800499
:1012B8003CBF01F5801130BD01F0004545F0FE410D
:1012C80041F470014FF0000030BD7FEA645C1ABF42
:1012D800194610467FEA655C1CBF0B46024650EA79
:1012E800013406BF52EA033591EA030F41F40021A5
:1012F80030BD00BF90F0000F04BF0021704730B52B
:101308004FF4806404F132044FF000054FF00001FF
:1013180050E700BF90F0000F04BF0021704730B5C0
:101328004FF4806404F1320410F0004548BF404295
:101338004FF000013EE700BF42004FEAE2014FEAEA
:1013480031014FEA02701FBF12F07F4393F07F4FC5
:1013580081F06051704792F0000F14BF93F07F4FF7
:10136800704730B54FF4607401F0004521F000413A
:1013780020E700BF50EA010208BF704730B54FF0C0
:1013880000050AE050EA010208BF704730B511F0C5
:10139800004502D5404261EB41014FF4806404F1FD
:1013A80032045FEA915C3FF4DCAE4FF003025FEA7F
:1013B800DC0C18BF03325FEADC0C18BF033202EB07
:1013C800DC02C2F1200300FA03FC20FA02F001FA61
:1013D80003FE40EA0E0021FA02F11444C1E600BF00
:1013E80070B54FF0FF0C4CF4E06C1CEA11541DBFB3
:1013F8001CEA135594EA0C0F95EA0C0F00F0DEF87E
:101408002C4481EA030621EA4C5123EA4C5350EA62
:10141800013518BF52EA033541F4801143F48013B3
:1014280038D0A0FB02CE4FF00005E1FB02E506F044
:101438000042E0FB03E54FF00006E1FB03569CF099
:10144800000F18BF4EF0010EA4F1FF04B6F5007F9F
:1014580064F5407404D25FEA4E0E6D4146EB060611
:1014680042EAC62141EA55514FEAC52040EA5E509A
:101478004FEACE2EB4F1FD0C88BFBCF5E06F1ED844
:10148800BEF1004F08BF5FEA500E50F1000041EB7B
:10149800045170BD06F0004646EA010140EA020028
:1014A80081EA0301B4EB5C04C2BFD4EB0C0541EA4A
:1014B800045170BD41F480114FF0000E013C00F35F
:1014C800AB8014F1360FDEBF002001F0004170BD83
:1014D800C4F10004203C35DA0C341BDC04F114049C
:1014E800C4F1200500FA05F320FA04F001FA05F228
:1014F80040EA020001F0004221F0004110EBD370F5
:1015080021FA04F642EB06015EEA430E08BF20EA20
:10151800D37070BDC4F10C04C4F1200500FA04F3C3
:1015280020FA05F001FA04F240EA020001F0004155
:1015380010EBD37041F100015EEA430E08BF20EAC8
:10154800D37070BDC4F1200500FA05F24EEA020E10
:1015580020FA04F301FA05F243EA020321FA04F03F
:1015680001F0004121FA04F220EA020000EBD370F6
:101578005EEA430E08BF20EAD37070BD94F0000FF6
:101588000FD101F00046400041EB010111F4801F2A
:1015980008BF013CF7D041EA060195F0000F18BFDB
:1015A800704703F00046520043EB030313F4801F17
:1015B80008BF013DF7D043EA0603704794EA0C0FD1
:1015C8000CEA135518BF95EA0C0F0CD050EA4106E7
:1015D80018BF52EA4306D1D181EA030101F0004164
:1015E8004FF0000070BD50EA410606BF104619468C
:1015F80052EA430619D094EA0C0F02D150EA013698
:1016080013D195EA0C0F05D152EA03361CBF1046D8
:1016180019460AD181EA030101F0004141F0FE4177
:1016280041F470014FF0000070BD41F0FE4141F4FB
:10163800780170BD70B54FF0FF0C4CF4E06C1CEAFB
:1016480011541DBF1CEA135594EA0C0F95EA0C0FB0
:1016580000F0A7F8A4EB050481EA030E52EA03356B
:101668004FEA013100F088804FEA03334FF080558C
:1016780045EA131343EA12634FEA022245EA1115B9
:1016880045EA10654FEA00260EF000419D4208BF6A
:10169800964244F1FD0404F5407402D25B084FEA17
:1016A8003202B61A65EB03055B084FEA32024FF4C3
:1016B80080104FF4002CB6EB020E75EB030E22BF20
:1016C800B61A754640EA0C005B084FEA3202B6EBE0
:1016D800020E75EB030E22BFB61A754640EA5C008F
:1016E8005B084FEA3202B6EB020E75EB030E22BF1F
:1016F800B61A754640EA9C005B084FEA3202B6EB20
:10170800020E75EB030E22BFB61A754640EADC00DE
:1017180055EA060E18D04FEA051545EA16754FEA40
:1017280006164FEAC30343EA52734FEAC2025FEA5E
:101738001C1CC0D111F4801F0BD141EA00014FF0ED
:1017480000004FF0004CB6E711F4801F04BF0143BE
:101758000020B4F1FD0C88BFBCF5E06F3FF6AFAEDA
:10176800B5EB030C04BFB6EB020C5FEA500C50F16A
:10177800000041EB045170BD0EF0004E4EEA1131ED
:1017880014EB5C04C2BFD4EB0C0541EA045170BDF4
:1017980041F480114FF0000E013C90E645EA060E38
:1017A8008DE60CEA135594EA0C0F08BF95EA0C0F66
:1017B8003FF43BAF94EA0C0F0AD150EA01347FF4AE
:1017C80034AF95EA0C0F7FF425AF104619462CE785
:1017D80095EA0C0F06D152EA03353FF4FDAE1046E8
:1017E800194622E750EA410618BF52EA43067FF439
:1017F800C5AE50EA41047FF40DAF52EA43057FF4C9
:10180800EBAE12E74FF0FF3C06E000BF4FF0010CD3
:1018180002E000BF4FF0010C4DF804CD4FEA410C37
:101828007FEA6C5C4FEA430C18BF7FEA6C5C1BD004
:1018380001B050EA410C0CBF52EA430C91EA030F85
:1018480002BF90EA020F0020704710F1000F91EAE2
:10185800030F58BF994208BF90422CBFD8176FEAB0
:10186800E37040F0010070474FEA410C7FEA6C5C7E
:1018780002D150EA013C07D14FEA430C7FEA6C5C85
:10188800D6D152EA033CD3D05DF8040B704700BFB1
:101898008446104662468C461946634600E000BFFF
:1018A80001B5FFF7B7FF002848BF10F1000F01BDD1
:1018B8004DF808EDFFF7F4FF0CBF012000205DF89C
:1018C80008FB00BF4DF808EDFFF7EAFF34BF012021
:1018D80000205DF808FB00BF4DF808EDFFF7E0FFBA
:1018E80094BF012000205DF808FB00BF4DF808ED0B
:1018F800FFF7CEFF94BF012000205DF808FB00BF72
:101908004DF808EDFFF7C4FF34BF012000205DF853
:1019180008FB00BF4FEA4102B2F1E04324BFB3F530
:10192800001CDCF1FE5C0DD901F0004C4FEAC0024E
:101938004CEA5070B2F1004F40EB830008BF20F032
:101948000100704711F0804F21D113F13872BCBFEC
:1019580001F00040704741F480114FEA5252C2F141
:101968001802C2F1200C10FA0CF320FA02F018BF8A
:1019780040F001004FEAC1234FEAD32303FA0CFCDD
:1019880040EA0C0023FA02F34FEA4303CCE77FEA6C
:10199800625307D150EA01331EBF4FF0FE4040F4B6
:1019A8004000704701F0004040F0FE4040F4000065
:1019B800704700BF80F0004002E000BF81F00041A6
:1019C80042001FBF5FEA410392EA030F7FEA226CDD
:1019D8007FEA236C6AD04FEA1262D2EB1363C1BF6D
:1019E800D218414048404140B8BF5B42192B88BFDC
:1019F800704710F0004F40F4000020F07F4018BFFF
:101A0800404211F0004F41F4000121F07F4118BF1E
:101A1800494292EA030F3FD0A2F1010241FA03FCC6
:101A280010EB0C00C3F1200301FA03F100F00043AE
:101A380002D5494260EB4000B0F5000F13D3B0F176
:101A4800807F06D340084FEA310102F10102FE2AE5
:101A580051D2B1F1004F40EBC25008BF20F0010055
:101A680040EA03007047490040EB000010F4000F03
:101A7800A2F10102EDD1B0FA80FCACF1080CB2EB96
:101A88000C0200FA0CF0AABF00EBC25052421843F5
:101A9800BCBFD0401843704792F0000F81F400019A
:101AA80006BF80F400000132013BB5E74FEA41036D
:101AB8007FEA226C18BF7FEA236C21D092EA030FD9
:101AC80004D092F0000F08BF0846704790EA010F53
:101AD8001CBF0020704712F07F4F04D1400028BF80
:101AE80040F00040704712F100723CBF00F5000062
:101AF800704700F0004343F0FE4040F40000704798
:101B08007FEA226216BF08467FEA23630146420243
:101B180006BF5FEA412390EA010F40F48000704756
:101B28004FF0000304E000BF10F0004348BF4042FC
:101B38005FEA000C08BF704743F0964301464FF038
:101B480000001CE050EA010208BF70474FF0000394
:101B58000AE000BF50EA010208BF704711F00043D5
:101B680002D5404261EB41015FEA010C02BF8446A5
:101B78000146002043F0B64308BFA3F18053A3F504
:101B88000003BCFA8CF2083AA3EBC25310DB01FA4B
:101B980002FC634400FA02FCC2F12002BCF1004FCF
:101BA80020FA02F243EB020008BF20F00100704760
:101BB80002F1200201FA02FCC2F1200250EA4C00B4
:101BC80021FA02F243EB020008BF20EADC707047FA
:101BD8004FF0FF0C1CEAD0521EBF1CEAD15392EA08
:101BE8000C0F93EA0C0F6FD01A4480EA010C4002E4
:101BF80018BF5FEA41211ED04FF0006343EA50103E
:101C080043EA5111A0FB01310CF00040B1F5000F7F
:101C18003EBF490041EAD3715B0040EA010062F12E
:101C28007F02FD2A1DD8B3F1004F40EBC25008BF18
:101C380020F00100704790F0000F0CF0004C08BF36
:101C480049024CEA502040EA51207F3AC2BFD2F103
:101C5800FF0340EAC250704740F400004FF0000311
:101C6800013A5DDC12F1190FDCBF00F0004070474B
:101C7800C2F10002410021FA02F1C2F1200200FA89
:101C880002FC5FEA310040F1000053EA4C0308BF50
:101C980020EADC70704792F0000F00F0004C02BFA1
:101CA800400010F4000F013AF9D040EA0C0093F01C
:101CB800000F01F0004C02BF490011F4000F013B76
:101CC800F9D041EA0C018FE70CEAD15392EA0C0FE4
:101CD80018BF93EA0C0F0AD030F0004C18BF31F04F
:101CE800004CD8D180EA010000F00040704790F025
:101CF800000F17BF90F0004F084691F0000F91F0C9
:101D0800004F14D092EA0C0F01D142020FD193EA8E
:101D18000C0F03D14B0218BF084608D180EA010016
:101D280000F0004040F0FE4040F40000704740F0F2
:101D3800FE4040F4400070474FF0FF0C1CEAD052C0
:101D48001EBF1CEAD15392EA0C0F93EA0C0F69D01C
:101D5800A2EB030280EA010C49024FEA402037D087
:101D68004FF0805343EA111143EA10130CF000407E
:101D78008B4238BF5B0042F17D024FF4000C8B426E
:101D880024BF5B1A40EA0C00B3EB510F24BFA3EB4E
:101D9800510340EA5C00B3EB910F24BFA3EB91031E
:101DA80040EA9C00B3EBD10F24BFA3EBD10340EA78
:101DB800DC001B0118BF5FEA1C1CE0D1FD2A3FF6BE
:101DC80050AF8B4240EBC25008BF20F00100704773
:101DD8000CF0004C4CEA50207F32C2BFD2F1FF0316
:101DE80040EAC250704740F400004FF00003013A47
:101DF80037E792F0000F00F0004C02BF400010F4EB
:101E0800000F013AF9D040EA0C0093F0000F01F0FE
:101E1800004C02BF490011F4000F013BF9D041EA20
:101E28000C0195E70CEAD15392EA0C0F08D1420253
:101E38007FF47DAF93EA0C0F7FF470AF084676E726
:101E480093EA0C0F04D14B023FF44CAF08466EE7FF
:101E580030F0004C18BF31F0004CCAD130F00042CD
:101E68007FF45CAF31F000437FF43CAF5FE700BF25
:101E78004FF0FF3C06E000BF4FF0010C02E000BF4E
:101E88004FF0010C4DF804CD4FEA40024FEA4103F0
:101E98007FEA226C18BF7FEA236C11D001B052EAA6
:101EA800530C18BF90EA010F58BFB2EB030088BF6C
:101EB800C81738BF6FEAE17018BF40F001007047DB
:101EC8007FEA226C02D15FEA402C05D17FEA236CBD
:101ED800E4D15FEA412CE1D05DF8040B704700BF04
:101EE800844608466146FFE70FB5FFF7C9FF00289B
:101EF80048BF10F1000F0FBD4DF808EDFFF7F4FFD4
:101F08000CBF012000205DF808FB00BF4DF808ED6C
:101F1800FFF7EAFF34BF012000205DF808FB00BF8F
:101F28004DF808EDFFF7E0FF94BF012000205DF8B1
:101F380008FB00BF4DF808EDFFF7D2FF94BF012062
:101F480000205DF808FB00BF4DF808EDFFF7C8FF5B
:101F580034BF012000205DF808FB00BF42000ED20C
:101F6800B2F1FE4F0BD34FF09E03B3EB126209D4CC
:101F78004FEA002343F0004323FA02F070474FF082
:101F88000000704712F1610F01D1420202D14FF0F7
:101F9800FF3070474FF00000704700BF00F026F890
:101FA8000C4880F30888002103E00B4B5B58435032
:101FB80004310A480A4B42189A42F6D3094A02E009
:101FC800002342F8043B084B9A42F9D317F086FBEA
:101FD8007047000000C0002098350308000000206A
:101FE800600E0020600E0020684200207047FEE767
:101FF80010B586B0002301244FF46022114801A9CE
:1020080001938DF80930039204938DF808408DF8F8
:10201800144021F0A7F90B48214621F0C9F90948D5
:1020280021F0D0F9074821F0D2F90028FAD1054863
:1020380021F0D1F9034821F0D3F90028FAD106B0EC
:1020480010BD00BF00240140014610B50D48012213
:10205800032321F0D3F90B48012121F0C5F97F2092
:1020680022F002F80748022121F012FA0028F6D0DF
:102078000448022121F012FA0248BDE8104021F07C
:1020880004BA00BF002401400C4A0C2303FB0123BF
:1020980010B59C880CB9588010BD5B8803F11304F7
:1020A800844204DA142B07D9133B834204DC0C2343
:1020B80003FB012102238B8010BD00BFBC2500203B
:1020C8000A4B10B500241C7021464FF4E0720848F2
:1020D800FEF760F9074B4FF474501C70064B1C70E8
:1020E8000EF04AFE054B187010BD00BFDC10002032
:1020F800A8120020F314002070140020721400208D
:10210800074B1978013101F01F011970054B1A7836
:102118008A4203D1013202F01F021A70704700BFD1
:1021280070140020F314002010B50E4A0E2303FB90
:1021380000200D4A014614780C4A03FB042300F1E1
:102148000C0251F8044B914243F8044BF9D10A8828
:1021580000211A800E22FEF71DF9BDE81040FFF796
:10216800CFBF00BFE010002070140020A81200208C
:10217800084B1A5C002352FA03F111F0010FD8B290
:1021880002D00130C0B270470133042BF3D10120D3
:10219800704700BF9D15002000F07F0000F57450C7
:1021A8002DE9F84305300C46154698460EF0E4FD37
:1021B80000284ED043F63837002638460EF0DCFDAE
:1021C800C0B25FFA86F988B120280FD04FEA5909C2
:1021D8004AF20B5048440EF0CFFDC0B208B10228B5
:1021E80004D10123B34022781343237011370136F9
:1021F800B7F56F5FE1D14AF2B2300EF0BDFDC0B263
:1022080080B120280ED02B784AF2A13043F0010388
:102218002B700EF0B1FDC0B220B1202802D00123EE
:1022280088F800304AF2E3300EF0A6FDC0B280B163
:1022380020280ED02B784AF2A13043F002032B70ED
:102248000EF09AFDC0B220B1202802D0012388F8F0
:102258000030BDE8F8830000034610465A1E10B54A
:10226800032A1CD8DFE802F00E0E0207114A527842
:1022780002F0100203E00F4A527802F00802D2B2CC
:1022880072B10BE00C4A927802F04002D2B23AB135
:102298000A4A127802F003029A4200D140B10022A1
:1022A8000748105C984203D00132052AF8D1002172
:1022B800084610BD78400020C0310020733400204B
:1022C800A0120020F8B5064643F638350024284603
:1022D8000EF052FDC0B2E7B268B120280BD07F08DB
:1022E8004AF20B5038180EF047FD012803D1A040E0
:1022F80033781843307001341135082CE7D1F8BD14
:1023080003780E2202FB0313084AD3189978002396
:1023180051FA03F010F00100DAB202D0501CC0B23A
:1023280070470133082BF3D1704700BFA812002073
:102338002DE9F04101248C40284A29490346E4B29A
:10234800107891F800C019E0264F0E2606FB00769B
:10235800F178A9B996F80680B8F1000F10D196F86F
:102368000580B8F1000F0BD196F80480B8F1000F82
:1023780006D1F67926B9013000F01F00054626E09F
:10238800FBB1012B05D0022B06D10E2101FB0077F2
:1023980039790C4218D014E0042B04D10E2101FB2A
:1023A8000077B9790CE0032B04D10E2101FB0077EB
:1023B800797905E0052B07D10E2101FB0077F97922
:1023C80011B11570BDE8F081013000F01F006045C3
:1023D800BAD11570FF20BDE8F08100BFF3140020CA
:1023E80070140020A81200202DE9F043434D444BFF
:1023F8002A780E2101FB0232917A85B0044698466C
:1024080031B101390523594301F56F5189B201E012
:102418004FF46F51204604220EF0BFFC2B780E2596
:1024280005FB038393F80B80354E344FB8F1000F4A
:1024380025D131232371073363713B7801A86B439E
:102448000422F15E06F014FA3B7802A805FB036348
:102458000222997A06F00CFA3B780DF10A0005FB86
:1024680003650322697A06F003FAA01D01A909226F
:10247800FEF766FA4FF00F0984F8108012E0B8F101
:10248800010F0FD132232371053363713B784FF06D
:10249800080905FB036393F90130E3713B785D4359
:1024A800735BA371002320461A4612E010F8011B43
:1024B800A1F13005EDB2092D04D8EB183029DBB2B3
:1024C80003D004E037395B1800E00A33DBB201328D
:1024D800D2B24A45EAD10F21B3FBF1F10801411A02
:1024E8005B1AC3F10F03DBB2092BA35401D83033B5
:1024F80000E03733A35405B0BDE8F083A6120020EE
:10250800A8120020024B1A7842F001021A70704794
:10251800D517002008B50C4B0C4A1B780E2101FB7F
:102528000323D97A21B101290CBF0921002100E038
:10253800102140221346064805F0BEFF054B1A78C5
:1025480042F002021A7008BDA6120020A81200204C
:1025580073140020D5170020034B1A7802F0F802F4
:102568006FF3C3021A707047D5170020024B1A7810
:1025780042F004021A707047D5170020024B1A78EF
:1025880042F008021A707047D517002038B5114B71
:102598001C7814F0010502D1FFF7B4FF05E004F040
:1025A8000405EDB21DB9FFF7E1FF284638BD04F078
:1025B8000805EDB215B9FFF7E1FFF6E704F00204EC
:1025C800E4B21CB9FFF7A6FF204638BDFFF7C4FFE9
:1025D800012038BDD5170020014B1878704700BF7F
:1025E800DC10002030B51E4B85B01B780446002B4C
:1025F80034D11C4D2B78034113F0010F2ED01A4B08
:102608001A4A1B780E2101FB0323DA78024112F0E3
:10261800010F1CD11B79034113F0010317D110F0EE
:10262800010001F1F1014FEA540206D00132009194
:10263800019302926D20FE3905E00132009101906C
:1026480002923C20012103220B460EF013FC0123C9
:1026580013FA04F42B7823EA04042C7005B030BD77
:102668007214002069140020F3140020A81200201E
:10267800037830B513F0010F144A4FF00E0419D146
:1026880004FB01210133012212FA03F3CD7825EA74
:102698000303CB7004780D79A41812FA04F425EA20
:1026A80004040C7103789B189A408B7823EA020281
:1026B8008A7030BD04FB0121013B012212FA03F3A9
:1026C8008A7822EA03038B7030BD00BFA81200206D
:1026D80010B500230278590052FA01F404F00304FB
:1026E800022C05D1013414FA01F122EA0102027028
:1026F8000133042BEED110BD2DE9F04F85B00192C6
:10270800BDF838201C46734B0092DA78054612F063
:1027180020028B4640F0D8808DF80E208DF80F20CF
:102728008DF80D20DCB99B7803F04003DBB21BB1B8
:1027380001238DF80F3020E0674B5B7803F002032C
:10274800DBB21BB101238DF80E3016E00DF10F013D
:102758000DF10E020DF10D03FFF71EFD0DE0012C2A
:102768000BD19B7803F04003DBB223B90DF10F00C6
:10277800FFF7A8FD01E08DF80F409DF80F3023B951
:102788009DF80E00002800F0A28044B905F07F01F2
:10279800490001F574510DF10A00623109E0012C7C
:1027A8000AD1E90101F50C413C310DF10A0001EBB8
:1027B8004B0102220EF0F1FABDF90A3013B9002CD0
:1027C80000F08480009B33B9444B454F93F8008058
:1027D800FFF796FC08E0434B434F93F8008008F15D
:1027E800010202F01F021A700DF10F00FFF770FFCF
:1027F800002C44D1BDF80A3069B240F6B83212EA6A
:10280800210238BF4FF47A72D2180E2303FB08F363
:10281800ADF80A20FA529DF80F9022464946012049
:10282800FE18FFF719FD4946F07022460220FFF70F
:1028380013FD86F8029030719DF80E9022464946A5
:102848000420FFF709FD4946B0718246224603205D
:10285800FFF702FD05F07F0570713572BAF1000FC0
:1028680000D128B1214B1B7813B99DF80D3000E039
:102878000023F37186F809B0019AB2721CE0012CAA
:102888001AD10E2303FB08F3BDF80A202046FA529A
:102898009DF80F6000223146FD18FFF7DDFC314638
:1028A800E87000220220FFF7D7FC00232871AE70E1
:1028B800AB716B71EB71AB720E2303FB0877FC7283
:1028C800009B0120BB8102E0002000E0204605B00B
:1028D800BDE8F08FC031002078400020701400203F
:1028E800A8120020DB100020E0100020BA170020FA
:1028F80073B5154B04461B780E46D3B113482146D1
:102908001FF0D7FE0546A0B9012E04F1010606D135
:102918002046FFF72DFC00950246812005E0204661
:10292800FFF726FC00950246982031462B46FFF714
:10293800E3FE214605481FF0A6FE0548214602B0E1
:10294800BDE870401FF0AABE71140020D816002000
:10295800001500202DE9F7437B4B04461B7843B153
:102968007A4B1B7803F02403042B02D1002900F0D2
:10297800E880774B774F1B78002B00F0C7807648AC
:1029880021461FF096FE002840F0C08007F5C4706D
:1029980021461FF08EFE8046002840F0B7803B1984
:1029A80093F880302D2B01D0532B3AD16B4E3578CC
:1029B80045B30EF055FD04F10108054650B1204617
:1029C800FFF7D6FB337802461E3300939320414627
:1029D800002307E02046FFF7CBFB0095024641465F
:1029E80093202B46FFF788FE0EF03AFD014628B1EA
:1029F800337803201E330093002101E00090032068
:102A08000A4680E02046FFF7B3FB611C02462B46CE
:102A180093200095FFF770FE0095032029462A466B
:102A280071E0542B09D12046FFF7A2FBCDF80080B6
:102A38000246611C9420434666E0462B474D20D150
:102A48002E78BEB10EF00CFD04F10109064648B11E
:102A58002046FFF78DFB2B7802461E3300939A2001
:102A6800494622E02046FFF783FB00960246494686
:102A78009A2025E02046FFF77BFB009602469A2025
:102A880039E02E78002E2CD00EF0EAFC04F11C0957
:102A9800064660B12046FFF76BFB2B7802461E33D3
:102AA80069F07F000093C0B2611C434609E02046EC
:102AB800FFF75EFB024669F07F000096C0B2611C1A
:102AC8003346FFF719FE0EF0CBFC21B2024628B1BF
:102AD8002B7803201E330093002214E0009003207B
:102AE80011E02046FFF744FB024604F11C0060F0A9
:102AF8007F000096C0B2611C3346FFF7FDFD0096CB
:102B08000320214632460123FFF7F6FD12482146ED
:102B18003F191FF0B8FD97F880302D2B0AD0532BA2
:102B280008D0542B06D0462B04D00D4821461FF060
:102B3800C0FD30B10B48214603B0BDE8F0431FF09B
:102B4800ADBD03B0BDE8F083DE100020C61600203E
:102B580071140020E8230020D81600203017002028
:102B680070250020D0160020002302780E2101FBDA
:102B78000232044901338A180021062B9170F4D1DE
:102B8800704700BFA8120020064B00201870064BA3
:102B98001A78064B1B789A4202D00146FFF7C8BB49
:102BA800FF207047DC10002070140020F314002070
:102BB8000121814038B5114BC9431A78104BC9B26D
:102BC80002F0030203F5E074012A04D1DD7801EA7A
:102BD8000505DD7005E0022A03D11D7901EA050526
:102BE8001D710E33A342EFD1FFF7FCFC4FF4745074
:102BF8000EF0C2F8034B187038BD00BF73340020C4
:102C0800A8120020721400202DE9F743A34D8DF877
:102C180007002B78A24C1BB12378C2B29A4204D089
:102C28004FF474500EF0A8F828709DF80730237000
:102C38009C4C2278072A00F22D81DFE812F0080068
:102C48002400360054005D0072008D00BA00964AD8
:102C58003C211170954A1946107800F00300FFF7DF
:102C680067FB934BFF28187000F036811EF022FA9C
:102C7800904B002093F8742042F0010283F87420EE
:102C88008D4B187064E0884B1B78002B00F0248172
:102C98001EF0D8FB012840F04D812378142201331F
:102CA8002370864B01381A7047E17F4B1B78002B45
:102CB80000F01281814E307808B901234AE01EF0F5
:102CC800C1FB022804D01EF0BDFB032840F032816E
:102CD8001EF0F0F923780422013323701D2333708A
:102CE800774B1A7026E1704B3C221A707548FFF733
:102CF8007BFB2378013323706B4B1B78002B00F090
:102D0800EB806E4B1D78002D40F014811020FFF7EA
:102D18003DFC002800F011812378284601332370F8
:102D28000BE1614B1B78002B00F0D68005F02EFCE0
:102D3800002800F00281614B7D221A705E4B002052
:102D480018705C4B93F8742042F0010283F87420E9
:102D5800237801332370F0E0534B1B78002B00F0ED
:102D6800BB801EF06FFB0128544E03D01EF06AFB97
:102D780003280FD19DF80720012111FA02F2524BC6
:102D8800197821EA02021A70642333702378013318
:102D98002370CFE03078002840F0CC80484A0323E5
:102DA80023701378013BDBB21370002B00F0948082
:102DB800C3E0404A414E92F86A201AB13278002A9C
:102DC80040F0B88000223270013212FA03F3DFF8C3
:102DD800E0803E4F98F800104FF00E0909FB017291
:102DE800DB4392F803E0DBB203EA0E0E907882F838
:102DF80003E092F804E003EA0E0E0340937082F8B1
:102E080004E00DF10700FFF733FC98F8003009FBE8
:102E18000372D278DFF894902AB999F8002002F06A
:102E28000302012A0AD00E2202FB03721279B2B9F8
:102E380099F8002002F00302022A10D10E2202FBA8
:102E48000377BA785AB9224F3A789A4207D1184884
:102E5800FFF78AFE3B78013303F01F033B7099F8B4
:102E680000009DF8071000F00300FFF761FA144B0B
:102E78000422FF281A7088F80000164B42D0987870
:102E880000F04000C0B200283CD1032323701A335D
:102E9800337052E0002020704FE000BF7214002011
:102EA800DF100020DC1000206A140020733400209A
:102EB800A6120020F8330020DD100020DA100020D0
:102EC800681400207314002069140020A812002040
:102ED800F3140020C0310020FFF73EFB00232370CD
:102EE8001EF0E8F82B78013BDBB22B702BB1144BAA
:102EF8009B7803F04003DBB2F3B19DF80700FFF7BE
:102F080057FE19E09B780E4A03F04003DBB22BB161
:102F1800136843F400031360FFF7D2F8FFF71CFBB4
:102F28001EF0C8F8002323704FF474500DF024FFEE
:102F3800287001E0002000E0FF20BDE8FE8300BF0C
:102F4800C0310020044B1A780AB1013A1A701B7874
:102F58000BB9FFF72DBE704772140020044A054BC9
:102F680010781B7803EA501000F00100704700BF8A
:102F7800C03100209F160020044B054A1B781078AA
:102F8800C3F3400303EA1010704700BF9F160020E8
:102F9800C0310020034B044A1B78D078C3F3800368
:102FA800184070479F160020C0310020044B054A86
:102FB8001B78D078C3F3C00303EA5000704700BF02
:102FC8009F160020C0310020044B054A1B78D0789A
:102FD800C3F3001303EA9000704700BF9F16002058
:102FE800C0310020044B1878044BDB785B005BB2DF
:102FF800DB1103EAD01070479F160020C031002073
:103008002DE9F041154E0024B04620E0204629461F
:103018001BF000F890B1F35DFF2B0FD04FF4A073B5
:1030280063430A2202FB053318F80330DB0905D095
:103038000B4B1878C0F30010BDE8F08101350A3752
:10304800202DE3D10134022C06F5A07602D000270A
:103058003D46DBE70020BDE8F08100BF4535002094
:103068009F16002008B51AF0D7FB034B1B7800EA1F
:10307800931000F0010008BD9F160020044B054A7C
:103088001B78D078C3F3401303EAD000704700BF21
:103098009F160020C03100202DE9F84FFFF75EFF92
:1030A8008146FFF769FF8246FFF774FF8346FFF703
:1030B8007DFF8046FFF788FF0446FFF7A1FF05461E
:1030C800FFF7DCFF0746FFF7CDFF0646FFF78AFF4D
:1030D8004FEA8B0343EA4A0343EA090343EAC80376
:1030E80043EA471343EA861345EA040443EAC01354
:1030F800E0B243EA0010BDE8F88F0000044B98786E
:1031080000F00F00A0F10203584240EB03007047A3
:103118003D150020044B987800F00F00A0F1010243
:10312800504240EB020070473D150020044B987850
:1031380000F00F00A0F10301484240EB0100704786
:103148003D150020054B987800F00F00A0F1060C03
:10315800DCF1000040EB0C00704700BF3D1500207B
:10316800514AF0B513781446012B29D003D3022B0A
:1031780040F098805EE04D484D4B047819786FF325
:10318800C304047001F0F80158786FF3C301197093
:1031980000F08001C9B2002900F08480012111707B
:1031A8009C78062204F00F04544302464148005D0F
:1031B80060F306025A701A7861F302021A70F0BDC1
:1031C8003B494D780B4625F07F00002838D00A7817
:1031D80002F00802D2B222B9344A117841F008014B
:1031E80011709A7802F00F02012A04D12F4A11783F
:1031F80041F00101117015F07F0F53D119789E78B5
:1032080001F00700062206F00F0602FB0606294F0A
:103218005D78BE5D013066F3060500F007005D705D
:1032280090FBF2F502FB150262F30201197002230A
:103238002370F0BD1E494D780B4625F07F0028B954
:103248008B7860F303038B701070F0BD174A117808
:103258006FF3C3011170997801F00F01012903D1AF
:1032680011786FF30001117015F07F0F1AD11978DA
:103278009E7801F00700062206F00F0602FB0606FC
:103288000C4F5D78BE5D013066F3060500F007005F
:103298005D7090FBF2F502FB150262F302011970F2
:1032A80001232370F0BD00BF8C150020FF140020FF
:1032B8003D1500201041020810B51F4A1F4B92F916
:1032C800031009B1002231E008B1032119701978FF
:1032D800032930D8DFE801F00209192C11780029F8
:1032E80029D0154881700121197092F902001249FC
:1032F80020B1134B1A786FF3861217E0487808B993
:10330800032213E088700221197092F902100A480A
:1033180089B90B4A147861F386141470026861F352
:103328000F22D1B261F31742026001221A7010BD58
:1033380000211160197010BD34170020FD14002001
:103348005033002038B5044643F6EF2343F6F02007
:10335800012A08BF18460D460DF00EFD2378C0B2AD
:103368001842104C09D043F6EE200DF005FD2368F5
:1033780060F307036FF30F230CE02B7818420AD091
:1033880043F6EE200DF0F8FC2368C0B260F30703A3
:1033980060F30F23236094F9003013B1014B0F221F
:1033A800DA7038BD3417002008B543F6F7200DF061
:1033B800E3FC014B187008BDFE140020014B187087
:1033C800704700BFA8160020024B1A5C6FF3030277
:1033D8001A547047E615002070B50C46C10001F577
:1033E800CE411B488B3108220DF0D7FC0025184828
:1033F8002946EEB21FF05DF908B9237823BB154BB7
:103408002278EB5C1A421FD13046FFF7DDFFF60841
:103418004AF2B34030180DF0AFFC05F00703C0B214
:10342800184110F0010F0FD10B4829461FF041F940
:1034380050B1294608481FF031F9074B06F5CC4032
:10344800CA30995D0DF08EFC0135402DCFD170BD8D
:10345800AA1600209D1500204015002038B546F218
:10346800127540242046FFF7AFFFA5F5CC43094A63
:10347800D23BD15C11F0100F06D06FF30411D15478
:10348800284600210DF06EFC0134E4B20135B92C58
:10349800E8D138BDE61500203F287FB5054607D896
:1034A80000F5E2400D300DF067FCC3B22BB92AE1FC
:1034B800994A1478002C00F02B81984E725D02F026
:1034C8000F014C1C04F00F0464F303023F2D7255E6
:1034D80033D8002C00F01C8101339C4240F0158148
:1034E8008F4B5A1992F88020522A725D03D161F3EA
:1034F8000302725509E16FF30302EC081B197255B8
:1035080093F8902105F0070352FA03F313F0010F23
:1035180040F0FD80294683481FF0B5F8814B04F53B
:10352800CC40195DCA3001240DF01CFC2D19022372
:103538000093019402951820CEE0002C00F0E8805A
:10354800754B1B7801339C4240F0DF80735D05F5B5
:10355800CC406FF30303D230012173550DF002FC08
:10356800735D43F010037355A5F14003DBB2032BE1
:1035780007D80422009201330232019202931920E3
:103588002FE0A5F14803DBB2032B07D804220092F1
:1035980001330332019202931A2060E0A5F150032F
:1035A800DBB2012B07D804220092013303320192C7
:1035B80002931B2053E0572D07D1042300930124C5
:1035C800033301930294212086E0A5F15B03DBB26B
:1035D800012B09D80422009201330232019202938E
:1035E80022200121033A8AE05D2D06D104230093AD
:1035F8000193043B029328467FE05E2D07D1042304
:10360800009301330193053B02935E2075E0A5F119
:103618005F03DBB23F2B09D80422009201339218D2
:103628000192029333200121053A68E005F1610314
:10363800DBB2032B07D80422009201330332019234
:1036480002935F200BE005F15903DBB2012B09D887
:103658000422009201330332019202936020012177
:10366800043A4CE0AA2D07D1042300930124043B1B
:103678000194029361202FE0A92D07D10423009320
:10368800023B0193023B0293622036E0AD2D08D144
:10369800042300930322043B019202936320012137
:1036A8002DE0AB2D06D104230093043B0193029334
:1036B800642022E0AC2D06D104230093043B01933F
:1036C8000293702019E0AE2D0CD10423009301243D
:1036D80002330193029468202146032223460DF009
:1036E800C9FB15E04E35EDB2012D10D80423009327
:1036F80001350233019302956A20012103220B460A
:103708000DF0B8FB03E01C4602E0002400E00124B1
:10371800204604B070BD00BF00000020E615002060
:10372800E823002040150020024B185CC0F300106D
:10373800704700BFE6150020F8B508220E460021A4
:103748000746FCF727FE46F28B75002433782341A1
:1037580013F0010F08D02946064808220DF01DFB7A
:10376800384604491EF05DFF01340835042CEDD1BC
:10377800F8BD00BFB4160020024846F2CA6108220C
:103788000DF00BBB4015002070B5044600F56A50DB
:1037980044300DF0F1FA0B4D06462B7813F0010F6B
:1037A80002D1CC201FF072FD2B8843F001032B803F
:1037B800054B1E55054B13F8242042F0010203F86F
:1037C800242070BDC61600202115002010150020E9
:1037D800024B185C084100F0010070479D1500205D
:1037E80070B505460024094BE0B2E618E35C4BB11E
:1037F8002946FFF7EDFF28B100233370044821461E
:103808001EF04CFF0134402CEDD170BDE8160020AD
:103818002D15002038B5054600242846E1B2FFF7EB
:10382800D7FF10B1044BE35C23B90134042CF4D165
:10383800002038BD012038BD2115002038B50546C7
:103848000DF00EFEA0B100242846E1B2FFF7C0FF3C
:1038580040B1084B13F8243013F0010F02D0064B87
:10386800E35C23B10134042CEED1002038BD0120E3
:1038780038BD00BF1015002021150020F8B51148EB
:1038880000214022FCF786FD46F28B7500240127B3
:103898000D4829460822A7400DF07FFAFFB20026FE
:1038A800094831461EF005FF20B1064BF25C47EA95
:1038B8000202F2540136402EF2D101340835042CAC
:1038C800E5D1F8BD9D150020B41600202DE9FF4173
:1038D80000263446B0461A4B1B78234113F00102E8
:1038E800184B23D0184F1D5D17F82430A84538BF52
:1038F800A84613F0010F1AD0CDB965F3000307F8F5
:10390800243023B20122F71902935B2029462B4663
:10391800009201950DF0AEFA7B78B878F9781843E3
:10392800621C2B460095FEF7E7FE00E01A550134AD
:103938000436042CCFD1054B83F80080BDE8FF8105
:10394800FE1400202115002010150020FC14002072
:1039580010B50C4B1B78A3B10B4B1B788BB1002413
:103968000A4821461EF0A5FE40B1094821461EF02E
:10397800A0FE18B920460121FEF7ECFF0134402CC7
:10398800EED110BD71140020DE100020D0160020EA
:103998004E1E00202DE9F043324C334A238800267E
:1039A8006FF386136FF3C4032380304B304F85B019
:1039B80016701E709146984617F8013B5BB3227843
:1039C800D20052B243EAA2122388402E62F3C40303
:1039D80043F0400323801ED000253046E9B2FFF7AC
:1039E800F7FEA8B117F8013C13F0010F06D0012229
:1039F800AA4099F800100A4389F8002013F0020F32
:103A080006D00123AB4098F80020134388F8003013
:103A18000135042DE1D10136F6B2412ECCD12378FF
:103A280003F04005EDB2D5B903F02403042B0BD104
:103A3800FFF78EFFFF2300934020294601222B46E3
:103A4800019502950DF016FA238800226FF34513AD
:103A58006FF382036FF3C4032380064B1A7005B01B
:103A6800BDE8F083C6160020EC32002009330020A0
:103A78004B150020A916002010B500240548214642
:103A88001EF017FE08B9044BE0540134402CF5D160
:103A980010BD00BFA01600204B15002010B51278ED
:103AA80004469DF80810DAB1D3B111B10D491EF0E2
:103AB800ADFDACB1082246F2CA610B480DF06DF9B4
:103AC800214609481EF0ADFD0749082246F2CA60A2
:103AD8000DF05DF905480449BDE810401EF0B7BD7A
:103AE80010BD00BF80250020F414002040150020E0
:103AF80030B5064B04781D7824EA05040C7001786B
:103B08001B7823EA0103137030BD00BFFE140020A8
:103B180038B50A4D002415F8013F2D2B09D0532B39
:103B280007D0542B05D0462B03D0054821461EF05C
:103B3800B5FD0134402CEED138BD00BF672400200C
:103B4800D016002010B50F481EF058FD00240E486E
:103B580021461EF0AEFD80B10C4BE31893F880307F
:103B6800482B06D003D82D2B03D0462B00E0542B2E
:103B780003D1044821461EF086FD0134402CE6D1CD
:103B880010BD00BF8D150020D0160020E8230020AE
:103B9800094A0A4B117831B1997801F00F01814235
:103BA80001D0002111709A7860F303029A705A7854
:103BB80042F080025A7070478C1500203D15002095
:103BC8007FB5604B154604461A780E4600235E49B9
:103BD80011F8231011F0010F05D001219940C1F10E
:103BE8000F0101EA02020133042BF0D1574B1A707E
:103BF800002C6FD014F0010F0AD0FF23012100938D
:103C0800FF3B0193029352200A460B460DF032F90E
:103C180014F0020F0AD0FF2301210093FF3B019308
:103C2800029353200A460B460DF024F914F0040FB2
:103C38000AD0FF2301210093FF3B019302935420F4
:103C48000A460B460DF016F914F0080F0AD0FF23A8
:103C580001210093FF3B0193029355200A460B462E
:103C68000DF008F914F0100F0AD0FF23012100937A
:103C7800FF3B0193029356200A460B460DF0FAF8D3
:103C880014F0200F0AD0FF2301210093FF3B01937A
:103C9800029357200A460B460DF0ECF814F0400F3B
:103CA8000AD0FF2301210093FF3B01930293582080
:103CB8000A460B460DF0DEF814F0800F0AD0FF23F9
:103CC80001210093FF3B0193029359200A460B46BA
:103CD8000DF0D0F8CEB10024284621461EF0E9FCAC
:103CE80060B1FF230093FF3B0193631C1BB20121CA
:103CF80002935A200A460B460DF0BCF82146284686
:103D080001341EF0CBFC402CE6D110481049114A72
:103D1800FFF7EEFE104B00221A70013200920632B5
:103D28000192083202920A490A4A08480AF0BCFB82
:103D38000A4B3C2251201A7004B0BDE870400DF0C7
:103D480075BC00BFFE14002010150020401800208C
:103D5800161900200A190020051800202015002037
:103D680010B5FFF799F9044607481EF075FCD0F125
:103D7800010138BF002104B929B1034A2046BDE832
:103D88001040FFF71DBF10BDDE150020054B03EBEB
:103D9800D00393F8903100F0070053FA00F000F0D8
:103DA80001007047E823002010B50F4B04461B782C
:103DB80013F0010315D0FFF72DFD28B90B4B1B1984
:103DC80093F88030462B0DD10DF04AFB18B92046E8
:103DD800FFF7DCFF30B1064821461EF054FC0120F5
:103DE80010BD184610BD00BFC6160020E8230020ED
:103DF800DE150020024B1878003818BF01207047E4
:103E08002015002010B5034C04EB830358709970FB
:103E1800DA7010BD1015002010B5002409480021E3
:103E280000190E220E34FCF7B5FAB4F5E07FF5D18F
:103E3800054A00231370054A002199520233AA2B20
:103E4800F9D110BDE0100020DB1000208A190020F5
:103E58007FB5474B04461B780E46AA2B78D04548B9
:103E680021461EF026FC0546002871D12046FFF7A2
:103E78009BFF00286DD1404821461EF01AFC50B91E
:103E88003E4821461EF015FC054620B92046FFF79E
:103E980003FB00285DD13A4B1B7823B9394B1B78BB
:103EA80013F0010F09D1384BDB7803F02003DBB2A4
:103EB8001BB9364B032283F84020012E05D82E4823
:103EC80021461EF0F6FB40B142E0022E07D12B48F6
:103ED80021461EF0EEFB10B13AE0274800E02748E3
:103EE80021461EF0D0FB2A4821461EF0D7FB022EA1
:103EF80015D10125294603222B4600964A2066192A
:103F0800019502960CF0B6FF2046FEF731F9002322
:103F18000246314618200093FEF7EEFB19E0012E09
:103F280009D102230093631C0293019612203146A3
:103F38000322334609E07EB9012102230093631866
:103F480002930191112003220B460CF093FF03E02A
:103F58000025284604B070BD2046FEF709F9024640
:103F680001200023211800930125FEF7C5FBF0E787
:103F7800A816002040150020001500202817002052
:103F8800FE14002086190020C03100204B150020A7
:103F9800D81600202DE9FF4704460D4675482146EE
:103FA8001EF087FB8146002840F0DF8021467148DB
:103FB8001EF069FB704821461EF070FB6F4E0DBB6A
:103FC80001274FF00208E3190293424603203946BD
:103FD8003B46CDF8008001970CF04CFF327862B177
:103FE8000DF03EFA024630B1337840461E33009356
:103FF80021462A4604E0009000E00092404621460F
:104008003B4628E0012D2BD15D4B04F5E2400D30F5
:104018001F5D0CF0B1FE07F00F07874209DA631C39
:10402800022202930E2029462B46009201950CF09D
:1040380021FF327892B10DF013FA024638B14F4B96
:104048000D201B7821461E330093002202E00090C9
:104058000D2021460123FEF74FFB5EE00092F7E7B3
:10406800022D0BD101230193E31802931420494632
:104078002A464B4600950CF0FDFE4EE0032D4CD130
:1040880001272A464FF0020804EB070A4D2039465B
:104098003B46CDF800800197CDF808A00CF0EAFE69
:1040A80035783DB30DF0DCF9024630B1337840463F
:1040B8001E33009321464A4602E0009021464046BE
:1040C8003B46FEF719FB0DF0CBF9671C054648B1D6
:1040D8002046FEF74DF8337802461E3300931A2027
:1040E80039462CE02046FEF743F80095024639464B
:1040F8001A202DE021462A463B4640460095FEF709
:10410800FBFA2046FEF734F8514602462B461A20A1
:104118000095FEF7F1FA384628E03578EDB10DF054
:104128009FF904F11C06054658B12046FEF720F811
:10413800124B02461B7830461E330093611C002345
:1041480007E02046FEF714F8009502463046611C49
:104158002B46FEF7D1FA012008E02046FEF708F8C2
:104168000095024604F11C00F1E7002004B0BDE808
:10417800F08700BFD0160020D81600203017002086
:10418800E6150020064B1B1893F84001492804D077
:10419800452814BF0320022070470120704700BF44
:1041A800E82300202DE9F041244F00243C702448E6
:1041B80021461EF07EFAE5B2224B002837D01E5D5C
:1041C8003B789E4200D303B93E70002E30D1314671
:1041D8001C484022FCF7DEF81B4B1C4803EBD503B8
:1041E80093F8888104F0070348FA03F8214608F099
:1041F80001081EF05EFA68B9B8F1000F02D028462F
:10420800022101E028463146FFF7C4FE28460DF09A
:104218000DFA0DE0B8F1000F0AD12846FFF7B2FFFA
:104228000B4BDB7803F02003DBB20BB9094B1855B5
:104238000134402CBBD1BDE8F08100BF301700200D
:104248002D150020E8160020E8230020D0160020B5
:10425800C03100204B1500202DE9F04F914B89B05B
:104268001B7813F0010F06D08F4B1A786FF3861264
:104278001A7001F030BA8D498D4A0B7810788D4D3F
:10428800984218BF8C49137018BF0B706B7803F0F5
:104298000803DBB24BB143F6CF200CF06DFD864B23
:1042A80018702B886FF3CB232B80844B1B78AA2B99
:1042B80008D18349AA3B0B702B8843F080032B80DD
:1042C80000F076BE6A787B4B02F01002D2B27D4CC9
:1042D800A2B11A886FF30C321A807B4B1B7823B972
:1042E8007A4B1B7813F0010F08D1E37803F0200311
:1042F800DBB21BB9764B032283F840202368754F45
:104308006FF3186323603A7802F00202D2B232B92E
:104318006B494A781AB16B4A43F080731360E678A8
:1043280016F0010648D05D20FFF7FEF900285AD1A3
:104338006B78DFF8808103F00203DBB22BBB5D30C2
:10434800FFF7AAF8064600BBB8F80030012143F48D
:104358000073A8F80030042303220093019302900D
:104368000B460D200CF086FD45200DF05FF9314617
:10437800012233460D200096FEF7BEF9092031468A
:10438800324601230096FEF7B7F96B7803F0020373
:10439800DBB243B34C4B1B7823B94C4B1B7813F05F
:1043A800010F20D1E37803F02003DBB2DBB9484BDF
:1043B800032283F8402016E06B7803F00203DBB297
:1043C8006BB13146324601230A200096FEF794F974
:1043D8008D203146012233460096FEF78DF92B8851
:1043E8006FF349232B802368354A6FF359632360A1
:1043F80093787BB1D37823B93B7813F00C0F05D1B0
:1044080008E03B7803F00C03042B03D0236843F047
:1044180000732360E17801F00201C9B200295BD082
:104428005E20FFF781F9002865D16B78214F03F0F2
:104438000403DBB2EBB95E30FFF72EF80646C0B9CD
:104448003B88012143F480633B80042300930133BC
:104458000322019302900B4617200CF00BFD452018
:104468000DF0E4F80D203146012233460096FEF7A0
:1044780043F96B7803F00403DBB2002B3BD0124BFB
:104488001B7823B9114B1B7813F0010F33D1E37854
:1044980003F02003DBB273BB0D4B032283F84020EB
:1044A80029E000BF4118002050330020B216002038
:1044B800B3160020C616002031170020A8160020C9
:1044C800600E0020C0310020FE1400208619002054
:1044D8004B150020E62300206B7803F00403DBB2C1
:1044E8002BB18D2001220B460091FEF705F92B8890
:1044F8006FF38A232B802368DFF8DCB26FF3DF7356
:1045080023605F2306930026D94696E03046394655
:1045180019F080FD002871D01BF80A30FF2B6DD0F0
:104528004FF4A0727243A8F15E03DBB207930A232B
:1045380003FB072219F802E009EB02035FEADE1E1B
:1045480050D02268404642F0004222600593FFF7AF
:10455800EBF8059B00285CD11A7912F0040F24D1DE
:104568004046FEF799FF059B8446F0B91A79322038
:1045780042F004021A710799042300930291DB1890
:104588000121032201930B46CDF814C00CF072FCF4
:104598004A200DF04BF8DDF814C00C2007990122D1
:1045A8006346CDF800C0FEF7A7F84FF4A073734335
:1045B8000A2202FB07334B441B7913F0040F28D05F
:1045C800804B1B7823B9804B1B7813F0010F20D147
:1045D800E37803F02003DBB2DBB97C4B032283F8DA
:1045E800402016E01B7913F0040F07D08C200799A0
:1045F80001227346CDF800E0FEF77EF84FF4A07371
:1046080073430A2202FB07334B441A796FF3820281
:104618001A71013708F10108202F5FFA88F80AF1AA
:104628000A0A7FF473AF069A013602F12003DBB25F
:10463800022E0BF5A07B069305D04FF0000ADDF89B
:104648001880574662E72368614923F080636FF357
:104658009E7323600B79002B00F017845D4ADFF806
:104668007CB106924FF09F0800271BF8011F3E46B9
:104678000137002952D02368A8F15F0A43F080630C
:104688005FFA8AFA23605046FFF74EF800285CD19B
:1046980017237343DFF8489119F8032012F0100F1D
:1046A80023D150460593FEF7F7FE059B8246E0B9F5
:1046B80019F80320012142F0100209F8032004230D
:1046C8000093023301933BB2032202930F200B465F
:1046D8000CF0D0FB45200CF0A9FF0D20514601221B
:1046E8005346CDF800A0FEF707F81723734319F8CF
:1046F800033013F0100F28D0324B1B7823B9324BFC
:104708001B7813F0010F20D1E37803F02003DBB20C
:10471800DBB92E4B032283F8402016E0172373439E
:10472800DFF8BC9019F8033013F0100F05D08D2076
:1047380001220B460091FDF7DFFF1723734319F899
:1047480003206FF3041209F80320069A12F8011FD8
:104758000692002946D02368404643F080432360F0
:10476800FEF7E2FF002854D14FF0170909FB06F9BC
:10477800DFF86CA01AF8093013F0200F49D1404631
:10478800FEF78AFE0646002843D11AF809300121AF
:1047980043F020030AF809300423009303330193FC
:1047A8003BB2032202934B200B460CF063FB5020D4
:1047B8000CF03CFF19203146012233460096FDF7E4
:1047C8009BFF26E0FE140020861900204B150020D0
:1047D800600E002060320020453500208532002020
:1047E8008D32002017237343DFF8FC9219F8033049
:1047F80013F0200F05D0992001220B460091FDF7F8
:104808007BFF17235E4319F806306FF3451309F849
:10481800063008F10108042F5FFA88F87FF425AF05
:10482800AA4ADFF8C8B206924FF05008043F1BF8B6
:10483800011F3E460137002950D0236808F1620A5B
:1048480043F080635FFA8AFA23605046FEF76CFFF4
:10485800002858D1DFF89892330119F8032012F094
:10486800400F23D150460593FEF716FE059B82465E
:10487800E0B919F80320012142F0400209F80320A9
:1048880004230093023301933BB20322029369206D
:104898000B460CF0EFFA45200CF0C8FE0D205146EF
:1048A80001225346CDF800A0FDF726FF330119F881
:1048B800033013F0400F26D0854B1B7823B9854B66
:1048C8001B7813F0010F1ED1E37803F02003DBB24D
:1048D800CBB9814B032283F8402014E0DFF8109213
:1048E800330119F8033013F0400F05D08D20012251
:1048F8000B460091FDF700FF330119F803206FF311
:10490800861209F80320069A12F8011F0692002958
:1049180033D02368404643F080432360FEF704FF0A
:1049280000283FD1DFF8C8A14FEA06191AF8093064
:1049380013F0200F36D14046FEF7AEFD064688BB81
:104948001AF80930012143F020030AF8093004233A
:104958000093033301933BB20322029310200B46CA
:104968000CF088FA50200CF061FE19203146012223
:1049780033460096FDF7C0FE14E0DFF8749133016A
:1049880019F8033013F0200F05D0992001220B46A7
:104998000091FDF7B1FE360119F806306FF34513A3
:1049A80009F8063008F10108022F5FFA88F87FF449
:1049B8003EAF4A4B1978002946D02368AE2043F011
:1049C80080632360FEF7B0FE00284CD1444B1A7870
:1049D800984612F0400F20D1AE30FEF75DFD074635
:1049E800D8B998F80030012643F0400388F8003021
:1049F8000423009302333146032201936720334690
:104A080002960CF037FA45200CF010FE0D203946BE
:104A180032463B460097FDF76FFE98F8003013F0DA
:104A2800400F20D02A4B1B7823B92A4B1B7813F050
:104A3800010F18D1E37803F02003DBB29BB9264BB2
:104A4800032283F840200EE0254E337813F0400F00
:104A580005D08D2001220B460091FDF74DFE3378DD
:104A68006FF3861333701F4B1978002942D02368DF
:104A7800572043F080432360FEF756FE002848D1B4
:104A8800174E337813F0200F43D15730FEF704FD4B
:104A9800074600283DD13378032243F020033370C2
:104AA8000423012600930333314601931F20334624
:104AB80002960CF0DFF950200CF0B8FD19203946A9
:104AC80032463B460097FDF717FE22E0C33100202F
:104AD800FE140020861900204B150020FC31002010
:104AE80010320020013200208D3200205032002088
:104AF800313200209E4E337813F0200F05D09920D4
:104B080001220B460091FDF7F7FD33786FF345134B
:104B180033704FF000094FF0A70AC8464E46954B30
:104B280008F10108F15C00294ED02368AAF14C0B6A
:104B380043F080635FFA8BFB23605846FEF7F4FD71
:104B4800002854D1182373438B4FFA5C12F0200FBE
:104B580022D158460593FEF79FFC059B8346D8B99A
:104B6800FA5C012142F02002FA5404230093023334
:104B780001930FFA88F30322029320200B460CF0CE
:104B880079F945200CF052FD0D20594601225B466B
:104B9800CDF800B0FDF7B0FD18237343FB5C13F0AC
:104BA800200F24D0754B1B7823B9754B1B7813F055
:104BB800010F1CD1E37803F02003DBB2BBB9714BC2
:104BC800032283F8402012E0182373436A4FFB5CEA
:104BD80013F0200F05D08D2001220B460091FDF720
:104BE8008BFD18237343FA5C6FF34512FA54664B36
:104BF800F15C002936D02368504643F08043236097
:104C0800FEF792FD002842D15B4B4FF0180B0BFBCF
:104C1800063B9BF8013013F0200F38D15046FEF7C1
:104C28003BFC0746002832D19BF80130012143F0B4
:104C380020038BF8013004230093033301930FFA08
:104C480088F3032202934C200B460CF013F95020F2
:104C58000CF0ECFC1920394601223B460097FDF781
:104C68004BFD14E0444F182303FB06735B7813F0E5
:104C7800200F05D0992001220B460091FDF73CFD3D
:104C8800182303FB06777B786FF345137B703F4B44
:104C98001B78002B00F090803D4B374FF35C1822B7
:104CA800002B77D002FB06F3FA5C07EB0901C2F38D
:104CB800801BBBF1000F1BD142F04002FA5478224E
:104CC80004234A800093DB18012101930FFA88F32B
:104CD800032202932E200B460CF0CCF846200CF051
:104CE800A5FCCDF800B00920414601225B4661E0F1
:104CF800B1F9021029BB5FEAD21B22D143F6DE20AC
:104D080005930CF039F8059BD8B1FA5C012142F003
:104D18008002FA5404230093DB1801930FFA88F3F6
:104D2800032202932F200B460CF0A4F847200CF026
:104D38007DFC0920414601225B46CDF800B0FDF715
:104D4800DBFC18237343FB5CDB0935D00B4B1B786A
:104D580023B90B4B1B7813F0010F2DD1E37803F027
:104D68002003DBB243BB074B032283F8402023E038
:104D7800103200205E320020CC310020FE140020CA
:104D8800861900204B1500205432002009320020DB
:104D9800033200207243B95C11F0400F0CD063F36A
:104DA800861163F3C711B9544F447B80892000935F
:104DB80041460122FDF7A0FC01360AF1010A022E44
:104DC80009F118095FFA8AFA7FF4A9AEDFF8C4A3DB
:104DD8004827023E1AF8011FB0460136002937D08D
:104DE8002368384643F080432360FEF79DFC002883
:104DF80047D14FF01D0909FB08F9DFF884B31BF808
:104E0800093013F0200F3CD13846FEF745FB8046A9
:104E1800002836D11BF80930012143F020030BF894
:104E28000930042300930333019333B2032202931E
:104E380013200B460CF01EF850200CF0F7FB19203D
:104E4800414601224346CDF80080FDF755FC18E0A5
:104E58001D2303FB08F3DFF8289319F8033013F038
:104E6800200F05D0992001220B460091FDF744FC44
:104E78001D2303FB08F819F808306FF3451309F8E8
:104E880008300137042EFFB2A4D1A37803F0080339
:104E9800DBB2002B40F08C8048F6F234A4F50A47C8
:104EA800A7F5F977A14839461DF003FC28B9A048B1
:104EB80039461DF0FEFB002874D09E4839461DF087
:104EC800F8FB00286ED139469A481DF0DCFB2046D5
:104ED8000BF052FF984EC0B23070002862D00138F3
:104EE800C0B230700BF060F800285BD13078934E78
:104EF80000F56A5078300BF03FFF914BC0B214F8C0
:104F08000380307000EA0808394688481DF0D1FB54
:104F1800DFF87CA2DFF82C9238B1854839461DF0BD
:104F2800C8FB10B99AF8003014E0814839461DF0E2
:104F3800C0FB38B17D4839461DF0BBFB10B99AF863
:104F4800003004E09AF8003018EA030F02D023EA90
:104F5800080801E048EA03087A487B4989F8008094
:104F68007A4AFEF7C5FD7848794912F047F968B1E1
:104F78000CF076FA50B9764809F000FB30B90123F5
:104F880073487449704A0093FEF788FD0023009324
:104F98000133019333786B4802936B496B4A6D4B2D
:104FA80009F082FA013448F632439C427FF476AF26
:104FB800694E73786FF3C71373702B7803F0800210
:104FC800D2B2002A00F0F08064490C78002C40F03E
:104FD800EB8003F02403042B0BD1FEF7B9FCFF236D
:104FE80000934020214601222346019402940BF0AD
:104FF80041FF2B8800246FF3C7136FF3820364F318
:10500800451364F3410364F30003554A64F34923E9
:1050180064F38A2314702B80524B1A7842F0C00232
:105028001A705A7864F3C3025A70FEF771FD4E483D
:105038001DF0E4FA4D481DF0E1FA4D481DF0DEFA86
:1050480041224C482146FBF7A5F94B4B1A7802F050
:10505800DF0264F304121A70DA7D02F0DF0264F3EF
:105068000412DA7593F82E2002F0DF0264F30412BA
:1050780083F82E2093F8452002F0DF0264F304122F
:1050880083F845203D4B1A7802F0DF0264F386125C
:105098001A701A7C02F0DF0264F386121A74384B15
:1050A8001A7864F345121A705A7F64F345125A77D6
:1050B80093F83A2064F3451283F83A2093F857207E
:1050C80064F3451283F857202E4B1A7802F0DF025A
:1050D80064F386121A702C4B5A7864F345125A708E
:1050E8001A7802F07F0264F345121A705A7E64F34C
:1050F80045125A761A7E02F07F0264F345121A7638
:1051080011E04FF4A07262430A2101FB03221F49F8
:1051180001338A181179202B6FF382011171F0D1B4
:105128000134022C38D00023EBE700BFCC23002049
:10513800D4230020DC230020DD150020D618002011
:10514800B698FF1F40180020161900200A190020E1
:1051580008150020051800203D150020600E0020CD
:10516800A916002050330020281700200015002021
:105178002D1500204B1500208D32002031320020E3
:105188006B33002010320020CC3100204535002040
:10519800FE1400202C320020042272480021FBF764
:1051A800F9F8714B00221A70704C2378002B48D103
:1051B80029786F4A01F00201C9B2D9B16D48118846
:1051C800477863F34D3163F3C30741F080014770BB
:1051D8001180CA201EF05AF8C6201EF057F81EF09B
:1051E800A3F8654A13780BB90CF0ACFAFEF736F958
:1051F800FEF712FE614A2B8811786FF341036FF3B3
:1052080000016FF3000311705D48002140222B80DC
:10521800FBF7C0F85B481DF0F1F95B481DF0EEF9AB
:105228005A481DF0EBF95A481DF0ECF904224D4894
:105238000021FBF7AFF84C4A00231370554A13704E
:105248006AE02F7807F00203DBB293B917F0010781
:105258000FD14C481DF0D2F92378F8B23B4113F036
:10526800010F03D0FEF790FA0CF0F0F80137042F85
:10527800F2D12B783E4F13F0010F25D0FEF770FDC9
:105288003B8843F002033B80FEF720FB364B93F844
:105298000080B8F1000F14D1CA201DF0F7FFCD200F
:1052A8001DF0F4FF3B883C4868F300033B80334B18
:1052B8001A7842F001021A701DF0A0F9FEF7CEF834
:1052C80002E00120FEF764FC2B7803F00202D2B260
:1052D80012B3304A12782AB113F0010F02D102201A
:1052E800FEF756FCFEF75EFF2C4927481DF0A4F98F
:1052F800254926481DF08AF9FEF724FC224928484A
:105308001DF084F9274926481DF08BF9FEF7B4FBF8
:105318001F481D491DF09BF9204923481DF076F9C7
:1053280015490B780BB9FEF735FB737803F080034A
:10533800DBB2002B40D12B7803F02403042B06D1D9
:1053480043F6EC200BF018FD08B1062032E0FEF71A
:1053580051FD08B105202DE00CF0DEFA30B3032032
:1053680028E000BF21150020FC140020FE140020B6
:10537800C616002050330020600E0020FF140020C5
:10538800E81600202D290020A01600202D15002049
:10539800E016002030170020DE1500204015002000
:1053A800D01600208D1500202515002001F056F894
:1053B80010B10420FEF7ECFB694B1B781BB1737826
:1053C8006FF3C7137370674A137813B1664B1B7872
:1053D800CBB12B78654E03F04403402B13D1002149
:1053E800BF3300933F200B460222019102910BF03C
:1053F80041FD338843F6CE2043F0040333800BF09D
:10540800BBFC5B4B187057495A4E0B789BB1564BF7
:10541800197881B92A78554B02F04002D2B252B1BC
:105428001A8861F382021A80337823B943F6CE20B2
:105438000BF0A2FC30702A78DFF8308102F004000B
:10544800C0B24D4B00287AD002F02000C0B2484FBD
:1054580090B11A78002042F0C0021A70FDF72CFFB4
:105468003B78002B71D1B8F8002063F3820263F314
:105478004512A8F8002068E0D20052B219789211BB
:10548800D2B241F0C00112F0010F197003D0C9B2B5
:1054980060F3C711197012F0020F03D01A786FF376
:1054A80086121A701B78344A03F04003DBB24BB9FA
:1054B800537843F00803537023781BB12B8843F4C7
:1054C80000532B800120FDF7F7FE43F6CD200BF0AB
:1054D80053FCC0B20128307002D1264B02221A7048
:1054E8003C78002C31D1FEF733FAFF2301220093D8
:1054F800402021462346019402940BF0BBFC2B88E4
:1055080043F6CD2043F020032B800BF035FC184BDD
:105518001A4A1870144B14701A780AB1013A1A70A2
:10552800197891B90F4A13787BB1FF230093412072
:1055380002220B46019102910BF09CFC05E01A78BF
:1055480042F0C0021A70FDF7B7FE0CF095F90C484E
:105558001DF082F80B4BB8B91A7860F3820216E096
:105568005E3A0020B216002031170020C61600202F
:10557800A91600204A15002050330020600E002094
:1055880095150020FF1400201A7842F004021A70C2
:105598006A78524812F001011A780CBF61F341028F
:1055A80042F002021A704E491DF051F84D494B481D
:1055B8001DF037F849484C491DF033F83378012B72
:1055C80040F089802B8800246FF349236FF38A23E6
:1055D8002B80464B41221C7021464548FAF7DAFEDB
:1055E80044481DF00BF8FEF793FA3E481DF006F804
:1055F8003D481DF003F8404B1A7802F0DF0264F3CF
:1056080004121A70DA7D02F0DF0264F30412DA750C
:1056180093F82E2002F0DF0264F3041283F82E20A0
:1056280093F8452002F0DF0264F3041283F8452062
:10563800324B1A7802F0DF0264F386121A701A7C71
:1056480002F0DF0264F386121A742D4B1A7864F3A1
:1056580045121A705A7F64F345125A7793F83A2024
:1056680064F3451283F83A2093F8572064F34512FF
:1056780083F85720234B1A7802F0DF0264F386126E
:105688001A70214B5A7864F345125A701A7802F04E
:105698007F0264F345121A705A7E64F345125A76F3
:1056A8001A7E02F07F0264F345121A7611E04FF475
:1056B800A07262430A2101FB0322144901338A18AC
:1056C8001179202B6FF382011171F0D10134022C72
:1056D80001D00023EBE709B0BDE8F08FB22D002020
:1056E800D016002000150020281700204A15002099
:1056F8004B1500202D1500208D320020313200205E
:105708006B33002010320020CC31002045350020BA
:105718002DE9FF4104460D460CF0D8F8A04B1A19A4
:1057280092F880709F4A98461278AA2A0AD1A7F15F
:105738004F03DAB20B2A00F2AD819B4A5BB29A4062
:1057480040F1A881994B0C2202FB04335A7A0833A2
:10575800AA42C0F09F81FF2A00F09C81FF229A7024
:10576800934808EBD403214693F888511CF0A1FF15
:105778000646002840F08E8104F007031D41502F93
:1057880005F0010500F0268114D8462F00F0F280BC
:1057980009D8412F00F09E80452F00F01B812D2F46
:1057A80040F0768134E0482F00F0C5804F2F40F05C
:1057B8006F810EE0542F67D006D8522F00F08A80F0
:1057C800532F40F065811CE0A7F15903012B00F22B
:1057D8005F81784821461CF06CFF0646002840F09F
:1057E80059815A2F01D1744802E0592F04D17348C6
:1057F80021461CF048FF54E121466F481CF043FF46
:10580800F5E76F4821461CF054FF002800F042815C
:105818006C4821461CF04DFF8046002840F03A8134
:10582800214668481CF02FFF674821461CF036FFC8
:105838000227012655B1A419142041463A46434689
:105848000097019602940BF015FB2AE129463A4687
:10585800334604F101080A2000970196CDF8088024
:105868000BF008FB2046FCF783FC414602462B461A
:1058780013200095FCF740FF384629462A46334650
:105888000095FCF739FF0CE14E4821461CF011FF4A
:105898000746002840F0058101260222314633469A
:1058A800A5193E200092019602950BF0E3FA2046D6
:1058B800FCF75EFC294602463B4614200097FCF79D
:1058C8001BFF21463F481CF0DEFE21463E481CF0E7
:1058D800E5FEE6E03A4821461CF0EBFE06460028C5
:1058E80000F0DF80374821461CF0E3FE064628B961
:1058F8002046FDF7D1FD002840F0D380002D40F070
:105908008E802046FEF750FA002840F0C5802046D9
:10591800FEF738FC2D4BDB7803F02003DBB20BB924
:105928002B4B1855412F00F08880522F40F0B08043
:105938002046012183E0234821461CF0BAFE28B9FD
:105948002046FDF7A9FD002840F0A480002D66D16F
:105958002046FEF729FA002840F09E801B4BDB7892
:1059680003F02003DBB2002B67D1194B032283F825
:10597800402062E0134821461CF09BFE064628B9E9
:105988002046FDF789FD002840F08B802046FEF771
:105998000BFA00287ED1002D41D1204603214EE08C
:1059A800E8230020A816002000003080BC25002035
:1059B80040150020DC230020CC230020D423002025
:1059C800A0160020D0160020D8160020C0310020D4
:1059D8004B150020354821461CF06BFE0646002872
:1059E8005FD02046FDF72AFF20B1214630481CF041
:1059F8004AFE4FE0502F28D12E4B1B782BBB204658
:105A0800FDF708FF08BB2C4821461CF052FE06464D
:105A180020B92046FDF740FD002842D115B12046A7
:105A280002210CE02046FEF7ADFB244BDB7803F0A7
:105A38002003DBB20BB9224B185520460021FEF794
:105A4800A9FA061E18BF01262BE02046FDF7E2FE44
:105A58000546F8B91B4821461CF02BFE0646D8B966
:105A68002046FDF719FD0746D8B9164821461CF00F
:105A78000AFE154A135D8BB910494E7806F02006C8
:105A8800F6B26EB908EB040393F80031135508E039
:105A9800012606E0002604E02E4602E03E4600E02D
:105AA8001E46304604B0BDE8F08100BFA0160020B5
:105AB800DE15002030170020D0160020C03100204D
:105AC8004B1500202D150020E8160020032210B5E4
:105AD80005490648FAF734FF054806490222BDE899
:105AE8001040FAF72DBF00BF262100200402002035
:105AF800090200202421002070B5804C237813F07F
:105B0800010F0AD00BF0B4FC38B100207C4902F038
:105B180089FE7C4B7C48197849E07C4D2B78002B1A
:105B28004AD00BF0ABFC002846D0794B1B7873B9F0
:105B3800784B5B7813F0010F09D00BF091FC30B96A
:105B4800237803F02403042B01D10330B6E0724C10
:105B5800207870B10020714902F064FE217801229A
:105B68006F4802F085FE00201021621C08F068F8DA
:105B780002E06C4902F056FE6B4C644808F0B4F839
:105B88002378002B00F00F810BF072FC002800F046
:105B98000A81664966481022FAF7D2FE64485B21FA
:105BA800FAF776FC002800F0FE8021780130832285
:105BB800BDE8704002F05CBE5E4C237803F005033C
:105BC800012B5DD100205C4902F02CFE202110221F
:105BD8005A48FAF7DFFB601D59490322FAF75AFEC3
:105BE80040BBE01C57490222FAF754FE30B9564828
:105BF800FAF720FE5449024650480BE0E01C53498E
:105C08000222FAF747FE40B95148FAF713FE504905
:105C180002464A48FAF794FE0EE0E01C4D4902227B
:105C2800FAF738FE30B94C48FAF704FE4A490246FA
:105C38004248EFE7FFF74AFF6278303AD3B2092BC0
:105C480000F2B1803B4B9B78303BDBB2092B00F272
:105C5800AA800A2101FB0231C9B2002900F0A38001
:105C6800334BFF220C291A7740F29D8010295A776E
:105C780040F2998013299A7740F29580DA7770BDBF
:105C8800234E3378F3B9234B5B7813F0010F19D007
:105C98000BF0E6FBB0B931481CF0DEFC68B1304CC3
:105CA800304B226802EA03033BB917F0B5FD20B96F
:105CB800E37803F04003DBB223B10020BDE8704075
:105CC80009F056BC337863B90BF0CAFB48B1264BD0
:105CD8001B7803F00603042B03D02B780BB90120A3
:105CE800ECE7FEF787F810B10020204957E0204B79
:105CF8001C78002C40D01F4951E000BFC616002078
:105D080059D60208FC14002000020020FE140020CE
:105D1800D418002086190020221800206CAB020835
:105D2800050200202AAB0208301700204BAB0208FE
:105D3800F40100202121002073B002080402002091
:105D4800A4320308A8320308D6B00208AB3203080D
:105D5800B5B00208AE32030894B0020895150020C9
:105D6800C03100203000000FFF140020FCBD0208E5
:105D7800650E00208DAB02080B4802F002FD0A48B0
:105D880002F0F6FC094802F0F3FC1BF011F9084B8D
:105D9800DB7803F02003DBB22BB106492046BDE8CF
:105DA800704002F03FBD70BD181900204C1800204B
:105DB800C031002085AA0208054B1B78D8019B0139
:105DC8005BB2DB1140B243EAE070C0B2704700BF7B
:105DD800C616002070B50E4686B041000122054661
:105DE80001F5E97105A80AF0D8FF0021012E8DF808
:105DF80015104FF0FF0205F1010305D10092019142
:105E080002930920FB3A04E00092019102931E20BC
:105E180004220B460BF02EF805A83D49FAF7BEFB05
:105E280050B105A83B49FAF7B9FB28B105A83A498A
:105E3800FAF7B4FB002867D105A83749FAF7AEFB93
:105E4800364B0446F8B95A78214642F010025A7087
:105E5800FF23022200930190FE3B02903D200BF0AD
:105E680009F84D200BF0E2FB691C012223461220A1
:105E78000094FCF741FC122021462246012300949D
:105E8800FCF73AFC03E05A786FF304125A700024C6
:105E9800E0B2552115F066F838B12846214615F0CC
:105EA80002FA10B1204615F0EDF90134082CEFD1B3
:105EB8003EBB1B481B491C4AFDF71AFE19481B49E3
:105EC80011F09CF968B10BF0CBFA50B9174808F0FB
:105ED80055FB30B9012315481549124A0093FDF7BF
:105EE800DDFD144B0F491D7000230093053301930A
:105EF800114B0D4A1B780A4802930D4B08F0D4FA4F
:105F080002E00E4B00221A7005A806B070BD00BF53
:105F180035330308B13203084135030850330020F4
:105F280040180020161900200A1900200815002022
:105F380005180020DF330020D61800202015002087
:105F480007B54100012201A801F5E9710AF025FF12
:105F5800002301A804498DF80530FAF71FFBD0F19A
:105F6800010038BF00200EBD3533030807B54100D6
:105F7800012201A801F5E9710AF00FFF002301A829
:105F880004498DF80530FAF709FBD0F1010038BF54
:105F980000200EBDFE34030870B5154B04461B18CF
:105FA80093F88050B1B1134821461CF082FB88B9A0
:105FB800114821461CF067FBA5F15903DBB2012B00
:105FC8000CD94F2D0AD0542D08D021460B481CF06F
:105FD8005AFB07E0084821461CF060FB07482146A9
:105FE8001CF05CFB04480649BDE870401CF00EBB81
:105FF800E8230020401500209515002035150020C5
:10600800E0160020024B1878C0F38000704700BFEC
:10601800FF140020024B1A8860F308221A80704788
:10602800C6160020034B5878C00140B2C011C0B258
:10603800704700BFC6160020014B1878704700BF94
:10604800FE14002030B5457800230021C218917055
:1060580055FA03F111F0010F08D0064959188C7C44
:10606800017804EA0101A14208BF91700133042BB1
:10607800EBD130BD2218002046F6753104220AF013
:106088008CBE000070B5104C054611222046002138
:10609800FAF780F9002004F8010C2A78103414F873
:1060A800011FC3B291420BD152B10849013301F823
:1060B800013B112246F6C553BDE8704002F0FEBA16
:1060C80001300428EBD170BD2318002022180020CD
:1060D8001FB520B1134B1A8842F480521A80124B14
:1060E80000245A78214642F010025A70FF230222F7
:1060F80000933D20FE3B019402940AF0BBFE4D2024
:106108000BF094FA20210122234612200094FCF778
:10611800F3FA12202146224601230094FCF7ECFAF8
:106128001FBD00BFC6160020503300202DE9F341E3
:106138002D4C0722E37848F6883702FB003348F6EF
:10614800A930DBB218180AF017FE257964795FFACE
:1061580080F8002648FA06F313F0010F3AD03946C2
:10616800042201A80AF019FE9DF804009DF80530E4
:106178009DF806109DF8072000282BD0002929D06B
:10618800002B27D0002A25D0934204D19C4221D14C
:1061980085421FD30FE09A4210D99C421AD39442E9
:1061A80018D89C4201D994421AD39C4201D1854205
:1061B80016D294420ED18D420CD811E09C4201D1E6
:1061C80085420DD2944201D18D4209D99C4207D80B
:1061D800944205D301360437082EBBD1002000E0D5
:1061E8000120BDE8FC8100BFCC37002010B5044673
:1061F80048F6E13000EBD4000AF0BEFD04F00704D5
:10620800C0B2204100F0010010BD70B5C30848F6C7
:10621800E1355D19044628460E460AF0ADFD04F046
:106228000704C0B2012126B9A14040EA0101C9B260
:1062380002E0A14020EA01012846BDE870400AF0CA
:1062480091BD0000F0B57D4B8DB0DD78042200EBE8
:10625800C505EDB2E90001F5F04104A810310AF0D6
:106268009CFD774B774E1A78002304A9C95C312925
:1062780005D13039994041EA0202D2B205E030290D
:1062880003D12F39994022EA01020133042BECD1C2
:1062980032706C486C496D4AFDF72AFC6A4B1B78D2
:1062A80013B96A4B1B78F3B16748694910F0A6FF28
:1062B80068B10BF0D5F850B9654808F05FF930B906
:1062C800012363486349604A0093FDF7E7FB002315
:1062D800009302330193FD3302935A485A495B4AAB
:1062E8005C4B08F0E1F805EB0511002401F5F241DB
:1062F800347004A8D03108220AF04FFD2646E0B2D7
:10630800542114F02FFE002838D004AB1B5D312B2C
:1063180003D1204614F0BCFE38B104AB1B5D302B12
:106328002CD1204614F0B4FE40B34EB9FF2300939D
:106338003420314604223346019602960AF09AFD2B
:1063480004AE305D2146303814F0B0FE335D0126CE
:10635800312B4FF0030306D10093A3191BB201960A
:106368000293352005E00093631C1BB2019602934B
:106378003620002104220B460AF07CFD0134082C4B
:10638800BDD1A90101F5FA4104A8883120220AF0FB
:1063980004FD083C04AD274615F8013BE6B201347C
:1063A800302B03D13046FFF721FF38B115F8013CF7
:1063B800312B2CD13046FFF719FF40B34FB9FF23DB
:1063C80000933420394604223B46019702970AF08D
:1063D80051FD15F8011C30463039C9B2FFF715FFD9
:1063E80015F8013C0021302B4FF0FF0305D1009335
:1063F80023B201910293372004E0009323B2019164
:106408000293382004220B460AF034FD0127202C81
:10641800C2D1114D6B7803F00403DBB263B1203CA9
:106428002046FFF7E3FE38B90134E4B2202CF7D157
:106438006B7860F382036B700DB0F0BDCC37002031
:10644800FE14002040180020161900200A19002008
:10645800081500200518002050330020014B18783B
:10646800704700BF650E00202DE9F04F4E4B00220B
:106478001A704E4A85B01678002E40F091804C4B29
:106488004FF4B468DA78997808FB02F24FF03C08C8
:1064980008FB01285A78474F90441FFA88F8BA46F3
:1064A8006CE03AF815303C24DAB2544304EB132478
:1064B8004C44A4B2042CEEB207D842F25A73984561
:1064C80003D904F51C546034A4B2444511D948F6E4
:1064D800A8300AF051FCC8EB0403834209DC364BB0
:1064E8001A787B1993F83830934302D02E49012348
:1064F8000B702F4AD378B34232D142F26073B4FBA7
:10650800F3F203FB12439BB2434523D12B4B9B78F9
:1065180013F0090F44D12A4B5B7803F08003DBB2F8
:10652800002B3DD1274B5B7803F00203DBB2002B35
:1065380036D1254B1A781BEA020F11D10199009820
:1065480041EA02021A70FFF7F1FD48B90098FFF717
:1065580079FE05E01C4B02991A7801EA02021A70CA
:10656800013509F5B469072D1FFA89F999D1039EF8
:1065780007370136042E0AF10E0A11D04FF0010B2D
:106588000BFA06FB5FFA8BF301936FEA0B03F2B287
:10659800DBB24FF00009009202934D46039680E764
:1065A80005B0BDE8F08F00BF650E00203917002048
:1065B800CC3700203A170020FE140020C0310020FC
:1065C8005F330020AA2B00203817002073B50C4633
:1065D80001EBC001C9B2C90001F5F041054604222A
:1065E80001A810310AF0D9FB104B002003EBC402BC
:1065F800121B521982F8380001AA125C312A0AD1FA
:106608000121814003EBC402121B521992F8386031
:10661800314382F8381001300428EDD101A9312224
:1066280030231CF04EF8C0B27CBD00BF3A170020E2
:1066380000B501EBC001C9B2890189B001F5FA4181
:106648008831202268460AF0A8FB202069463122BA
:1066580030231CF036F8C0B209B000BD07B501EB15
:10666800C001C9B201EB011101F5F241D031082294
:1066780068460AF092FB08206946312230231CF054
:1066880020F8C0B20EBD00002DE9F84300263446BC
:106698002BE021462846FFF799FF214681462846E8
:1066A800FFF7C6FF214640EA09092846FFF7D6FF4B
:1066B8005FFA89F949EA000010F0FF0F05D040465B
:1066C800394602220AF069FB03E04FF0FF33A8F8CD
:1066D80000300135EDB20237072D08F10208D8D194
:1066E8000134E4B20E3E042C07D0054BC6F5EE4744
:1066F800C6EB0308A0370025CBE7BDE8F88300BF49
:106708003A17002010B51DF043F84FF480301DF003
:106718005FF81DF077F90128044628D110201CF0F5
:1067280059FF02201CF04AFF00201DF091F80020BC
:106738001DF0A2F84FF480601DF094F84FF440402B
:106748001DF0A4F84FF480304FF4E0111DF05CF810
:1067580020461DF065F839201DF040F90028FAD0D0
:1067680002201DF063F81DF06BF80828FBD17C208F
:1067780001211DF0FDF846F6012001211DF0F8F871
:106788000C4801211DF000F90B4801211DF0FCF80F
:10679800042001211DF0F8F87E201DF01FF938B102
:1067A8001DF046F9054B04211A7861F344021A706A
:1067B80010BD00BF0340060020080818413A002019
:1067C80010B50C46014620B110220C48FAF7B8F86B
:1067D80004E00A4820211022F9F7DCFD34B108480A
:1067E80021461022BDE81040FAF7AAB80448202133
:1067F8001022BDE81040F9F7CDBD00BFF40100201C
:106808000402002010B5FF2B1446029A03D0421848
:1068180002F8013C08E06FF07F439A4204D0131459
:10682800437013128370C27019F0C4FA02E07F201B
:106838001DF01AFC19F0AAFA0028F8D1ACB10B48DF
:1068480090F82010163001F00F0119F0B3FA02E0A9
:106858007F201DF009FC19F099FA0028F8D1044BA3
:1068680093F8693013F0010FE9D110BD900C0020A6
:106878005C39002010B50A4B002203EBC003013B32
:106888001046084951184C7813F8011F8C4205D15D
:106898000130C0B20C320828F3D1F73010BD00BF68
:1068A8003A410208BC25002070B50D4C05460E463D
:1068B8004FF4007200212046F9F76CFD2A46314654
:1068C80004F50070F9F7BEFC642024F8035C1AF0A4
:1068D80041FE0023A4F82D33024B64221A6070BDD8
:1068E800C53A00202C21002010B5054C0021204677
:1068F8004FF40072F9F74EFD0023A4F82D3310BDB4
:10690800C53A0020164B2DE9F0415D8A0746284616
:10691800FBF706F91349FBF70FFA134B134E1860F0
:10692800D723B5FBF3F5EDB2822229460446F019C8
:1069380001F09EFF2846FBF7F7F801462046FBF7D3
:106948003DF80B49FBF744F9FBF708FB0337BE1981
:10695800C1B281223046BDE8F04101F089BF00BFD5
:10696800F82800200000574390170020F401002069
:10697800000020410000000070B54B4D2868FAF770
:10698800DBFC45A3D3E90023FAF776FBFAF7C2FF4D
:10699800FAF7D2FC42A3D3E90023FAF721FD3EA37C
:1069A800D3E90023FAF746FEFAF7B4FFFAF7C4FC76
:1069B800FAF7CEFAFAF7AEFF3C4906462860FBF72D
:1069C800AFFA20B13046FBF7C9FAC4B25EE03046F0
:1069D8003649FBF7B9FA50B130463549FBF7A0FA0A
:1069E80028B13046FBF7BAFAC0B2441C4EE0304634
:1069F8002F49FBF7A9FA50B130462E49FBF790FA18
:106A080028B13046FBF7AAFAC0B2841C3EE03046F3
:106A18002849FBF799FA50B130462749FBF780FA25
:106A280028B13046FBF79AFAC0B2C41C2EE03046B3
:106A38002149FBF789FA50B130462049FBF770FA33
:106A480028B13046FBF78AFAC0B2041D1EE0304672
:106A58001A49FBF779FA50B130461949FBF760FA41
:106A680028B13046FBF77AFAC0B2441D0EE0304632
:106A78001349FBF769FA48B130461249FBF750FA57
:106A880020B13046FBF76AFAC0B2841D0A202146BD
:106A9800BDE870400AF066B9736891ED7CFF7F40ED
:106AA8000000000080842E4194170020000010414F
:106AB8000000F0410000484200008E420000B84249
:106AC8000000E0420000F2422DE9F04F9DB019F0BD
:106AD80007F909201AF0DAFE1AF0C0FC4FF46140F9
:106AE8001AF010FF09201AF08DFF0022A3484FF476
:106AF80080411CF0D4FDA24800211DF09DF9A14958
:106B080004224B78DFF8A0E26FF300034B709E4B32
:106B18009E4C1A705A715A709A70DA701A719A717A
:106B2800DA719B4B033A1A709A4B00201F328EF889
:106B3800000020705A7105900546069006467F2091
:106B48001DF092FA23780E2B01F2B681DFE813F0DC
:106B58000F004F009500E0007902DE033004850441
:106B6800EA06DC07EF075808B108D00882098A4E00
:106B78008A48317801F00F01013149014118FFF7C6
:106B88001FFE337813F00F0308D1854A92F80123CA
:106B9800012A41F09181834A138024E0012B03D11B
:106BA8007F4B93F819330BE0022B04D17C4B93F8FD
:106BB8000D33032B05E0032B06D1794B93F80D33E6
:106BC800012B41F079810EE0774901220A7077485C
:106BD8004FF400711CF063FD754BC8221A603378BE
:106BE8006FF30303BFE333785A1C01F05FB8704BAF
:106BF8001A6822B96D484FF400711CF050FDDFF897
:106C080098816C4898F8001001F00F010131490192
:106C18004118FFF7D5FD36B198F800305A1C62F3D9
:106C2800030388F800305F4B00221A8098F80010A0
:106C380001F00F02022A03D11A7842F010020AE08A
:106C4800042A03D11A7842F0040204E0052A05D187
:106C58001A7842F040021A7001F02EB9062A04D1BF
:106C68004D4B6FF3030119707EE301F00F01012210
:106C780012FA01F1198001F01FB9474E4E483178D8
:106C880001F00F01013149014118FFF799FD96F80C
:106C9800008008F00F08B8F1070F27DC18F0010F83
:106CA800464B02D00020588002E04FF0FF31598057
:106CB8004FEA6809062209F1010902FB09394FF078
:106CC800FF32A9F802204046FFF7D4FDFF2806D07E
:106CD8003B4B03EB40005823437401F0EDB800230D
:106CE800A9F8023008F1010801F08AB80021102241
:106CF80013A8F9F74FFB0FA800211022F9F74AFB58
:106D080023780133237033786FF3030301F07BB8E2
:106D1800DFF884A09AF8008018F00F0840F03F814F
:106D2800284E337803F04003DBB2F3B926486FF0FE
:106D38007F43817A0122009301F00F01FF23FFF7BF
:106D480061FD224B93F8692012F0400F08D093F8A8
:106D58006C3013F0040F03D0337843F040033370E2
:106D68007378142262F3C7037370737813F0F80F03
:106D780030D0174800F12001A7E300BF00180140F8
:106D8800002C01401A290020E82300209A1700202F
:106D9800630E00208D320020991700207A410208E6
:106DA800BC250020503300205C210020000C01404D
:106DB8002C2100201A420208FA4202080A33002055
:106DC800F4010020AB310020900C00205C39002039
:106DD8001A440208BC4B1B7803F04003DBB2002BBB
:106DE80000F0D980DFF80483DFF8049398F80030C6
:106DF80013F00C0B30D1B54E6FF07F4396F82B1083
:106E080006F12100009301F00F0101220523FFF78D
:106E1800F9FC96F84C104FF4860A06F1420001F08E
:106E28000F010122FF23CDF800A0FFF7EBFC96F835
:106E38004110FF2306F1370001F00F015A46CDF843
:106E480000A0FFF7DFFC042389F8003098F8003031
:106E580043F0080301F02EB803F00803DBB2002B5F
:106E680039D099F800A0BAF1000F03D0984800F182
:106E7800400138E0954E6FF07F4B717D06F10B00B5
:106E880001F00F010122FF23CDF800B0FFF7BAFC93
:106E980096F82B1006F1210001F00F0101220723BB
:106EA800CDF800B0FFF7AEFC96F836104FF4860325
:106EB800009306F12C00FF2301F00F015246FFF763
:106EC800A1FC98F800306AF3C303DBB243F0040373
:106ED80088F800305AE099F800C0BCF1000F08D0DB
:106EE8007B4800F16001FFF76BFC99F80020303215
:106EF80008E2764E6FF07F40717DFF23009001F02D
:106F08000F0106F10B000122CDF80CC0FFF77AFC47
:106F18009AF80030DFF8C4B103F0100A5FFA8AFA71
:106F2800DDF80CC0BAF1000F0CD098F800206CF313
:106F3800820288F800205A1C62F303038BF80030A1
:106F480000F0BABF96F82B106FF07F42009206F15E
:106F5800210001F00F0101220C23FFF753FC96F8E2
:106F680036104FF4860300935246FF2306F12C0097
:106F780001F00F01FFF746FC9BF8003083F0100288
:106F8800C2F3001262F304138BF80030042389F86B
:106F9800003000F091BF4E4800F1800195E2B8F151
:106FA800010F3CD14A4800F1A001FFF709FC002E6F
:106FB80000F082879AF80030444E5A1C62F30303AB
:106FC8008AF8003096F82B106FF07F4906F12100FF
:106FD80042460F2301F00F01CDF80090FFF712FC95
:106FE80096F82B1006F1210042460E2301F00F01FE
:106FF800CDF80090FFF706FC96F82B1006F121005B
:10700800424601F00F010F23CDF80090FFF7FAFB7D
:107018003048802142461CF042FB00F04DBF2C480E
:1070280000F1C001FFF7CCFB002E00F045872A4B8A
:1070380096221A609AF800306FF303038AF800303A
:1070480092E1264E317811F00F0A16D1244800F14A
:107058002001FFF7B5FB204B1B68002B40F02C8765
:1070680013A8F9F7E7FB40221346014613A801F0DD
:1070780023FA3378012200F019BEBAF1010F39D191
:1070880012486FF07F4390F82010002200931630CA
:1070980001F00F01FF23FFF7B5FB01F077FA002895
:1070A80000F00A873378022262F3030333700D4B32
:1070B8001A7842F080021A700B4B5A7842F002029A
:1070C8005A7000F0F9BE00BFAB310020900C0020D0
:1070D8001A440208001001402C21002099170020B2
:1070E800FA440208B03100206E340020E04000204D
:1070F8006742002001F00F0101F10E0303F00F03B6
:10710800012B44D89B4849014118FFF759FB9A487D
:107118006FF07F4390F8201000221630009301F0A2
:107128000F01FF23FFF76EFB19F0E0FF337803F040
:107138000F03022B13D116F03BFB002800F0BC868E
:107148008E4B1A7842F040026FF304121A705A7884
:107158006FF345125A703378032200F0A7BD16F07A
:1071680011FB78B116F0B0FB16F068FA844B0020DA
:107178001A7858816FF3C7121A703378042262F3B1
:10718800030333707F4B1A786FF3000263E5BAF19B
:10719800040F4DD1DFF8DC914901DFF81082494432
:1071A8004846FFF70DFB98F80010774B01F00402F2
:1071B800D2B27AB941F004016F4883F800A088F888
:1071C800001090F836104FF4860300932C3001F02D
:1071D8000F01EEE293F800A0BAF1000F40F06C86C0
:1071E80065486FF07F45417D01220B3001F00F01AA
:1071F800FF230095FFF706FB64480122817AFF23ED
:1072080001F00F010095FFF7FDFA98F8003005220C
:107218006AF3820388F800303378484662F3030340
:10722800337009F1A001FFF7CBFA554600F044BED0
:10723800DFF84481FF2398F8201000226FF07F497F
:1072480008F1160001F00F01CDF80090FFF7DAFA07
:107258002BB2072B18D1337808F121006FF3030301
:107268003370237801220133237098F82B100E23F2
:1072780001F00F01CDF80090FFF7C4FA44488021CF
:1072880000221CF00CFA0025424E96F86B3013F0E1
:10729800040F00F0118698F857106FF07F43002212
:1072A80000933D48FF2301F00F01FFF7ABFA96F872
:1072B8006B303A4A03F00F03012B137003D1002DF2
:1072C80008BF01250CE0022B04D12BB2012B08BF0B
:1072D800032505E0032B03D12BB2032B08BF072599
:1072E800ABB213F0010F02D02D4A3121517713F0C0
:1072F800020F02D02A4A3221917713F0040F00F0CE
:10730800DB853322264BDA7700F0D6BD1948254EA7
:1073180000F1C001FFF754FA96F80090DFF85C809E
:1073280019F00F090CD116F0A3F898F8003069F39A
:10733800000388F8003033785A1C62F30303337073
:1073480016F028F998F8003013F0010F00F0B48512
:107358000022154880211CF0A2F90A4B00225A701D
:10736800337862F30303337023780133237000F01A
:10737800A3BD00BFFA440208900C00206E34002020
:10738800B0310020E63300206742002001000020D1
:10739800001001405C390020DD0C0020AA310020DB
:1073A800F40100209917002000180140E040002057
:1073B8008648874E00F1E001FFF702FA0FA8F9F7B7
:1073C80039FA0FA902468348F9F7BAFA0021824828
:1073D800B18090F8C5106FF07F4300220093BB3056
:1073E800FF2301F00F01FFF70DFA7C4A92F86B10AA
:1073F80092F86C30327843EA012312F0010FB3801F
:1074080010D0A3F1EB0292B20A2A04D9A3F5E673CD
:107418009BB2282B02D8F3880133F38033786FF3BB
:10742800000333707378002B40F04685684AD28891
:107438007AB16B4A1BA8117863F3030111702278A3
:107448008DF86F300132227028228DF86C201CF0E4
:1074580045F90022F28000F02FBD624EDFF8ACA1A2
:10746800337803F004085FFA88F8B8F1000F15D1F3
:1074780009A841461522F8F78DFF5B4BCAF8008032
:107488001B684546CDF827303368474643F0040368
:107498003360564BA3F8368300F00EBD03F080032B
:1074A800DBB2002B67D1DAF80010002940F0048520
:1074B8004F48FFF785F94F484FF480511CF0E5F825
:1074C800012806D04A4800F1A001FFF779F900F039
:1074D800F3BC4649B1F83623002A43D0093146485F
:1074E800013AF9F72DFA444B03F1100113F8012B77
:1074F8000D2A01D00A2A02D1202203F8012C8B423E
:10750800F4D13E4B4FF03C0808FB073808F11E0841
:107518004046F9F78FF9414602463948F9F7BAF972
:10752800D8B9022F03D1336843F0100304E0032FC6
:1075380003D1336843F040033360327853005BB2C1
:1075480003EAC263DB173268DBB263F3C712326047
:107558001BB1FFF7C9F900F0AFBC0137FFB2042F28
:1075680008BF0227254B3C2606FB07363046F9F7AD
:1075780061F9314626E0DAF80080B8F1000F40F0F2
:107588009B84737803F02002D2B2002A40D11D4BAD
:1075980009A81A889B781C498DF82630ADF8242054
:1075A800F8F752FF114B5B7A302B07D1FFF79CF9A4
:1075B800336843F40053336000F07EBC09A8F9F740
:1075C80039F909A9FFF770F900F076BCFA44020806
:1075D800E633002008020020900C00205C390020CF
:1075E8009917002030210020B3320308BC3A00204C
:1075F800FA45020800080140040200200C0000209F
:10760800C53A0020B8320308BC3203082C210020F8
:1076180003F04003DBB2002B40F08980B14800F151
:107628006001FFF7CDF8B048F9F704F98046AE4994
:10763800AE484246F9F72EF9002873D1AC4B4344C3
:107648005B7A302B6ED1FFF74FF93368DFF8D092B1
:1076580043F48043336099F82B106FF07F43009315
:1076680009F12100082301F00F010122FFF7CAF8F0
:107678006423CAF800307F201CF0F6FCDAF80030EA
:10768800002BF8D1984699F88E10D633994E89F880
:1076980086304B3B6FF07F4A89F88730964801F077
:1076A8000F0142467433CDF800A0FFF7ABF896F807
:1076B800B91106F5D670033001F00F014246FF23D9
:1076C800CDF800A0FFF79EF896F8C41106F5DD7016
:1076D80001F00F014246FF23CDF800A0FFF792F812
:1076E80096F8CF1106F5E270013001F00F0142461D
:1076F800FF23CDF800A0FFF785F896F8DA1106F514
:10770800E87001F00F014246FF23CDF800A0FFF713
:1077180079F899F899107948CDF800A001F00F018F
:10772800424646E07648F9F785F875494AE796F8FB
:1077380002B0DFF8EC910BF0020B5FFA8BFBBBF1A8
:10774800000F3AD199F82010FF236FF07F4809F114
:10775800160001F00F015A46CDF80080FFF752F8E5
:10776800684B93F86B3003F00803DBB2002B00F092
:10777800A38399F82B10012209F1210001F00F01D0
:107788000323CDF80080FFF73DF83368554843F4EC
:10779800003300F180013360FFF712F855485A466C
:1077A80090F8E51100F5EC70CDF80080033001F099
:1077B8000F01FF23FFF726F87EE3CAF8008099F847
:1077C80020106FF07F4300934246FF2309F1160013
:1077D80001F00F01FFF716F82AB241F211139A428D
:1077E8001DD1434B5B7A302B13D1FFF77DF83368FB
:1077F800454668F3514368F38E3368F34D3333607D
:10780800414B1A7868F303021A7023780133237006
:1078180052E33E48F9F70EF83C49FFF745F8394E70
:1078280096F86B3013F0040F00F0468325B93848FA
:1078380020211022F8F7AEFD7F201CF015FC99F8E6
:1078480057106FF07F43002200933248FF2301F066
:107858000F01FEF7D7FF96F86B202F4B02F00F02AF
:107868000D2A1A7005D125B92C4A412191754FF47A
:1078780080551A78062A08D12AB2B2F5805F04D159
:10788800264A3621D1754FF488551A78082A08D126
:107898002AB2B2F5885F04D1204A3821117641F224
:1078A80010151B780B2B09D12AB241F210139A42FA
:1078B80004D11A4B2A225A7641F211150D486FF05D
:1078C8007F4390F8F0110022009300F5F370FF2336
:1078D80001F00F01FEF796FF96F86B3013F0010FD9
:1078E800AAD0E9E2FA4502081A010020C53A0020A8
:1078F800BC3A002001000020140D00201F0D0020BC
:10790800FC0000205C390020991700203801002075
:1079180004020020DD0C0020AA310020F401002020
:10792800900C0020A34B1A7842B300221A700F2043
:10793800FAF78AFB06460A20FAF786FB9E4B9F4910
:1079480058824A7812F0010F18D06436301A5883DA
:107958009B4B1A78642A01D19B321A701B78984E77
:10796800FF2B0BD00A21B3FBF1F1964B193119808B
:1079780095481CF061FA337801333370DFF864827C
:1079880098F8003013F00F0612D18E4B19228B484D
:107998001A804378192143F0010343708A481CF088
:1079A8004BFA8A4800F12001FEF70AFF04967CE2B0
:1079B800012E68D1804B5A8BA2F1690189B2112935
:1079C80008D8049911F0010F04D141F00101C9B29E
:1079D80004910592049A12F0020F0DD15B8A7C4A39
:1079E8001380A3F5C263023B9BB2D72B04D804983B
:1079F80040F00203DBB204931B20FEF783FF0599D6
:107A0800744B0AB2632A05DD642192FBF1F230322D
:107A18001A7401E0092A0CDD059A11B2642291FB5F
:107A2800F2F002FB10120A2012B292FBF0F230328E
:107A38005A74059802B2642092FBF0F100FB112100
:107A48000A2209B291FBF2F002FB101230329A744A
:107A58005B4B1B78FF2B08D158495B484B786FF379
:107A680000034B7000211CF0E7F9049A032A40F048
:107A780023825248002143786FF300034370524831
:107A88001CF0DAF911E2022E03D1534BC8221A6016
:107A98000BE2032E16D1504B1B68002B40F00C82D2
:107AA8004A4800F14001FEF78BFE1B20FEF72AFF33
:107AB800414B5B8AA3F51E630F3B9BB2542B00F22C
:107AC800FB81F2E1042E0CD13B4B988A0EF046FF65
:107AD800002840F0F1813D4800F16001FEF770FE9A
:107AE800E3E1052E07D1344B988A0EF037FF0328BF
:107AF80040F0E281D9E1062E40F0D78122786FF379
:107B0800030301322270D5E1344800F12001FEF769
:107B180057FE334B1B78002B00F0CE8123780133BE
:107B28002370304B1A786FF30302FFF794B82D4E89
:107B3800DFF8A480337813F00F021AD12A4800F135
:107B48002001FEF73DFE2948F8F774FE2749024652
:107B58002748F8F777FB2548F8F76CFE254BA3F87C
:107B6800160233785A1C62F30303337019F074FF5A
:107B780091E0012A16D1D8F80030002B40F09C8102
:107B880019F096FF012840F097811B48F8F752FE3C
:107B9800194902461948F8F77DFE002840F08C8103
:107BA80011486FE0D8F80020002A40F085810B21A9
:107BB8007BE000BF660E0020F82800201A2900206C
:107BC800A81700208C0C0020002C0140BA4602089F
:107BD8009C170020F40100202C2100203A470208BD
:107BE80098170020991700207A470208740100208E
:107BF800982F0020603E002092010020613E002066
:107C0800874E337813F00F080CD186484146FEF7AB
:107C1800D7FD33785A1C62F303033370824BA3F801
:107C2800028049E1B8F1010F18D1804804211BF006
:107C38002CFD002800F040817A4800F12001FEF771
:107C4800BFFD33784FF0FF315A1C62F303033370E2
:107C5800774B64221A60744B59802DE1B8F1020FFA
:107C6800DFF8CC811BD1D8F80030002B40F02481FC
:107C78006E4804211BF009FD002840F01D816A4B65
:107C88005880684800F14001FEF79AFD33785A1C85
:107C980062F3030333706423C8F800300CE1D8F8AA
:107CA8000020002A40F008810C21217062F30303B0
:107CB800A9E0604910234FF40052CB700D3B8B7044
:107CC8000A805D481BF092FC0A2200215B48F8F705
:107CD80061FB80201BF0EEFB237801332370504BAF
:107CE8001A786FF303021A70514BC8221A60E3E046
:107CF8005348DFF848A100F12001FEF761FD9AF82A
:107D08000030002B00F0D8804E48DAF80020444EAE
:107D18000260BAF8042082809AF8062082713178CD
:107D280011F00F0159D1DFF80881D8F800100029A7
:107D380040F0C2809AF80410A2F5A6524FF0640BE6
:107D4800103A0BFB01229AF805004FF00A0909FBCB
:107D580000200393F9F7E4FE3B49F9F7EDFF0246EB
:107D68009AF80200039BA0F5A65010380BFB030BF2
:107D78009AF80100354B09FB00B018600392F9F737
:107D8800CFFE039A01461046F9F71AFE304B1860E9
:107D9800F9F7D2FA1EA3D3E9002382468B46F9F7F6
:107DA800A5FD002800F08880504659461AA3D3E95B
:107DB8000023F9F791FD00287ED0FEF7DDFD33782A
:107DC80048465A1C62F303033370C823C8F80030CE
:107DD80008F0D2FFC0B207906EE001296CD10D30D7
:107DE8000799832200F044FD114BD3F80080B8F1C5
:107DF800000F61D140461BF05DFB237801332370EF
:107E0800337868F30303337056E000BFAFF30080A4
:107E1800736891ED7CFF7F400AD7A3703D008040D6
:107E280099170020DA4702080A330020000C0140A5
:107E38002C2100201629002000100140B017002036
:107E48003A4802080402002000007A44AC170020D7
:107E5800941700208448854E00F12001FEF7B0FCFD
:107E6800F37913F0010F27D0DFF8488298F80090D3
:107E780019F00F0920D17E4B0A2259781878103949
:107E880002FB0011B1701979D878103902FB001182
:107E98007170D9799B79103902FB0312327016F090
:107EA80031FFF37969F30003F37198F800305A1C35
:107EB80062F3030388F80030DFF8FC9199F800605A
:107EC80016F001063EF43BAE6A4B01221A7018F018
:107ED80069FD2378092B01D00D2B28D10120664993
:107EE80011F058FD654B664A5B7803F01F03D35CBD
:107EF800644A522B137002D1634B01221A70634BF0
:107F0800634A03F1200153F8040B8B4242F8040B37
:107F1800F9D1002117A811F067FD17A80D2119F054
:107F280037FD5C4B1A78013202F003021A7099F897
:107F3800006006F00206F6B2002E00F08B800EF00C
:107F4800BBFF13F03DF806980322431C93FBF2F2A3
:107F580002EB42029B1ADBB20693002B79D1DFF8C1
:107F6800488198F84960C246002E4DD0022E03D1B0
:107F780098F80130312B49D023780E2B13D146487D
:107F880046490522F8F786FC8246002840D1B21FF0
:107F980037484349F8F7D4FC344B5646DA7942F06F
:107FA8000102DA7135E00D2B03D13E483A49072228
:107FB80027E0032B22D13C4B002713F8012F2C2A52
:107FC80003D00137FFB2B742F7D113A832493A4676
:107FD800F8F7B6FC7B1C07E00AEB03025278303A4C
:107FE800D2B2092A03D80133DBB2B342F4D30AEB85
:107FF8000701FA430FA80231D21802E0264909A85E
:10800800721EF8F79DFC03E0069E02E0012600E0E0
:1080180000261E4B204A03F1100153F8040B8B4233
:1080280042F8040BF9D1214B214A03F1100153F80E
:10803800040B8B4242F8040BF9D1402388F8113025
:108048001C3B88F82230023B88F84B3019F028FA9C
:1080580000E0002699F8003003F0F5036FF3000301
:1080680089F80030FEF76BBD7A480208CC3700204B
:108078009E170020660E0020FD3D0020FC3D0020DC
:10808800387E02082332002098170020F4010020CF
:1080980066320020C63100206B3A0020BF32030848
:1080A800703A0020B01700206A3A0020040200202D
:1080B8007C3A002099170020443A0020AFF3008052
:1080C80010B5044640181146F8F756FB2046F8F755
:1080D800B1FBC0B210BD42540131C8B270470000B4
:1080E80010B50C4B0C4A1B780C460E2101FB0323E0
:1080F800997A31B101390523594301F56F5189B294
:1081080001E04FF46F510019042208F046FE201DCB
:10811800C0B210BD81400020A812002010B5054B48
:108128000C46197800190131042200F0A1FB201D2A
:10813800C0B210BD8140002000F5224000F5CF708C
:1081480008B5013008F018FE10F0FF0F14BF00202A
:10815800012008BD10B50A4600210446FFF7B0FF0C
:1081680001462046FFF7DAFF114A01462046FFF78D
:10817800A7FF232201462046FFF7ADFF0146204610
:10818800FFF7AEFF5B2201462046FFF7A4FF23223C
:1081980001462046FFF79FFF01462046FFF7A0FF54
:1081A8007C2201462046BDE81040FFF794BF00BF7F
:1081B800C532030810B55D220446FFF78CFF0D2277
:1081C80001462046FFF787FF0023235410BD38B52A
:1081D8001D460C4640182C1911461A4600F048FB5B
:1081E800E0B238BD2DE9F04118490446FFF7B2FF67
:1081F800174F0E263B78174D73430146EA5A20461F
:108208000423FFF7E4FF202201462046FFF763FF1F
:108218003B78014606FB035320469A7A0223FFF770
:10822800D6FF202201462046FFF755FF3B7801463E
:1082380006FB035520466A7A0323FFF7C8FF014669
:108248002046BDE8F041FFF7B5BF00BFC8320308BC
:1082580081400020A81200202DE9F047264E0E226A
:108268003378264F534337F90380FA1824494FF4DB
:108278007A73044698FBF3F8157AFFF76BFF4E22E2
:1082880001462046FFF727FF1E4B1C2202FB05353F
:108298005FFA88F8B8F1030F01460CBF05F1120226
:1082A80005F108022046FFF70BFFA146804600258E
:1082B80019E019F8013BA32B07D133780E2202FBF2
:1082C8000373204629465A7A08E0242B09D13378CB
:1082D8000E2202FB03739A7A204629460223FFF7EF
:1082E80076FF0135EDB24545E3D120462946BDE884
:1082F800F047FFF75FBF00BF81400020A8120020B1
:10830800D2320308587E0208074B187800F00400A0
:10831800C0B240B11A686FF382021A60034B0022A0
:108328001A70034B18787047C0310020D41700200A
:10833800BC170020054B00211970054B05481A6829
:1083480061F382021A601222F8F724B8D4170020C9
:10835800C0310020BC17002038B5084C08492278E5
:108368000546F7F76FFF23780021E954054B1A6893
:1083780061F382021A60207838BD00BFD41700204C
:10838800BC170020C0310020064A07491378112B7A
:10839800C85401D801331370044A136843F0040326
:1083A80013607047D4170020BC170020C03100208C
:1083B800054B1B7813F0010F05D1044B181810F862
:1083C800010CFFF7E1BF7047D5170020BA48020833
:1083D8002DE9F041334C002314F8101094F82A20AA
:1083E80001F00F0161F3030284F82A2004EB400036
:1083F80084F8293084F828304378DFF8B88063F3AC
:108408000712638C4FF4D277E38498F800302A2659
:108418007B4306FB0133244D2448E95A84F82A207B
:108428001BF008FD98F8003094F82A207B4302F0EE
:108438000F0206FB0233EB1859881C48013989B230
:108448001BF0FCFC01210A4618481BF0C3FC012163
:1084580016481BF0B0FC98F8003094F82A207B43AB
:10846800120906FB02331248E95A1BF0E3FC98F89C
:10847800002094F82A3057431B0906FB0376AD19F0
:1084880069880B48013989B21BF0D6FC01210A46DC
:1084980007481BF09FFC06480121BDE8F0411BF08E
:1084A8008ABC00BFD6170020C64802080008004052
:1084B800003401400218002030B5164C94F82B50B7
:1084C800A38445F00105002384F82B50628484F8C6
:1084D800211084F8203019E0C55CA5F13002D2B231
:1084E800092A08D9A5F14102D2B2052A9ABFA5F1F5
:1084F8003702D2B22A46084D013305EB420292F800
:10850800495392F84823257062700234DAB28A42DD
:10851800E2D330BDD6170020C6480208124B10B56A
:108528009A8C0024DA8483F8294083F8284022466C
:1085380001210E481BF04EFC64210C481BF07AFC0C
:1085480032210A481BF07AFC0121224608481BF018
:1085580041FC642106481BF06DFC05483221BDE84A
:1085680010401BF069BC00BFD6170020000800406F
:108578000034014010B500212C220348F7F70AFF08
:10858800BDE81040FFF7CABFD617002070B5214CD0
:108598002378042B39D8DFE803F0030D152A3000BF
:1085A8001D4B012093F82B3013F0010F30D02070B1
:1085B800013870BD184B93F82000FFF709FF02231C
:1085C800237022E0144DEE8CFEB9FFF7A7FF95F853
:1085D800203095F821200133DBB29A4285F820300B
:1085E80001D8042300E003232370304670BD0A4BF2
:1085F800D88C50B90123237070BD074BDD8C35B979
:10860800FFF7B8FF2570012070BD002070BD002065
:1086180070BD00BF03180020D6170020044B0022AD
:108628005A701A709A7842F001029A70704700BF27
:1086380018190020202102480A46F7F7ABBE00BFF0
:10864800F401002038B5044608460D46F8F7F2F85C
:1086580098B10319202B094BC8BFC4F120001C197D
:10866800002308E014F8012BE02A14BFEA5C20225A
:1086780004F8012C01338342F4DB38BDF4010020F7
:108688000D4B46F635321B689B6893420FD043F674
:10869800F82293420BD0122B09D0B3F5E97F08D00A
:1086A80046F6D9301B1A584240EB030070470120A8
:1086B80070470120704700BF3C180020F0B51F46E6
:1086C80087B006460C46084600211546F7F762FEB5
:1086D800244B07B19F80B3F9041005A801EB86016C
:1086E800042208F05AFB002605AB9B5D013BDBB278
:1086F800B92B34D81D2B4FEA031208D8D31803F529
:10870800164168465231112208F047FB0BE0164922
:10871800D3185B186A4603F11007186859680833BC
:10872800BB4203C2F9D12046F8F784F8C7B26846BD
:10873800F8F780F83818A84203D8E0196946F8F71E
:108748001BF86846F8F776F87B1C1B18AB4203D277
:10875800E0190649F7F778FE0136042EC4D107B0B0
:10876800F0BD00BF18190020F0140308EA3203080E
:1087780010B500216C220446F7F70CFE0123A37004
:1087880010BD002343700370837843F001038370A6
:10879800704700002DE9F0419378804613F0010FEF
:1087A8000D4614463AD06FF30003937018F050FE4C
:1087B8006378002B32D123780BB90A336370A3781E
:1087C800174F6FF30003A37018F042FE217807EBF0
:1087D80008066118073130462A46F8F7B1F83046DE
:1087E800F8F728F8C6B2AE420DD80AD20023237093
:1087F80006EB08000A33637038182021AA1BF7F724
:10880800C9FDAE420AD12278A3181B7A1BB10132E6
:108818002270BDE8F08123700A236370BDE8F081FF
:10882800F4010020054B1A780AB100221A701B784F
:1088380046F68A4202FB0311FFF704BF1F18002007
:10884800F8B505460C460818002108F08BFA013CDB
:10885800E4B26719384608F08FFAC6B2202E03D85A
:108868003846002108F07EFA0CB1202EEFD9F8BD69
:1088780002F00F03032B22F07F0230B5D2B20CD9DD
:108888004FF47A7491FBF4F42025E4B2057002B138
:1088980014B13034047000220130B1F57A7F05DB61
:1088A8004FF47A7491FBF4F504FB1511022B0BD9E4
:1088B800642491FBF4F42025E4B2057002B114B1EC
:1088C8003034047000220130632904DD642491FBF4
:1088D800F4F504FB1511012B0AD90A2391FBF3F3D4
:1088E8002024DBB2047002B10BB1303303700130C5
:1088F800092904DD0A2391FBF3F203FB121130313D
:10890800017030BD13B5104B01461B689A899C7BDA
:1089180012F0100214BF0220012034B10B4C9B7CD2
:108928002478634303FB001109B23AB10DF1060044
:10893800022208F032FABDF8060002E0084608F004
:108948001BFA00B21CBD00BF3C180020C91800204B
:1089580010B50F4B1B689A899C7B12F0100214BF4C
:108968000221012134B10B4C9B7C2478634303FB27
:10897800010000B22AB108490222BDE8104008F0FF
:1089880006BA054B1968BDE8104008F0EBB900BFFE
:108998003C180020C9180020E01800203038C0B268
:1089A800092894BFFF20002070470000024B1A7866
:1089B8006FF300021A7070470919002070B5FFF7AD
:1089C800F5FF884B1A781E2A01D91E221A70864C88
:1089D8002678254606F0F006202E72D108F040FDD4
:1089E80000286ED1814B1B7833B92378C3F3031267
:1089F800013262F307135EE07D4B1B7803F08003BE
:108A0800DBB2002B59D07B48F7F714FFC5B27A4C7C
:108A1800BDB1204679493246F7F792FF0A2D0BD8A7
:108A28002A4620467349F7F78BFF60193146C5F18E
:108A38000A02F7F7AFFC04E020466E490A22F7F76E
:108A48007FFF6F4B1B7813F0010F01D0472300E025
:108A58002023E372684C042204F10C00A521F7F7E7
:108A680099FC684B1A7852B1FF23012A237306D95F
:108A7800022A637303D0032AA37318BFE373624CFB
:108A8800257815F0600502D194F8A33013B95F4832
:108A98005F4902E05D4804F1A3010622F7F750FFA1
:108AA8005C4B1B78452B40F09A81002D40F0978154
:108AB800237843F08003237070BD4F4856493246EF
:108AC80082E12C7804F0F004102C3FD108F0C8FCA7
:108AD80000283BD1202251494748F7F731FF464843
:108AE8004E492246F7F72CFF4D4B1B7813F0010F28
:108AF80006D04C48F7F79EFE4A4902464A4805E028
:108B08004A48F7F797FE494902464748F7F718FFDA
:108B1800364B1B781BB946484649102254E1444855
:108B280045491022F7F70CFF314B1B7803F08003FF
:108B3800DBB22BB13B48F7F77DFE02463F484FE0DA
:108B48003A48F7F777FE02463C4842E02B7803F0B4
:108B5800F003302B7ED108F083FC00287AD1264C14
:108B6800202237492046F7F7EBFEA521052204F11C
:108B78000B00F7F70FFC334B1B78042B02D9FF23AC
:108B8800E37300E002D1FF23A37301E0032B02D1BA
:108B9800FF23637301E0022B02D1FF23237300E05C
:108BA8000BB1FF23E372284B5B7813F0600F05D0FD
:108BB8003F23E37223736373A373E373234B1B781D
:108BC80003F02003DBB233B11848F7F733FE02464F
:108BD8001F481649F8E01348F7F72CFE02461C48D0
:108BE8001049F1E015190020091900205C21002026
:108BF8003021002034210020F4010020DCDA0208B2
:108C08007840002029220020642100200E02002044
:108C1800F7B00208041800209ADA0208DF100308E7
:108C28006E34002029120308010200204A120308AA
:108C380004020020AC1603080011030811020020EA
:108C48009CB10208E723002020290020C031002021
:108C58000F0200202B7813F0F0030CD1202260497A
:108C68006048F7F76DFE604B5E4819888322BDE8BF
:108C78007040FFF7FDBD602B1ED108F0F1FBD8B99D
:108C88005A4920225748F7F75BFE5948F7F7D2FDB3
:108C9800574902465748F7F753FE5748F7F7CAFDB2
:108CA800554902465548F7F74BFE5548F7F7C2FDB8
:108CB80053490246534887E02B7803F0F003102B02
:108CC80006D108F0CDFB18B146484F4920227BE079
:108CD8002B7803F0F004402C02D0502C78D108E017
:108CE80040484A492022F7F72BFE494B1B784BB9DD
:108CF8004CE03C4847492022F7F722FE464B1B78B8
:108D08003BB943E0454B5A7882B11B78022B14D10A
:108D180005E0434B1B7813F0010F07D00DE04148E5
:108D2800F7F788FD3F4902463F4835E03F48F7F7E7
:108D380081FD3E4902463C482EE03D48F7F77AFD62
:108D48003B4902463848F7F7FBFD402C0BBF334B35
:108D5800384B5B78DB78022B0AD0042B0FD0012B21
:108D68001CD13548F7F766FD3349024633481BE006
:108D78003348F7F75FFD32490246304814E031487E
:108D8800F7F758FD2F4902462C480DE02E48F7F713
:108D980051FD2D4902462448F7F7D2FD2B48F7F735
:108DA80049FD2A4902462548F7F7CAFD284B1B7892
:108DB800ABB9202107222148F7F7ECFA2248F7F748
:108DC80039FD214902461D48BDE87040F7F7B8BD96
:108DD800204A6FF3071313701F4B00221A6070BDEF
:108DE80039B10208F40100201A18002018B102084D
:108DF80018AA0208F801002022AA02080802002086
:108E08001DAA02080F0200207BB1020821110308E5
:108E1800A8310020421103085C210020BA2D00204F
:108E280078400020E7110308FD0100208C12030898
:108E38002912030804210020631103080D020020F1
:108E480084110308A51103086B120308C61103084F
:108E58009F2B0020091900203C180020204B70B5DA
:108E6800F022204D1A702B7813F0010F0BD01E4CF6
:108E7800207810F0010006D11C49FFF7D3FC2378B5
:108E880043F0010323701A4E3378532B0ED1164C3E
:108E9800237813F0010F07D000201649FFF7C2FC12
:108EA80023786FF300032370FFF780FD3378232BBB
:108EB80014D10D4B1B7813F0010F0FD1FFF776FD7E
:108EC8002B780D4A43F006032B701378013BDBB275
:108ED80013700A4A52F82320094B1A6070BD00BF6C
:108EE800151900200919002041180020B0060308B0
:108EF800041800208F060308F7180020F81800202F
:108F08003C1800202DE9F0415C4BF0225C4D1A70B2
:108F18002A7802F01003DBB2002B2DD1594963F3F4
:108F280047120B601C462A70574A9A5C2D2A01D0BA
:108F38000134E4B20133082BF6D1544E3A213046BD
:108F4800F7F7A6FA38B1801BC0B2013030182146B5
:108F58000222FFF78DFC4E4B1B78452B40F08B808F
:108F680000242046013412F083F8082CF9D12B781C
:108F780043F010032B7038E0464C237813F0010FB0
:108F880017D1404E4448FFF7F3FB404F316838464D
:108F980001310222FFF76CFC2D23BB70307846F6B6
:108FA80061533E496522FFF789FB237843F00103AB
:108FB800237003200D21384AFFF7ECFB2D78304E43
:108FC80015F0E00541D110203549FFF72BFC304B57
:108FD8001B78442B0DD12B4A136801332A4903F01F
:108FE8000703C95C2D29F8D01360BDE8F041FFF7ED
:108FF800DDBC532B0DD132784E3B63F347123270F0
:10900800204A28491268062000FB02125380BDE856
:10901800F081232B2FD11B4B1D60337803F0EF0316
:1090280065F347133370FFF7C1FC23781E4A43F0FA
:10903800060323701378013BDBB213701B4A52F806
:1090480023201B4B1A60BDE8F081104C10201949F1
:10905800FFF7E8FB04F110002821F7F719FA50B1DF
:10906800001B3178C0B20130201849098022BDE8C0
:10907800F041FFF7FDBBBDE8F08100BF15190020E6
:1090880041180020E0180020ED320020F4010020F3
:109098000418002009190020181900201F190020A1
:1090A8002C0603080A330020F7180020F8180020BF
:1090B8003C1800204D060308454B2DE9F041F022ED
:1090C800444E1A703378444D43F0010333702B68D3
:1090D800424C9B7C022B06D1414B1B7803F040038A
:1090E800DBB23BB10FE0012B0DD13E4B1B7813F0E7
:1090F800010F08D108F026FB236800206FF35553B1
:109108002360394944E0A378344F03F02003DBB2ED
:10911800C3B908F017FBF87800F02000C0B288B98E
:109128002968324B897C1A7861F301021A703B680E
:109138002D4943F400133B60FFF774FB2C4B80224E
:1091480083F843200CF0BAFF804678B12B689B7CEB
:10915800012B08D1234B5B7803F01003DBB213B16A
:109168000020244914E00020234911E00CF0D6FF28
:10917800074610B1404621490AE00DF017F810B132
:1091880038461F4904E01A4B93F8433013B91D4978
:10919800FFF748FB1C4B1B78232B16D1FFF706FC67
:1091A800337843F00603337008F0CCFA23686FF382
:1091B800555323600BF076FE144A1378013BDBB25B
:1091C8001370134A52F823302B60BDE8F08100BFBA
:1091D80015190020091900203C180020C031002072
:1091E800302100206E340020D1060308733400209B
:1091F800B11C002013070308F206030855070308EB
:10920800340703087607030804180020F71800201D
:10921800F81800202DE9F3416E4B6F4DF0221A70BB
:109228002B686E4C9B7C1BB9637843F0100302E0FB
:10923800637843F008036A4E6370337843F00103A0
:109248003370238823F47E6323F01E03DB04DB0CD6
:10925800B3F5805F08D0634B1B7883B15F4B5B78B5
:1092680003F00803DBB253B1637800206FF34103C6
:109278005D496370FFF7D6FAF8F722FF84E0637858
:10928800564F03F00203DBB2FBB9BB78EBB9574B7F
:1092980093F8008018F0010817D1F8F711FF7B78D0
:1092A80043F002037B702B68B3F91030022B7B78F4
:1092B8000CBF43F0040368F3820300217B7008208D
:1092C80001220B460091F9F717FAA378434A032BBA
:1092D80028D003D8012B0BD00DD806E0052B2DD0B4
:1092E800517825D3FF2B32D12BE000203E4949E0AD
:1092F80000203F4946E03F48F7F79CFADFF82C8109
:10930800C7B23C4908F110003A46F7F719FB0F2F8E
:109318003AD807F1100040442021C7F11002F7F7AE
:1093280039F831E0344B187800282DD1334929E039
:109338006FF3410151700020314923E00020314989
:1093480020E06FF34101517000202F491AE0053BDE
:10935800DBB26FF34101022B517002D100202B497F
:1093680010E0012B02D1002029490BE0032B02D188
:109378000020284906E0052B02D10020264901E0FB
:1093880026490020FFF74EFA637803F00203DBB2A8
:109398000BB9F8F795FE224B1B78232B18D1FFF752
:1093A80005FB3378002243F0060333706378A2701C
:1093B80003F0E50362F382036370F8F781FE194A4C
:1093C8001378013BDBB21370174A52F823302B6035
:1093D800BDE8FC81151900203C18002078400020C9
:1093E80009190020BA2D0020D10603087E4000206C
:1093F80014030308874000207C400020350303083D
:10940800D9070308B90303081C0403085603030813
:109418007703030898030308DA030308FB03030828
:1094280004180020F7180020F8180020F401002084
:109438007B4B2DE9F341F0227A4E1A7033787A4D3E
:1094480043F0010333702B68784C9B7C022B11D1BD
:10945800774B1B7803F04003DBB293B1754B1B7855
:1094680003F02003DBB2BBB1A37803F04003DBB207
:109478003BB111E0012B0FD16F4B1B7813F0010F9B
:109488000AD1F8F71DFE2368002023F480036FF348
:10949800D753236069498FE0A778DFF8908107F0F8
:1094A8004003DFB2002F34D1F8F70AFE2968644B75
:1094B800897C1A78384661F301021A70D8F80030AE
:1094C8005E4943F4800367F3D753C8F80030FFF7C9
:1094D800A9F92B68198A21B90091082001220B46A5
:1094E80015E00BB2022B0CD101223B46082039466D
:1094F8000097F9F701F9534B1A7842F008021A70ED
:1095080007E0012B05D100970E2039463A46F9F7B6
:10951800F3F80CF0D3FD074678B12B689B7C012B40
:1095280008D1454B5B7803F01003DBB213B1002080
:10953800454941E0002045493EE0414B394618780D
:1095480000F00300F8F7F4FEFF280FD13D4B1B781D
:1095580003F01803182B31D0A07800F08000C0B2B7
:1095680010B138463A4927E03A4925E00CF0D6FDD3
:109578008046E0B1334B187800F008085FFA88F8A5
:10958800B8F1000F0AD1F9F727F8C0B2022801D8BC
:1095980040460AE0062811D8404604E000F01000D2
:1095A800C0B210B138462C4906E02C4904E00CF052
:1095B800FDFD18B12A494046FFF734F9294B1B78BD
:1095C800232B29D1FFF7F2F9337843F006033370E0
:1095D800F8F776FD236823F480036FF3D7532360ED
:1095E800184B1A786FF3C3021A701F4A1378013B9D
:1095F800DBB213701D4A52F823302B60104B1B78D6
:1096080003F00303022B02D10CF02EFD20B102B0AF
:10961800BDE8F0410BF046BC02B0BDE8F08100BFE8
:1096280015190020091900203C180020C03100201D
:1096380030210020642100206E340020D106030868
:1096480073340020401A002013070308F2060308A9
:10965800D9070308FA070308B80703089707030898
:109668003407030804180020F7180020F818002011
:1096780010B5FFF79BF9124B2522DA77114B124CE4
:109688001B6818219A7C01FB0242517801F00F00F7
:109698000F2814D00A2803DD0A2060F30301517053
:1096A8009B7C182202FB034463780A2103F00F0312
:1096B800594306486B32BDE81040FFF7D9B810BDD2
:1096C800F40100203C180020CC31002010020020BA
:1096D8002DE9F74F984BDFF8B0A2F0221A70DAF8AC
:1096E8000030D0469C6847F2DB13E11A4C4244EB49
:1096F8000104D83A6243914B9D5C9F18C5F300055D
:10970800EEB29946002E29D130468D49FFF78AF8E6
:109718008C4B1B78232B40F038857B7866F3041339
:109728007B70FFF743F9884B1A7842F006021A70EB
:10973800864A1378013BDBB21370854A52F823300E
:10974800CAF80030834B1D70834B1D70834B1D700E
:10975800834B1E60834B1D7000F017BD824E814DF8
:10976800337893B1814A4FF4A071137803F01F0046
:109778005B0959430A2303FB00137D49CB18DB78A7
:10978800002B40F06682137084E06E4B1B78532BDD
:1097980040F0FC8095F80080B8F1000F2ED14046CB
:1097A800214614F080FE5FFA80FABAF1000F25D046
:1097B8007B7868F304137B706E4F3A781AB92046A9
:1097C80014F088FD13E0531E6B49002B184603EA7A
:1097D8000101B8BF02F11E004011002903DA013966
:1097E80061F01F01013114F0C1FD00233B7014F03A
:1097F800EDFE85F800A00022594BE2E02B78002B03
:1098080000F0278256490A680F460B2A01D10C231B
:1098180016E00C2A11D1013B6101544A5918117004
:10982800554903EA0101002903DA013961F01F01F2
:109838000131204614F09AFD1CE0092A02D10A23BE
:109848000B60D0E10A2A27D14B49013B03EA010109
:10985800002903DA013961F01F010131204614F0B3
:10986800C7FD2B786201D318DBB2404A591E11702C
:10987800404A13704FF00008C7F80080FFF796F8C9
:10988800182303FB04935A7842F010025A7085F8A3
:10989800008014233370DCE1043A042A3FD83749A6
:1098A800D2B20878364F60B300200870397841B1D9
:1098B8003448401810F8010C032802D0002840F062
:1098C800C881013B0A2058434FF4A07E0EFB0400D8
:1098D800DFF89CE070448018417160011B18D8B211
:1098E80000EB800000F5EC405F30801807F03AFA92
:1098F800387818B1013814F0D1FEAAE10DF088FBD0
:10990800A7E101200870013B0A214B434FF4A071E5
:1099180001FB04331649CB189A1853790AE00F4F04
:109928003B7823B901223A700A4A137091E1FFF794
:109938003DF800233B708CE115190020CC31002044
:1099480067BF02080418002009190020F718002032
:10995800F8180020211800204A180020C9180020F3
:10996800E0180020D318002018180020CA1800207A
:1099780045350020851900201F000080DF180020D1
:1099880084190020E82300203C180020432B1AD11A
:10999800964A1278002A40F043812B78002B00F079
:1099A8005881934B1A78002A40F05381914B1968DB
:1099B8000C2903D00A2903D02A7014E10B2200E0F5
:1099C80009221A600FE1232B7ED1884A1278002AD7
:1099D80040F026812978DFF818A2002935D09AF8B6
:1099E800003053B184490F2B0A7084490A7000F281
:1099F800308101338AF800302BE17E4A1368082B46
:109A08001ED84FF4A077674301394FF00A0E0EFBBA
:109A180001717B4F181F7918C9780627013907FB90
:109A28000101784800EB810151F8040F0133002847
:109A380040F0D880032B40F2D580082BF4D9D1E030
:109A4800092B40F006810233CCE07B786E4E61F33F
:109A580004137B7032781AB9204614F03BFC13E0EB
:109A6800531E6A49002B184603EA0101B8BF02F1E8
:109A78001E004011002903DA013961F01F0101318C
:109A880014F074FC0023337014F0A0FD0DF0C0FA3C
:109A9800FEF78CFF5E4B1A7842F006021A705D4A98
:109AA8001378013BDBB213705B4A52F82330524AF9
:109AB800C8F8003000231370504A8AF80030137039
:109AC8004C4A2B70136060E32A2B3CD1474A12782A
:109AD800002A40F0A58046490B784BB14648012B37
:109AE80002704648027040F2B480013B0B70B0E04F
:109AF8002878002800F0AD803E4A1368002B00F05B
:109B0800A880092B1AD84FF4A071614301384FF08F
:109B18000A0E0EFB00103A491F1F0818C1780620CC
:109B2800013900FB0171374800EB810151F8040D40
:109B3800013B002856D1032BF8D853E00B2B40F0FB
:109B48008880023B4EE0442B1AD1284A1278002A1A
:109B580066D1274B1B78002B7BD12878431EDBB2BC
:109B68001E2B76D8214614F09EFCC0B2002870D077
:109B7800204A13680C2B6CD00A2B6AD028701BE083
:109B8800552B4DD1194A1278002A49D1184B1B7808
:109B9800002B5ED1287801285BD90238214614F0C1
:109BA80093FCC0B2002854D0124A13680C2B50D032
:109BB8000A2B4ED019490870043B042B13D84FF4D4
:109BC800A071614301380A2707FB00100C490818E7
:109BD800C1780620013900FB01330A4951F82330C6
:109BE8000BB904331360FEF7E1FE32E0DF18002002
:109BF800C9180020E0180020211800204A18002069
:109C080045350020840D0020851900201F000080A4
:109C180009190020F7180020F8180020D318002090
:109C2800303BDBB2092B14D89C4A1268043A042A48
:109C38000FD89B4A117861B99A4A12784AB19A4A60
:109C48000A27107807FB0033DBB2402B137088BF5C
:109C580011702F78DFF8B482002F5FD198F80000D8
:109C680010F0010012D114B92046904900E0904943
:109C7800FEF7D8FD98F8003043F6DF2043F00103E3
:109C880088F8003007F078F88A4B1870337813B9E1
:109C980089488A4901E0884889490A22F6F750FE2E
:109CA800204614F0EFFB874D0146022205F119000A
:109CB800FEF7DEFD844B1B7803F08003DBB22BB389
:109CC800824B1B88EB81337803BB814B18781A468B
:109CD80018B9204614F0CAFA18E07E4B411E01EA72
:109CE8000303002B03DA013B63F01F0301334FF436
:109CF800A07161430A2505FB03137749CB18DB786C
:109D080013B914F091FB01E000231370182303FB2F
:109D18000494637843F01003637036E24FF4A07341
:109D28006343013F0A2202FB07336B4EF31893F893
:109D380003B06301FF1898F80030FFB213F0010F69
:109D480046D16648FEF714FD07EB071101F5E2411D
:109D5800DF311022624807F020F8604B5948112281
:109D68009A7144230370173BC370791C01300F3A72
:109D7800FEF77EFD494B1B6813B9102059491FE0B7
:109D8800012B02D1102058491AE0022B02D11020D1
:109D9800564915E0092B02D11020554910E00A2B2D
:109DA80002D1102053490BE00B2B02D1102052494D
:109DB80006E00C2B02D11020504901E05049162032
:109DC800FEF730FD98F8003043F0010388F80030C2
:109DD800334B1A789846002A00F0EB8007EB0717F8
:109DE80007F5E247DF3710223648394606F0D5FF37
:109DF80000229146334B995C9A4641B109F1010919
:109E08005FFA89F90132B9F1100FF3D106E003EBDB
:109E180009002021C2F11002F6F7BCFA98F80000F8
:109E280048450BD90138C01906F0A6FF30B91C4BBC
:109E3800202118780138C01906F094FFDFF8D09077
:109E480099F8003018460193FEF7A8FD4A46019B91
:109E5800DFF8C09018B9432B40F0858001E0432B10
:109E680004D1002389F80030202173E0DFF8A8E04E
:109E780024499EF800C024489C454FD10B78ACF18A
:109E8800300C0133DBB24FF00A0E0B700EFB0C33B3
:109E9800C35C002B54D10B7052E000BFE0180020C7
:109EA800C9180020DF180020841900200CC00208FF
:109EB80090C0020853320020FA01002035C1020880
:109EC80056C10208F4010020C0310020E93203081D
:109ED800851900201F000080453500201819002032
:109EE8001F1900205EC202083DC202087FC2020894
:109EF800EAC302080BC402082CC402084DC40208B5
:109F08006EC402084A180020344C020809190020BF
:109F180004180020211800201E1800208EF8003098
:109F280099F800304FF0000C81F800C043B198F860
:109F380000300F2B04D803F1010E954B83F800E095
:109F4800402389F8003013780978303B0A2202FB55
:109F58000313C15C98F8000001380AF8001038189B
:109F680006F000FF0EE08B4B1B7803F08003DBB29A
:109F780043B199F800302BB998F80030FF225344C8
:109F880003F8012C99F8003013B1834A013B137090
:109F980099F80030012B11D198F800300F2B02D816
:109FA8007B4A013313707D4A002389F8003013700F
:109FB80004E004200C217A4AFEF7ECFB794B1F6879
:109FC8001FBB4FF4A07254432B780A22013B02FBBB
:109FD8000344361975782D090F2D00F0D680724C80
:109FE800A52104F11C00063AF6F7D4F9FF232377DC
:109FF800002D00F0CA80012D637700F0C680022D85
:10A00800A37700F0C280E377BFE0012F18D14FF4A7
:10A01800A07254432B780A21013B01FB03443619F3
:10A02800737803F00F030F2B00F0AF80092B04DCCB
:10A0380001335E485943BD3AA2E05C4859436AE09F
:10A04800022F38D10BF1FF3B5FFA8BFBBBF1070FF7
:10A0580098BF574BDFF850819CBF5B4493F86470FE
:10A0680008F11B0088BF002720210522F6F792F986
:10A078002878C7EB08080138002318E04FF4A072CD
:10A0880062430A2101FB0022B25C08EB07011A4176
:10A0980012F0010FC7F1000202D08A18DB2101E09B
:10A0A8008A18A52182F82010013308F10108DAB2D4
:10A0B800BA42E3D369E0032F2FD14FF4A07254437F
:10A0C8002B780A25013B05FB0343F218F35C13F0D8
:10A0D800400F02D01020374906E093785A1ED2B2BA
:10A0E800FD2A06D93449102003B0BDE8F04FFEF729
:10A0F80099BBFE2B02D110203049F5E710203049DA
:10A10800FEF790FB2F4B30481B78013B05FB0344BF
:10A118002E4D2C19A178832232E0043F042F34D825
:10A128000622FFB20BF1FF3B02FB0B7B284B2948B1
:10A1380053F82B100A31F6F703FC274B1B7893B121
:10A14800144B1B7803F08003DBB23BB1234820217A
:10A15800022203B0BDE8F04FF6F71CB9204B1F48A8
:10A16800197882220CE02B780A22013B53434FF4E2
:10A17800A07202FB04343619F71918487979BE3AE7
:10A1880003B0BDE8F04FFEF773BB03B0BDE8F08F36
:10A19800C9180020C0310020211800204A180020CA
:10A1A80018190020E0180020F40100200F020020F8
:10A1B800344C0208A8C30208A0C20208C1C202089F
:10A1C800C9C30208D3180020110200204535002019
:10A1D800840D002004020020DF1800201202002055
:10A1E800841900202DE9F0474C4C4D4F2378F0227C
:10A1F80043F0010323704B4BDFF85C911A703B6806
:10A20800494A9E6847F2DB13F01A464246EB0006BD
:10A2180018217143555C5318C5F300055FFA85F89A
:10A228009246B8F1000F23D140464049FEF7FAFAAA
:10A2380099F80030232B6FD1FEF7B8FB23783C4AFE
:10A2480043F0060323701378013BDBB21370394ADD
:10A2580052F823303B60384B1D70384B1D70384B1B
:10A268001D70384BC3F80080374B1D70BDE8F08770
:10A2780099F80020232A23D15A786FF304125A70D0
:10A2880014F0A4F90CF0C4FEFEF790FB2378284ADA
:10A2980043F0060323701378013BDBB21370254AA1
:10A2A80052F82330244A3B6000231370234A13706A
:10A2B800234A1370234A1360234A1370BDE8F087BA
:10A2C800532A0DD15A78C2F300144CB942F0100247
:10A2D8005A7021463046013414F048F8202CF8D141
:10A2E800304614F0CFF8182303FB06A67378C1B2E2
:10A2F80013F0100F0AD0202902D10020134901E0E1
:10A3080013490020BDE8F047FEF78CBA1148022235
:10A31800BDE8F047FEF7ACBABDE8F08709190020A0
:10A328003C18002015190020CC31002067BF020816
:10A33800F7180020F8180020211800204A180020DB
:10A34800C9180020E0180020D3180020E9090308E4
:10A358000A0A03080D020020041800202DE9F04124
:10A368002D4E2E4F307800F5E240BD3006F004FD4A
:10A378003B78C4B213F0010F26D0294D2B78552B0A
:10A388000AD1EC2C01D0013CE4B23078214600F52A
:10A39800E240BD3006F0E6FC2B78442B0DD1A4F149
:10A3A8001403DBB2D72B01D90134E4B2307821464B
:10A3B80000F5E240BD3006F0D5FC2B78532B03D1D5
:10A3C800FEF7F4FA0CF024FE164B1B7803F080031A
:10A3D800DBB253B13B7813F0010F06D012482021AD
:10A3E8000422BDE8F041F5F7D5BF14F0800F0F48FF
:10A3F80005D12B230A2103746143113006E02D2374
:10A408000374373B5C43113004F520610322BDE837
:10A41800F041FEF72DBA00BFC91800200919002025
:10A4280004180020C031002004020020F40100209C
:10A438001FB5204B20491A781AB1087840F001005E
:10A44800087009781C4C11F0010F31D01B490978AC
:10A45800532901D00AB103E082B901221A700DE034
:10A4680023290BD1002018701549FEF7DBF9FEF7F8
:10A478009DFA237843F00603237019E01B78012B1B
:10A4880016D120210A460F48F5F784FF0E4B68467F
:10A498001B681022996806F080FC002409491DF801
:10A4A800040001EB4401013418F01EF9102CF5D119
:10A4B8001FBD00BFC918002009190020041800207A
:10A4C800220D0308F40100203C180020034B1B78E0
:10A4D800532B01D1FEF76ABA704700BF0418002059
:10A4E800084BFF281A68936807D1917B41B1064948
:10A4F800927C097801FB023302E0927C02FB003374
:10A50800184670473C180020C91800204328F8B5A1
:10A5180004460D46174608D1114B0A261A7891FBB6
:10A52800F6F66FF3C3021A7000E00E462046FEF7F7
:10A5380035FA90B10A4B303C1A780A2602F0080125
:10A54800C9B2002918BF002506FB05466FF3C302F0
:10A5580036B21A70BE42A8BF3E4630B2F8BD00BF40
:10A5680009190020634B2DE9F3411A689846157CB8
:10A57800977C614C2DB1614821780222FEF778F969
:10A5880000E02570FF01237807F50C473C3707EBFF
:10A5980043075B4E0BB90DB10FE015B901A8394659
:10A5A80001E001A8B91E022206F0F7FB9DF804306D
:10A5B800F3759DF80530337605E006F117003F2165
:10A5C8000222F5F7E7FE5B23B375023373764D4B32
:10A5D8001B7813F0010F61D04B4B1B78A3F13002AD
:10A5E800D2B2092A35D822780AB9002D40D1474A73
:10A5F800117814469942464A01D000211170DFF8BB
:10A6080014E10DF1080C9EF800E0A3F13000E644D7
:10A61800DFF80CC1117800EB8000604400EB010CFE
:10A628000131C9B240189CF86CC090F86C000EF863
:10A6380004CC117008B1032901D9002111702370CD
:10A648000DB9384600E0B81E01A9022206F09FFBAA
:10A6580017E0232B04D12F4B1A7892B9013205E069
:10A668002A2B05D12B4B1A785AB1013A1A7008E0F7
:10A67800532B06D1284A533B1370264A1370FFF711
:10A6880025FF264B1B7803F08003DBB2002B2FD06D
:10A69800204B1B78F6182023F37529E045B31A4B95
:10A6A8001878A0F13003DBB2092B10D81A4A1378B6
:10A6B80003B92370013303F001031370D8F8003095
:10A6C8002178B3F91020FFF721FF207005E0432817
:10A6D80003D1114B1B7803B92370104B1B7803F07F
:10A6E8008003DBB223B1054820210222F5F752FE90
:10A6F800BDE8FC813C1800204B1800200202002015
:10A70800F401002009190020041800201E18002058
:10A718004A1800201C180020D3180020C03100203F
:10A72800344C0208F7B5394E394D3378394C6FF34C
:10A738004103337016F07EFCFFF7C8FE02238DF844
:10A7480007302B788BB1344AD17941F00101D171AE
:10A75800324A207802EBC303D3F8A07093F8A520FF
:10A768003978FFF7D3FE38700DE0337813F0010F16
:10A7780006D02378303BDBB2062B9CBF264AD37029
:10A7880003238DF80730337813F0010F12D0244BD0
:10A798001B7803F08003DBB263B129781F4B214893
:10A7A80003EBC10393F8A4309DF80720C0182021BB
:10A7B800F5F7F0FD2378232B09D11B4A2B78126873
:10A7C800927C013A934202DA114A013313702378DA
:10A7D8002A2B04D12B7813B10D4A013B137023782F
:10A7E800532B0FD114F08EFA0B4B00212970DA7914
:10A7F80061F30002DA71FFF769FE0C4B9A7942F0B7
:10A8080004029A7100232370FEBD00BF09190020BD
:10A81800D318002004180020CC370020344C02083C
:10A82800C0310020F40100203C180020341A002018
:10A838002DE9F74F864E874C3378874D232B874F6A
:10A8480025D12368986843F6F123984217D1DFF899
:10A858003482296898F8000000F56A50713006F0D3
:10A8680081FA98F80000013000F0010088F8000033
:10A8780000F56A50713006F07FFA286007E000B2F0
:10A88800FEF740F828603B7843F008033B703378C4
:10A89800532B40F06E81236848F6E9329B68934257
:10A8A80002D12A686E4B15E04AF28A32934202D1ED
:10A8B8002A686C4B0EE04AF20732934202D12A68AA
:10A8C800694B07E048F63A42934204D12A68674B3D
:10A8D80002B101221A7023689A6843F6DD239A426E
:10A8E8000AD1634B29681A7861F300021A7006F0DE
:10A8F800B7FD08B106F0D2FD236843F6E0229B6855
:10A90800934206D15A4B29681A7861F3C7121A7014
:10A9180019E043F6EA22934206D1554B29685A7842
:10A9280061F300025A700EE043F6E72293420AD11F
:10A938002968504B19B11A6842F0005202E01A68AF
:10A9480061F35D721A6023689A684AF220439A425A
:10A958000AD12968484B19B11A7842F0200202E05E
:10A968001A7861F345121A7023689A684AF2AD435F
:10A978009A4202D1287817F0C5F8236843F6DA22FC
:10A988009B68934202D12A683C4B05E043F6E822D3
:10A99800934203D12A683A4B1A7008E048F6F2321B
:10A9A800934204D12B6813B92B4B01221A602368F8
:10A9B8009A684AF2AE439A420BD1324A2B6812780F
:10A9C8003149032B8B5404D1304B5A7942F0100291
:10A9D8005A71236848F632429B68934202D129682B
:10A9E8002B4A05E048F63542934203D12968294AA3
:10A9F800117016E048F63642934203D12968264A78
:10AA0800117015E048F63842934203D12968234A69
:10AA180011704DE048F63942934202D12A68204B22
:10AA280013E043F60452934202D12A681D4B0CE00E
:10AA380049F24062934202D12A681B4B05E04AF270
:10AA48009E32934234D12A68184B1A703BE000BFFB
:10AA5800041800203C180020E018002009190020E4
:10AA68005C210020A83100209F2B00200218002024
:10AA780086190020C0310020784000205A3A002072
:10AA880009320020C9180020A0120020042100204B
:10AA9800403500203E35002071340020E533002089
:10AAA800B41A0020DE10002039170020BA17002041
:10AAB80048F6EA32934206D12A68A14B01201A705F
:10AAC80001460DF0AFF82368986843F6F1239842E1
:10AAD8000DD1DFF87882296898F8000000F56A50EF
:10AAE800713006F03FF9002388F8003002E000B228
:10AAF800FDF72EFF23689A6843F698139A4236D1D9
:10AB08002968DFF844B2DFF84CA20BEBC1031B79CC
:10AB1800DFF83882C3F34113012BDFF83C9221DDC3
:10AB280098F8000000F56650203006F01BF998F8F8
:10AB38000030DAF8001009EB030211720BEBC102C6
:10AB48001279C2F34112032A0CD17E4A1268906826
:10AB58001030C01806F006F998F80030DAF800202E
:10AB68004B441A7498F800302A6809F80320FFF754
:10AB7800ADFC3B78DFF8E48113F0010F00F0F080C2
:10AB8800216843F698128B68934240F081806E4AA0
:10AB98002B68914602EBC3010979C1F341110129E0
:10ABA80006DD6A4A1278072A02D9FDF7FFFEE3E0BC
:10ABB8003278442A36D15FFA83F82DE008F101088B
:10ABC800614B5FFA88F803EBC8031B79C3F34113A1
:10ABD800012B06DD5E4B1B7823BB5C4B1B78072BD8
:10ABE80020D8DFF868A19AF800301F2B08D806F0A3
:10ABF80037FC70B109EBC8031B7913F0100F08D1AB
:10AC08009AF800301F2B07D909EBC8031B79DB0919
:10AC180002D0C5F8008005E009EBC8031B7913F0E2
:10AC2800080FCBD03378552B40F0A6802E782CE037
:10AC3800013EF6B209EBC6031B79C3F34113012B9E
:10AC480009DD434B1B78002B40F096803F4B1B7867
:10AC5800082B00F29180DFF8F48098F800301F2B61
:10AC680008D806F0FDFB70B109EBC6031B7913F099
:10AC7800100F08D198F800301F2B06D909EBC6032E
:10AC88001B79DB0901D02E6076E0002ED0D173E06D
:10AC98004AF2AE4293420BD006DCA3F52242A2F55B
:10ACA800CF72012A0ED803E04AF20B52934209D11F
:10ACB80033782F2B60D9B1F91020303293425BDC06
:10ACC800303B30E043F6F122934207D11F4B1B780B
:10ACD80023B13078B5F900103B222CE006F0C0FB18
:10ACE80018B3236843F6C4219A688A4203D047F20E
:10ACF800CD018A4204D13078B5F900102D221AE02E
:10AD0800A2F56A516139052903D943F6E9218A4236
:10AD180001D1012307E043F6E0218A4202D00A313B
:10AD28008A4203D100232B6026E023683078B5F9E6
:10AD38000010B3F91020FFF7E9FB28601CE000BF02
:10AD48005E3300203C18002014040020C91800209D
:10AD5800820D0020E0180020E823002009190020B7
:10AD68002368B3F90800FDF7CDFD286098F8003096
:10AD780043F0080388F80030FFF7A8FB236843F680
:10AD8800D222986890420BD12B6813B99C489D49F0
:10AD980001E09B489C490222F5F7D2FD0226B0E16A
:10ADA8004AF20B5290420AD12B6813B99748984936
:10ADB80013E0012B95480CBF964997490DE04AF2DC
:10ADC800AE42904218D12B68012B02D18F4893498B
:10ADD80003E0022B05D18D4891491022F5F7B0FD0B
:10ADE8008EE1032B02D189488E49F6E7042B874868
:10ADF8000CBF8D498D49F0E74AF29E3290420AD144
:10AE08002B6813B981488A49E7E7022B7F480CBFB2
:10AE180088498949E1E74AF29F3290420AD12B6872
:10AE280013B97A488549D8E7012B40F069817748FA
:10AE38008349D2E748F63742904203D043F6EE22E0
:10AE480090420ED128680A21B0FBF1F201FB1201F1
:10AE58007C4B3031D97730322E2199775A770326B7
:10AE68004FE143F6F12290423ED1774B1B78E3B98C
:10AE7800022229687548FDF7FBFC43F6F220FDF72E
:10AE880041FD022201465E48FDF7F2FC3B7813F0D3
:10AE9800010F00F086816E4B1B7803F08003DBB254
:10AEA800002B00F07E81694819E0FDF72BFD022296
:10AEB80001466648FDF7DCFC022251482968FDF787
:10AEC800D7FC3B7813F0010F00F06B81604B1B78C7
:10AED80003F08003DBB2002B00F063814848202197
:10AEE8000222F5F757FA5CE143F69812904240F0D7
:10AEF800F5802B68574EDFF8508156F83310102232
:10AF08004248F5F71DFD0DF1060298F800000DF115
:10AF180007010EF0C3FE4246334620B316784E4969
:10AF2800895D03291FD0296803EBC1010979C1F3A1
:10AF38004111012917D1072E15D948490B22484834
:10AF4800F5F7FEFC4748711C0222FDF791FC9DF8BD
:10AF58000710454801310222FDF78AFC9DF80610CA
:10AF68004248013118E02E68157803EBC6010979CB
:10AF780003EBC6063679C1F34111012906F007062D
:10AF8800C8BF05F00705012E0ADC394934480B22F1
:10AF9800F5F7D6FC3348691C0222FDF769FCAFE0DF
:10AFA800022E0BD133490B222D48F5F7C9FC324646
:10AFB8002C48691CFDF75CFC0E36A2E0032E0BD171
:10AFC8002D490B222648F5F7BBFC2648691C0222AE
:10AFD800FDF74EFC0D3694E0042E51D127490B2283
:10AFE8001F48F5F7ADFC1F48691C0222FDF740FC1D
:10AFF8001D4805F109010222FDF73AFC0C3680E0F4
:10B0080012020020044D0208064D02080402002026
:10B0180006F9020848F9020827F90208DDF70208CC
:10B02800FEF702081FF8020840F80208BCF70208F9
:10B03800ABF90208EDF90208CCF902082FFA020868
:10B0480050FA0208F4010020C91800200F0200205D
:10B05800C031002014040020E823002094130308C2
:10B06800F9010020FA010020FE0100200102002061
:10B0780052130308AD12030831130308EF12030833
:10B08800052E11D148490B224848F5F759FC484884
:10B09800691C0222FDF7ECFB464805F10901022272
:10B0A800FDF7E6FB0B362CE0062E29D142490B2290
:10B0B8003E48F5F745FC3E48691C0222FDF7D8FBDF
:10B0C8003C4805F109010222FDF7D2FB3B4805F196
:10B0D80011010222FDF7CCFB0A3612E0B3F9106029
:10B0E800092E04DD632ECCBF0326022600E00126CC
:10B0F80033482968801B46F08002FDF7B9FB00E061
:10B1080010263B7813F0010F0BD02E4B1B7803F061
:10B118008003DBB22BB12A482021801B3246F5F789
:10B1280039F9294EB37803F00203DBB2002B38D08B
:10B13800FDF7A6FA254D034628B92878F11D6522A2
:10B14800FDF7BCFA08E0B2792978B388F01D01FB55
:10B15800023109B205F021FE236847F2CD029B684F
:10B16800934213D006DC43F6C42293420ED043F632
:10B178009A5209E047F24D12934207D048F6F2324C
:10B18800934203D047F20D1293420AD105200B21B6
:10B198000D4AFDF7FFFA29780D4801310222FDF723
:10B1A80067FBBDE8FE8F00BFCE120308F90100203F
:10B1B800FA010020FE0100201013030802020020FB
:10B1C80014020020C031002018190020C9180020DE
:10B1D800F5010020F0B5114B1F78114B303F1E6868
:10B1E8000DE0D6F814C01CF803C00133644501D142
:10B1F80012E00023DAB28242F3D301350D70094B15
:10B208000622094902FB07330D785B1993F8D440ED
:10B21800002CEED10C70F9321046F0BD0418002055
:10B228003C180020344C02084A1800202DE9F74F3A
:10B23800974C984E23689A6843F605539A4203D16F
:10B2480033780BB9013333702368934F9968B3F996
:10B2580010303A78B3F1010848BF03F106084FEA05
:10B26800E808337808F1010812F0010F03FB081809
:10B278008A4D00F0AD808A4B1A789946432A4DD101
:10B2880028780FFA88FA0AEBD00005F075FD2268D5
:10B29800844B916846F2C4629142186001D12A78C1
:10B2A8003AB12A78012102F0070211FA02F250405D
:10B2B8001860287819780AEBD00005F053FD236848
:10B2C80047F2AD129B68934209D1744B1A78764BBA
:10B2D80003EBD203734A126883F8A0211EE046F6F6
:10B2E8007532934205D13178002001310CF0EEFF20
:10B2F80014E046F28B7A4FF0000B23689B685345A5
:10B3080004D101200BEB00010CF0E0FF0AF1080A60
:10B3180046F2AB739A450BF1010BEED199F8003068
:10B32800232B10D122682B78927C013A93420ADAB7
:10B338005A4A013313705D4B9B7803F00203DBB26A
:10B348000BB1FDF76BF999F800302A2B0CD12B784B
:10B3580053B1524A013B1370544B9B7803F00203DC
:10B36800DBB20BB1FDF75AF999F80030552B14D11F
:10B378002368997C0F2910D92A7808398A42474BC3
:10B3880001DA083200E000221A70484B9B7803F07B
:10B398000203DBB20BB1FDF741F999F80030442BF9
:10B3A80042D123689A7C0F2A3ED929783B4B07293A
:10B3B80002D90839197001E0083A1A703B4B9B789A
:10B3C80003F00203DBB2002B2ED0FDF727F92BE0A8
:10B3D80048F6A93399420ED1314B1B78A3F13101BC
:10B3E800C9B2032907D842F006023A70072253432C
:10B3F800284A573B137023689A6843F605539A42C4
:10B4080012D133781B2B08D9284B46F661429A8013
:10B418009A7842F002029A7006E05901C918244B42
:10B428000020C918FDF7FEF9FFF750F8214A2B78DC
:10B4380011789346994288BF137012780F3293425D
:10B4480002DD1C4A0F3B137023684FF0000A93F883
:10B458001290B9F10F0F9ABFC9F120095FFA89F963
:10B468004FF010099BF800004FFA8AF318180FFAEA
:10B4780088F202EBE000019305F07EFC9BF80020C7
:10B48800019B5FFA80FC9B1803F007032BE000BFC9
:10B498003C180020C918002009190020D3180020E2
:10B4A80004180020E0180020E823002018190020C4
:10B4B80060FC0208CB1800204CFA03F06549013300
:10B4C80000F0010000280CBFA520DB20DBB201F84A
:10B4D80009000AF1010A09F10109082B5FFA8AFA41
:10B4E8005FFA89F903D0B9F1200FE5D109E0B9F184
:10B4F800200F06D023684FFA8AF19B7C891899425D
:10B50800B0DB3B7813F0010F15D0236852499B7CC0
:10B5180009780F2B01F0800198BFC3F11003C9B25D
:10B5280094BFDBB2002331B1297810318A1A494916
:10B53800CB185F219954DFF8288198F802304746E4
:10B5480003F00203DBB2002B64D0FDF799F8034641
:10B5580000BB226846F6753192688A4206D02431CB
:10B568008A4203D043F6E5118A4204D130783B4938
:10B578006522002309E043F605518A4208D1307854
:10B588001C38C0B208F107016522FDF797F818E0EA
:10B598002878F7E7236846F635329B68934203D04C
:10B5A80043F6F822934202D1BA79317801E0BA79A8
:10B5B8002978BB88294801FB0231BA7909B205F01C
:10B5C800ECFB23689A7C102A02D905200B211EE087
:10B5D8009B6846F6353293420ED006DC43F6E512F8
:10B5E800934209D043F6F82204E046F675329342B6
:10B5F80002D02432934201D1102007E043F60552CD
:10B60800934202D10020102101E000200721144AB2
:10B61800FDF7C0F8226846F6D93193688B4216D0F8
:10B6280046F693218B4212D043F6ED218B4202D18C
:10B63800084BDB219977937C102B08D92978094886
:10B648000131022203B0BDE8F04FFDF711B903B094
:10B65800BDE8F08FF4010020C03100201F19002040
:10B6680018190020F5010020114B002270B50D4675
:10B678001A7118B11B7803B920234370BDB10D4866
:10B68800F5F7D8F80446681C5CB10A492246F4F775
:10B69800D9FD022C0BDC601C28182021C4F1030200
:10B6A80001E020210322BDE87040F4F773BE70BDAD
:10B6B800B8180020B918002038B50546002408E05D
:10B6C800601905F059FB3038C0B2092808D8013490
:10B6D800E4B2044B1B78303B9C42F1DB012038BDBF
:10B6E800002038BD2018002008B505F045FB0023D0
:10B6F800C0B2064AD25C824201D1202804D101336B
:10B70800082BF6D1002008BD012008BD444D0208D1
:10B7180070B506460D4600240DB12D232B55A019F2
:10B728000021013405F01EFB062CF5D170BD000088
:10B738002DE9F04F974C984F206839788368068A2E
:10B748009AB201FB06260D4647F610018B4287B0D8
:10B75800B6B20BD1914B1A785B7802F00702C3F3AB
:10B76800420303EBC20306EBC3062BE047F6D011F6
:10B778008B4212D1894B8A481A78597802F007020D
:10B7880088235A43C1F34201773B03FB012320215D
:10B798000822F618F4F7FEFD14E047F688518B42AC
:10B7A8000BD17E4B1A785B7802F00702C3F3420391
:10B7B80003EBC2039B01F61804E0B3F5E97F08BF69
:10B7C80002EB4506774B784D1A78984612F0010F30
:10B7D80053D123689A6846F6D5739A4204D046F640
:10B7E800D5539A4240F04481704B1B782A2B3BD1A9
:10B7F8006F4B93F8009009F1010909F0010983F8EA
:10B808000090B9F1000F1AD046F6D5539A4208D1E4
:10B81800684B46F661429A809A7842F002029A7022
:10B8280026E1202110226448F4F7B4FD3B7800207B
:10B838005901C918614BC918FCF7F4FF18E15D48B4
:10B84800FCF796FF236848469A6846F6D5539A420D
:10B858000CBF5B495B49FCF7E5FF39785A48013171
:10B868000222FDF705F803E1552B02D0442B40F0E6
:10B87800FF804F4B00221A70FAE023685869F4F7EA
:10B88800D9FF4A4B834693F800A09946BAF1450F71
:10B8980002D14E4B00221A705046FDF77FF800285F
:10B8A8004DD04B4B5FFA8BFB1A7852450ED1584658
:10B8B800FFF790FCFF2804D15846FFF78BFCFF28C0
:10B8C8003DD0444B1A7801321A7015E0DFF804A114
:10B8D80000228AF8002058460593FFF77BFCFF28D2
:10B8E800059B04D09AF8002001328AF8002099F8C4
:10B8F8000020FF281A7022D02168374A4B6910604F
:10B908001B5C886846F6D5718842136092460FD151
:10B91800562B01D0542B0BD13B78123BDBB2022BB8
:10B9280006D82B7830B2C01805F026FACAF80000FD
:10B938002B7830B2C018DAF8001005F013FA99F82D
:10B948000030552B17D12368997C0F2913D92A78F1
:10B9580008398A42144B01DA083200E000221A70D2
:10B96800144B9B7803F00203DBB20BB1FCF756FED5
:10B97800184B00221A7099F80030442B3BD12368E9
:10B988009A7C0F2A37D92978074B072926D90839ED
:10B99800197025E03C180020C9180020CE18002096
:10B9A8000402002009190020D318002004180020E0
:10B9B8001419002018190020F401002083F402084B
:10B9C80094F20208D6F20208F50100201C180020A3
:10B9D8001E1800204A180020E0180020083A1A70A3
:10B9E800964B9B7803F00203DBB20BB1FCF716FE13
:10B9F800934B00221A7099F80030432B0CD123681E
:10BA080030B25B6919788F4B19602B78C01805F034
:10BA1800A9F98B4B00221A7099F80030232B13D107
:10BA280022682B78927C013A93420DDA864A0133D8
:10BA38001370834B00221A70804B9B7803F002032B
:10BA4800DBB20BB1FCF7EAFD99F800302A2B0FD1D5
:10BA58002B786BB17C4A013B1370794B00221A702A
:10BA6800764B9B7803F00203DBB20BB1FCF7D6FDF3
:10BA7800FEF72CFD754A2B7811789246994288BFBB
:10BA8800137012780F32934202DD704A0F3B137025
:10BA980023684FF0000B93F81290B9F10F0F9ABF7B
:10BAA800C9F120095FFA89F94FF010099AF80000E6
:10BAB80033B218185844059305F05EF9644A02F841
:10BAC800090009F101095FFA89F9B9F11F0F059B0E
:10BAD80005D821680BF1010B897C8B45E6DB98F8CA
:10BAE800001011F0010F16D021685A48897C00789F
:10BAF8000F2900F0800098BFC1F11001C0B294BFB7
:10BB0800C9B2002138B128789AF80060103052186C
:10BB1800801B5F2111542268906849F23E6290426E
:10BB28000AD14D4B1B78532B2FD105F025F94B4BE0
:10BB3800187005F01BFA28E0B0F5E97F25D1464AD0
:10BB48001278532A21D11846FFF7CEFD0646E0B9F0
:10BB58003B78DA00D31A03F11200FFF7ADFD60B1AC
:10BB6800FF2300933E4B01961B7879200133029303
:10BB780031460422334605F07DF93B780021DA008E
:10BB8800D31A03F11200FFF7C3FD2C4EB37803F06C
:10BB98000203DBB2002B6ED0FCF772FD034680B9BE
:10BBA800226847F6885192688A420AD046F6D551EB
:10BBB8008A4214BF28783878F11D6522FCF77EFD8B
:10BBC8000FE02368B2799B682648B3F5E97F0CBF7C
:10BBD80039782978B38801FB0231B27909B205F0C6
:10BBE800DCF823689A7C032A08D99A6847F610017A
:10BBF8008A4203D046F6D5518A4214D19B6847F64B
:10BC0800100293420CD198F8003013F0010F01D0C4
:10BC180010202CE0202107221348F4F7BBFB2AE070
:10BC2800B3F5E97F02D105200B2121E046F6D55274
:10BC380093421BD1002010211AE000BF18190020E0
:10BC48004A180020E0180020D3180020CB18002044
:10BC5800F4010020C0310020041800202018002022
:10BC6800C91800201F190020040200200020072105
:10BC7800104AFCF78FFD23689A7C032A16D9B278FC
:10BC880002F00202D2B28AB19B6847F610029342D0
:10BC98000CD046F6D552934208D02978064801318F
:10BCA800022207B0BDE8F04FFCF7E2BD07B0BDE8DF
:10BCB800F08F00BF18190020F50100202DE9F04F82
:10BCC8007A4E8BB033689D6893F81290122D01D08C
:10BCD8000B2D09D1764A122D92F80090A9F130095E
:10BCE8005FFA89F915D01DE04AF2BB439D4203D0A3
:10BCF80028339D4240F055836E482821F4F7C8FB4D
:10BD08008046002800F0508301302821F4F7C0FB5A
:10BD18004AE39F7B37B9684BB846D879FEF7E0FB12
:10BD2800044615E00027B846FF20FEF7D9FB4AF283
:10BD3800AC239D4204460BD14AF28B3005F01CF827
:10BD4800C0B2089020B15C4B9B790BB1FCF72EFE7A
:10BD580033685A4D9A68122A1AD19B7BC3B12B7843
:10BD680013F0010F08D12046FFF7A6FC544B10B181
:10BD780001221A7000E018704F4B9B7943B120469E
:10BD8800FFF79AFC20B14E4B1B780BB1FCF70EFE67
:10BD98002978DFF848A111F0010100F089819AF8AB
:10BDA8000030DFF83CB118460793FCF7F7FD079B16
:10BDB800002800F0B7804349002008704248434AF1
:10BDC80090F800C013609C45414940F08B8033686F
:10BDD8009B8903F00F03032B21D1ACF1300C0A200F
:10BDE80000FB0CF03B4BDFF8F0C093F800E0059047
:10BDF800704409900EF1010E1CF80000DDF814C023
:10BE08005FFA8EFE106083F800E00CEB0E00DFF89E
:10BE1800C8E01EF80000002871D118706FE0082BE8
:10BE28002BD12C48ACF1300C03780CEB8C0E099319
:10BE3800294B9E44099B734493F86CE00993264B65
:10BE4800BEF1000F01D180F800E090F800E00CEBA3
:10BE58008C0C634403EB0E0C0EF1010E5FFA8EFEA0
:10BE680073449CF86CC093F86C30C2F800C080F83A
:10BE780000E0002B43D1174811E0072B11D1BCF18A
:10BE8800300F10D11348037823B14FF02B0EC2F8AE
:10BE980000E001E0C2F800C0013303F001030370C1
:10BEA8002DE0062B2BD10B78013327E03C1800201E
:10BEB8002018002004020020D618002009190020AC
:10BEC800670E00205F3A00201E180020E0180020AE
:10BED800D31800204A180020344C02080418002007
:10BEE80021180020DFF898E203709BF800304FF02B
:10BEF800010C8EF800C013B10B7863440B7040231B
:10BF08008BF800300B784B4503D39B4B09F1FF307E
:10BF1800187008781168201804F024FF2B7843F073
:10BF280004032B709AF80030232B2FD1924B09F180
:10BF3800FF311A788A4229DA72B932684AF2BB416B
:10BF480092688A4208D028318A4205D02046079351
:10BF580004F012FF079BC8B118780130C0B21870FE
:10BF6800201804F009FF28B9834B202118782018DD
:10BF780004F0F8FE814B40221A702B78804A43F077
:10BF880004032B7000238BF8003013709AF80030EC
:10BF98002A2B10D1784B1A786AB1013A1A70774B6C
:10BFA80040221A702B78764A43F004032B70002342
:10BFB8008BF8003013709AF80030432B1FD16E4B6A
:10BFC8001878484505D220182021079304F0CAFEA6
:10BFD800079B9BF800203AB91B7809F1FF3293427E
:10BFE80002DA654A013313702B78644A43F004037C
:10BFF8002B7000231370624A8BF8003013709BF883
:10C00800003013B15F4A013B13709BF80030012BDD
:10C018000ED1594B1A784A4501D201321A70584A42
:10C02800002313702A7842F004022A708BF800303B
:10C038002B7803F00402D2B2002A71D0524A6FF36F
:10C0480082031370002111225048F4F7A3F9504AD3
:10C05800494B11781B78994288BF137011780F31BA
:10C068008B4202DD4A490F3B0B701178474810227A
:10C07800611804F092FE4548F4F7DCFB33684AF295
:10C08800BB419B68C2B28B4202D028318B4205D19A
:10C0980022B94048F4F7CEFB421CD2B20F2A3FD84F
:10C0A8003A4820218018C2F11002F4F773F937E0FA
:10C0B800DFF8D8B011225846F4F76CF933684AF221
:10C0C800BB429B68934202D02832934209D1214651
:10C0D80004222E4804F061FE40463946FFF7C4FAB0
:10C0E8001EE021461022584604F057FE5846F4F741
:10C0F800A1FB02462021C2F110025844F4F74AF984
:10C1080021464A46244804F048FE244A10209378E1
:10C1180082F8069043F0020393700146FCF73AFB5D
:10C128009AF80030532B75D133689A684AF2AC23D9
:10C138009A4208D1204604F01FFE20B14AF28B3003
:10C14800012104F00FFE3368DFF838A09B68122B3A
:10C1580040D12046FFF7B0FA8346002830D0104B74
:10C16800FF2219780F4BF9B9009201911B787820BA
:10C1780001330293FB3A1FE0D31800205F3A0020F6
:10C188004A1800202118002009190020B81800209A
:10C19800CB180020B9180020531800204C18002094
:10C1A800670E0020C91800200021009201911B7819
:10C1B8007A200133029304220B4604F05BFE09E067
:10C1C8008AF800007D492046FFF7A2FA7C4B83F8E5
:10C1D80000B0EFE020464946FCF732FB794B0020DF
:10C1E800187033688AF800009B6849F252629342DB
:10C1F80002D10090013005E04AF2CE22934206D1E6
:10C20800012300930146024603460CF08BF86E4862
:10C21800FCF7AEFAFEF75AF92B7813F0010F17D096
:10C2280033684AF2BB429B68934202D02832934259
:10C2380004D140463946FFF717FA09E05F4B634AD5
:10C2480003F1100153F8040B8B4242F8040BF9D1A7
:10C2580033689A68122A1ED19B7BE3B12046FFF708
:10C268002BFAC0B12B7813F0010F14D1584B9A79DF
:10C2780022B9DA79574B1B789A420CD0564B1A7868
:10C288000023303A05E055492A20C91801330874BB
:10C29800DBB29342F7DB326893680B2B01D0122B89
:10C2A8000AD14A4B991D13F8010B202802D10D30F1
:10C2B80003F8010C8B42F6D192684AF2AC239A42F9
:10C2C80014D1434B9B798BB1089878B14FF0000992
:10C2D80009EB040004F050FD18B1404B2A224B44EE
:10C2E8001A7409F10109B9F1100FF1D12B7813F083
:10C2F800010F25D03A4B1B7803F08003DBB2FBB16A
:10C3080033689A684AF2BB439A422D4B03D04AF2EB
:10C31800E3418A420CD11B7833B9B8F1000F0FD032
:10C328005F3388F801300BE057B15F22FA5407E019
:10C33800244A1B78127810339B1A284A5F21D1545B
:10C34800284CA37803F00203DBB2002B32D0FCF7B1
:10C3580097F92049034628B908786522E11DFCF7BA
:10C36800ADF912E03068B4F90430A279846809782C
:10C37800122C01FB023105D1807B18B91449C97907
:10C3880002FB0131184804F008FD33689B68122B42
:10C3980010D10820134A01460BB0BDE8F04FFCF756
:10C3A800F9B90027B84600E0074609F1FF395FFAF6
:10C3B80089F9B9E40BB0BDE8F08F00BFB8180020C8
:10C3C800D3180020CB1800204C18002004020020AD
:10C3D800D6180020C918002020180020F4010020D9
:10C3E800C0310020181900201F19002024282DE929
:10C3F800F041144626D16B4B43F638321B686A4D20
:10C408009B686A4E934206D12B7813F0010F0ED029
:10C418002438674909E04AF2E34293420AD12B786B
:10C4280013F0010F03D063490020FCF7FBF92978CA
:10C43800490800E02978301901310222FCF718FA7E
:10C448000234AAE0E72809D1574B584819788018D0
:10C4580001310322FCF70CFA03349EE0A3282AD109
:10C46800514D2B783F2B15D810465349FCF7DAF974
:10C478005148F4F7DFF92A2124184C48E4B2F4F7BC
:10C4880007F8002800F08A80297802220131FCF799
:10C49800EFF983E05901494DC918691801F582413E
:10C4A8001046DF31FCF7BEF905F59240FE30F4F78F
:10C4B800C1F9241871E0F22821D13B4F3B4D39785E
:10C4C800072605EB0208B1FBF6F1404601310222CE
:10C4D800FCF7CEF939782D23B1FBF6F688F802304F
:10C4E800F3009E1B8B1B364FDBB207EB83031988C7
:10C4F800E21CA9529B78A818837006344DE02528C1
:10C508000BD1304B46F661429A8045229A719A784F
:10C51800053842F002029A703CE05E280BD1294BA4
:10C5280046F661529A8045229A719A783E3842F0CE
:10C5380002029A702EE07C280BD1224B46F244125C
:10C548009A8011229A719A785C3842F002029A70A5
:10C5580020E0EC280BD11B4B46F6A5529A804522C9
:10C568009A719A78CC3842F002029A7012E0A728A1
:10C578000BD1144B46F6C5529A8045229A719A7887
:10C58800873842F002029A7004E0E02801D1541C76
:10C5980003E018B1054B18550134E4B22046BDE854
:10C5A800F08100BF3C180020C9180020F4010020C9
:10C5B800E8EC0208A6EC020862F4020864AA020881
:10C5C800DDD602081819002038B50A4B46F68A4508
:10C5D8001B78002405FB030507E0074B2246197862
:10C5E800FFF704FF041B2D190446287808B11F2CF7
:10C5F800F3D938BD1F180020C918002070B50025D0
:10C6080043F61C64204604F0B7FB064604F1080014
:10C6180004F0B2FB16F0FF0F06D020F07F0010F0F8
:10C62800FF0F01D00135ADB246F23B139C4201D059
:10C638000934E7E7284670BD38B5B0F900500B4C0F
:10C6480005EBC50505F578552435284604F094FB17
:10C65800C1B211F0800F07D023882846013B01F0B2
:10C668007F01238004F07EFB208838BD1A18002043
:10C67800454B2DE9F74F1B88444A044689461788DD
:10C68800DFF80C8123B14FF0000A0AE09A4608E06F
:10C698000529FBD198F8003043F0040388F80030EE
:10C6A80070E098F8003013F0030F0BD013F0010F6F
:10C6B80002D0B4F1FF3F05D103F00203DBB21BB196
:10C6C800012C01D03F19BFB23BB2B3F1FF3F04D0F8
:10C6D800B3F57A7F08BF002701E040F2E7370FFA89
:10C6E80087FB0BEBCB0303F5785303F11C00019395
:10C6F80004F042FB10F0FF0F019B16D0B9F1050FB3
:10C7080009D103F1240004F037FB20F07F0010F07A
:10C71800FF0FC6D022E0B9F1000F1FD003F12400AB
:10C7280004F02AFB00F07F0618E00AF1010AB4F1D0
:10C73800FF3F1FFA8AFA04D198F8003043F001034A
:10C7480005E0012C05D198F8003043F0020388F881
:10C758000030BAF57A7F0DD03D46A2E74E4505D0A8
:10C76800B9F1000F02D0B9F1050F9AD1BAF1000F53
:10C7780005D000E03D46054A2DB2156002E0034BA6
:10C78800C3F800B0BDE8FE8F1A180020E01800209A
:10C79800E4180020F0B503789BB05A1ED2B2792A6B
:10C7A8000F4600F2C8805E01644AF3189B18644A79
:10C7B80046F68A461278457806FB0236E721304667
:10C7C800F3F766FE0446F0B930467C21F3F760FEC5
:10C7D8000446C0B930462521F3F75AFE044690B9FD
:10C7E80030462421F3F754FE044660B93046402110
:10C7F800F3F74EFE044630B93046F921F3F748FE08
:10C808000446002876D0A41B0FB14E4800E04E48DD
:10C8180031462246A619F4F793F83046E721F3F794
:10C8280037FE30B128466946652246F6A553FBF720
:10C8380045FF30467C21F3F72BFE50B1691EC9B283
:10C8480001EB011101F5C24168464431112204F09F
:10C85800A4FA30462521F3F71BFE38B1681EC0B292
:10C868006946652246F66143FBF728FF3046F92101
:10C87800F3F70EFE38B1681EC0B26946652246F667
:10C888006153FBF71BFF30464021F3F701FE50B11F
:10C89800691EC9B201EB011101F5E2416846DF31B9
:10C8A800112204F07AFA30462421F3F7F1FD50B151
:10C8B8000FB1244800E02448001929460222FBF75A
:10C8C800D7FF02340BE00FB11E4800E01E480019E4
:10C8D8006946F3F751FF6846F3F7ACFF0419002FD8
:10C8E80029D01A4A9378141943F00203937000234D
:10C8F800E37116E03046F3F79DFF05461FB912486D
:10C9080031462A4615E0102810DD2A460D483146E2
:10C91800F4F716F80D4A9378551943F0020393700B
:10C92800EC7110200146FBF735FF04E0084831465A
:10C938001022F4F705F81BB0F0BD00BF47DC020871
:10C948001F1800201F190020362A0020181900205F
:10C95800040200200C4B1B7813F0010202D00020C7
:10C968000A4905E003F00200C0B218B108491046B0
:10C97800FBF758BF03F00403DBB20BB10549F7E737
:10C9880005480121FFF706BFE418002020B202087D
:10C99800FFB1020841B202080B19002070B5124D10
:10C9A800124C00201249FBF74DFE2846A1780222BE
:10C9B800FBF75EFFE81CE1780222FBF759FF05F15F
:10C9C800080021790222FBF753FF05F10B0061797A
:10C9D8000222FBF74DFFA17905F10E000222BDE806
:10C9E8007040FBF745BF00BFF40100200B19002081
:10C9F8004D4D02082DE9F341504F514C3B689D7C49
:10CA0800237813F0010F2FD1022243F61A610DF19A
:10CA1800060004F0C2F94B4EBDF806304FF0FF3067
:10CA280033602946FFF724FE237843F0010323707F
:10CA3800454B1B7813F0030F14D1B6F90010434887
:10CA480001EBC10101F578511C31092204F0A5F967
:10CA58003F4B1B881BB13046FFF7EEFD10B9002095
:10CA6800F9F7D8FAFFF79AFF3A4E3378552B0DD1DC
:10CA7800DFF8D4803848FBF77BFE98F800304FF099
:10CA8800FF306FF3410388F800300DE0442B2BD1C1
:10CA9800DFF8B4803048FBF76BFE98F800300120CF
:10CAA8006FF3000388F800302946FFF7E1FD98F896
:10CAB800003013F0030F15D1224D2448B5F90010AA
:10CAC800092201EBC10101F578511C3104F065F927
:10CAD8001F4B1B881BB12846FFF7AEFD10B900207D
:10CAE800F9F798FAFFF75AFFFFF734FF3378232B4B
:10CAF80022D1154B184E1A7802F0FC026FF382020D
:10CB08001A70FBF753FFB3786FF34103B370134BFD
:10CB18001D7835B9FBF782FD3046FBF729FE3D60ED
:10CB28000AE02278013DEDB242F0060222701D7043
:10CB38000B4B53F825303B60BDE8FC813C180020C6
:10CB480009190020E0180020E41800200B19002023
:10CB58001A1800200418002018190020F7180020BF
:10CB6800F81800202DE9F0411646104A0F46537870
:10CB78000E21C3F342034B43117803F5EE43A03370
:10CB88000B4D01F00701044603EB4101022204F0BA
:10CB980004F9E81921780222FBF76AFE6178A819DE
:10CBA8000222BDE8F041FBF763BE00BFCE180020AB
:10CBB800F4010020044B02225978044BC1F34201CE
:10CBC80018180131FBF754BECE180020F4010020DC
:10CBD80010B5074B074C1B78074A03F0070304EB13
:10CBE80083031C88111814529B788B7010BD00BFEA
:10CBF800CE180020DDD60208F4010020084B1B786F
:10CC08009B0902D0012B06D102E01020054904E05F
:10CC18001020054901E005491020FBF703BE00BFBD
:10CC2800CE180020C2BE0208E3BE020804BF0208F4
:10CC38002DE9F041DFF868800F4698F80010174D8D
:10CC4800C1F382010446164605F1080001310222AB
:10CC5800FBF70EFE98F80010042201F01C0101F504
:10CC68000A41204601F5C47104F097F8E8192178C3
:10CC78000222FBF7FDFDF81C281861780222FBF759
:10CC8800F7FDA819A1780222FBF7F2FDF01CE17864
:10CC980028180222BDE8F041FBF7EABDF4010020A4
:10CCA8001D180020064B1B7803F08003DBB233B15C
:10CCB800435C04482021C0180222F3F76BBB70477D
:10CCC800C0310020F40100202DE9F743654D664C82
:10CCD8002B6821789B68022203EB41010DF10600C5
:10CCE80004F05BF82B68A9469A6843F6F4239A4245
:10CCF80008D100205D49FBF795FDBDF806804FF48B
:10CD0800B46303E0BDF806804FF46163B8FBF3F148
:10CD180003FB11883C221FFA88F8B8FBF2F302FBE8
:10CD28001388CFB2DEB2022251483946FBF7A0FD84
:10CD38005FFA88F802224F483146FBF799FD022234
:10CD48004D484146FBF794FD4C4B1B7813F0010FFF
:10CD58006ED04B4B4B4D1878232804D12B78012BE0
:10CD680062D8013305E02A2805D12B78002B5BD047
:10CD7800013B2B7058E0A0F13003DBB2092B01D93D
:10CD880043284BD12B7873B9D9F8003039B29A6857
:10CD980043F6F4239A4201D10A2200E01122FDF75A
:10CDA800B5FBC7B216E0012B0ED1D9F8003031B26D
:10CDB8009A6843F6F4239A4201D1172200E03B22F5
:10CDC800FDF7A4FBC6B205E041463B22FDF79EFBFA
:10CDD8005FFA80F8D9F800309A6843F6F4239A424B
:10CDE80009D13C235E434FF4B46303FB0767B8449F
:10CDF800ADF8068006E03846314642460EF08FFA16
:10CE0800ADF80600D9F8003020789B680DF10601CE
:10CE180003EB4000022203F0BAFF05E0532803D1D8
:10CE280000232B70FDF752FB17482978FFF73AFFCC
:10CE3800D9F800309A6843F6F4239A4210D0207843
:10CE4800124965220023FBF739FC05200B21104A03
:10CE5800FBF7A0FC21780F4801310222FBF708FDFF
:10CE6800BDE8FE833C180020C9180020E7F002083E
:10CE7800040200200A0200201202002009190020E2
:10CE880004180020D31800205E4D02081F19002046
:10CE980018190020F501002073B59A4B9A4D1A789D
:10CEA80012F0010F05D12A7812F0380204BF2A7057
:10CEB8006A701A78934E42F001021A702B78924CDD
:10CEC80013F038023ED191490978552904D113F05D
:10CED800070F2FD0DA1D0AE044290CD103F007020E
:10CEE80001323D3992FBF1F1C800411A521A62F33E
:10CEF800020323701EE053290AD1C3F3C201013192
:10CF080061F3C5032370637862F34303637011E030
:10CF180023290FD1FBF74AFD33787D4A43F00603F6
:10CF280033701378013BDBB213707A4A52F823202E
:10CF3800794B1A6000207949FBF774FC1C20FFF735
:10CF480047FEDDE0082A2ED175490020FBF76AFC70
:10CF58000620FFF72FFE0C20FFF73AFE15211822B6
:10CF680001A8FFF7FFFD694B1B78552B06D16378A5
:10CF780003F0FE03C3F34202013A07E0442B0BD14E
:10CF8800637803F0FE03C3F34202013202F00302A6
:10CF980062F343036370B3E0532B28D0232B40F094
:10CFA800AF802378A6E0102A51D15D490020FBF715
:10CFB80039FC0620FFF7FEFD0C20FFF709FE1521BE
:10CFC800182201A8FFF7CEFD6178564801F001014B
:10CFD800FFF768FE4D4B1878232801D02A2804D182
:10CFE8006378DA4362F30003D4E7532804D1237843
:10CFF800C3F3C202013280E0A0F13003DBB2092B97
:10D0080001D943287CD16B7802AA03F001033B21A4
:10D01800D41883F001024B43172606FB023214F89A
:10D02800041CFDF773FA04F8040C6B780E22C3F3A2
:10D0380042035343287803F5EE43A03300F007007A
:10D0480003EB400001A90C3A03F0A1FE58E0182AAE
:10D058004DD133490020FBF7E5FB0620FFF7AAFD79
:10D068000C20FFF7B5FDFFF7C9FD284B1B78552BA2
:10D0780007D1237813F0C00F42D0C3F38112013ACD
:10D0880006E0442B07D123789A09012A38DC0132BB
:10D0980062F3871333E0232B04D12378C3F3C2024E
:10D0A800023A2AE0532B2BD1FBF780FC33781E4A37
:10D0B80043F006033370164B1648197840F82120C0
:10D0C800013119702378C3F3C201013161F3C5033B
:10D0D800C3F381112370104B11B1012904D101E070
:10D0E8001C3202E0114A00E0114A1A6008E0114AB5
:10D0F80000211170C3F3C202013A62F3C503237021
:10D108007CBD00BF09190020CE180020041800209B
:10D11800F7180020F81800203C18002080BE0208EC
:10D12800A1BE0208614D0208644D02089C4D020828
:10D13800B84D0208D318002073B5494B494D1A78E9
:10D1480012F0010F04D12A7812F0030208BF2A70E6
:10D158001A78434E42F001021A702B78414C13F0B2
:10D1680003022ED1404A1278552A03D1C3F3820212
:10D17800013A04E0442A06D1C3F38202013262F381
:10D188008403237017E0532A03D15A1C62F3010366
:10D19800F7E7232A0FD1FBF709FC3378334A43F02A
:10D1A800060333701378013BDBB21370304A52F830
:10D1B8002320304B1A6001A810211B22FFF738FDED
:10D1C8004DE0012A4BD101A810211A32FFF730FD9A
:10D1D800254B1878232804D12378C3F34112013250
:10D1E80005E02A2807D12378C3F34112013A62F3F4
:10D1F800461323702DE0532804D12378DA1C62F3F8
:10D208000103F6E7A0F13003DBB2092B01D943286B
:10D218001FD12B7802AAC3F34113D4180C215A1C2E
:10D2280003F001034B4302F001021F2614F8041C0B
:10D2380006FB0232FDF76AF904F8040C287801A904
:10D2480000F01C0000F50A4000F5C470042203F049
:10D258009EFD29780848C1F34111FFF723FD7CBDE5
:10D26800091900201D18002004180020F7180020B4
:10D27800F81800203C180020D44D0208064B1B78F3
:10D2880003F08003DBB233B1435C04482021C018AB
:10D298000322F3F77FB87047C0310020F401002063
:10D2A8004328F8B504460D46174606D1104B00260C
:10D2B8001A786FF3C3021A7000E00E462046FBF797
:10D2C8006DFB90B10A4B303C1A780A2602F008012F
:10D2D800C9B2002918BF002506FB05466FF3C30233
:10D2E80036B21A70BE42A8BF3E4630B2F8BD00BF83
:10D2F800091900202DE9F3416E4F6F4E3B7843F03A
:10D3080001033B70347844B94AF2033003F034FD2A
:10D318006A4B6B491860204617E0012C02D10020A7
:10D32800684912E0022C02D1002067490DE0032C65
:10D3380002D10020654908E0042C02D1002064498C
:10D3480003E0052C03D163490020FBF76BFA317821
:10D35800D9B9614B1B78312B01D1013101E0302B58
:10D3680005D1564B4AF20330196003F0FBFC5B4BC6
:10D378001A785B4B02F08002D2B20AB1202202E096
:10D388004E4A12683032DA776EE001290BD0022952
:10D398000CD003290DD004290ED04AF2FF25052907
:10D3A80018BF00250AE04AF2EF2507E04AF2F32504
:10D3B80004E04AF2F72501E04AF2FB252946042257
:10D3C80001A803F0EAFC474B474A03F1100153F860
:10D3D800040B8B4242F8040BF9D1032243489DF811
:10D3E8000410FBF745FA032241489DF80510FBF7A6
:10D3F8003FFA03223F489DF80610FBF739FA3E48EA
:10D4080003229DF80710FBF733FA334B3B4C18788F
:10D41800232804D12378022B22D8013304E02A28B8
:10D4280004D12378E3B1013B237019E0A0F1300364
:10D43800DBB2092B01D9432812D194F8008002AA43
:10D44800904418F8041CFF22FFF72AFF08F8040C80
:10D45800207802AA131813F8041C281803F082FC79
:10D4680027482178FFF70AFF1B4B1B78532B1FD146
:10D47800224B00221A7033780133DBB2062B33704B
:10D4880004D0012B14D10D4B1B688BB1FDF71EF88E
:10D49800002333703B781B4A43F006033B70137834
:10D4A800013BDBB21370184A52F82320174B1A605D
:10D4B800BDE8FC8109190020C9180020E0180020E7
:10D4C8006D0A0308960B0308B70B0308D80B03086B
:10D4D800F90B03081A0C030804180020C0310020B7
:10D4E800F4010020DC3203080402002005020020B9
:10D4F800090200200D02002011020020D31800208C
:10D50800D84D0208F7180020F81800203C18002011
:10D5180070B5174C0D460646002120464FF4C172DF
:10D52800F2F738FFFF2D0AD1B10001F5D8412046A6
:10D538006131042203F031FC23789BB970BDFE2DC4
:10D5480001D1173E02E0FD2D02D10136267009E017
:10D55800B60006F5D8406130401903F00DFCC0B2A2
:10D56800207020B10248BDE8704015F019BE70BDAA
:10D578002C1B00202DE9F04115F044FE60B110206D
:10D588008F49FBF74FF98F4B1B78432B40F0EE8107
:10D59800BDE8F04115F058BE15F046FE002826D02B
:10D5A800894C23786BB110208849FBF73BF98848F0
:10D5B8002D211030F2F76CFF002800F0D781217878
:10D5C80010E010208349FBF72DF981482D211030F8
:10D5D800F2F75EFF0446002800F0C88115F03CFE13
:10D5E800014620468222BDE8F041FBF741B97A4C5A
:10D5F80043F6CC2223689B68934250D0774E744DF3
:10D60800307803EB800003F0B7FB0322014674482F
:10D61800FBF72EF92368986846F6C55398422BD035
:10D62800203B984228D03378013000EB830003F088
:10D63800A3FB0322014605F11500FBF719F923683E
:10D6480030789B68023303EB800003F095FB0322DC
:10D65800014605F11900FBF70BF9236830789B6840
:10D66800033303EB800003F087FB0322014605F137
:10D678001D00FBF7FDF80EE02D2103225948F2F7B3
:10D6880089FE2D2103225848F2F784FE57482D21A0
:10D698000322F2F77FFE20232B772B762B75544B32
:10D6A8001B7813F0010F00F0BD80236843F6CC22ED
:10D6B8009B68444D934261D04E4E484F327838783B
:10D6C800D31803EB800003F057FB4B4B014618605F
:10D6D80028789846A0F13002D2B2092A01D9432805
:10D6E8000FD109B2BA22FCF711FF236832789B6880
:10D6F8000146C8F800003878D31803EB800003F01F
:10D7080031FB2B782A2B04D1337813B1394A013BEA
:10D7180013702B78232B0ED13378022B0BD8226869
:10D7280046F6A55192688A4205D020318A4202D035
:10D73800304A013313702B78552B01D0442B0FD16D
:10D74800236831789B68A3F5D843B3F1610248BFD9
:10D75800A3F15E023B7803EBA202D0B2FFF7D8FE3A
:10D76800264B1B7803F08003DBB23BB13278184BB1
:10D7780003EB820320225A749A74DA742B78532BA1
:10D7880006D023689A6843F6CC239A4240F0EE808C
:10D79800FBF70CF9236846F661429B68934203D174
:10D7A8000E4B0220197806E046F6C552934227D15F
:10D7B8000A4B002019780131BDE8F0410AF086BD16
:10D7C8009CF3020804180020D810002073F2020805
:10D7D800F4010020BDF302083C180020C9180020FD
:10D7E80005020020090200200D020020110200207D
:10D7F80009190020D3180020E0180020C0310020AB
:10D8080046F6A552934204D1594B012019780918BC
:10D81800D2E746F66152934240F0A880544B032069
:10D828001978C8E7236849F252629B6893423ED14F
:10D838004F4E10204F49FAF7F5FF31784E4D01EB66
:10D84800011101F5164152311022284603F0A5FABC
:10D858002B4605F110012A461078474F78B94749F9
:10D86800FAF7E0FF3846E721F2F712FE78B131788F
:10D87800401B381801310322FAF7FAFF07E013F8C2
:10D88800010B10B9203003F8010C8B42E4D13C4D58
:10D898002B782A2B03D13078FD21FFF739FE2B781E
:10D8A800432B63D1307823680130C0B259E043F686
:10D8B800CC229342324E1AD010203249FAF7B2FFE6
:10D8C80033782A2B52D1304B1B689B68A3F5D84379
:10D8D800B3F1610248BFA3F15E02254BFF211B781B
:10D8E80003EBA202D0B2BDE8F041FFF711BE3378D6
:10D8F8001F4D552B04D12B78142B01D1033B2B70D2
:10D908003378442B05D12B78122B02D1184B1522D2
:10D918001A702B78DFF874805901C918414401F551
:10D92800944100201F31FAF77DFF08F5924110203D
:10D9380017312F78FAF776FF3378112F8CBF03272A
:10D9480000272A2B05D12878FE21C01BC0B2FFF77B
:10D95800DFFD3378432B09D12B78173BDF1B236876
:10D96800F8B2997CBDE8F04115F034BCBDE8F0810F
:10D97800C91800207BF30208F40100208BD40208A8
:10D988000418002039F302083C18002064AA020891
:10D9980010B50E4B1B78452B17D10D4B1A7842F05A
:10D9A80006021A700B4A1378032B0ED80A490B4C3F
:10D9B800086844F823000133137083680B60FAF792
:10D9C80039FEBDE81040FAF7F1BF10BD0418002079
:10D9D80009190020F71800203C180020F81800202A
:10D9E80010B50C4B04462146D8790DF05CFC60B1AB
:10D9F800204655210DF0B6FA48B120460DF048FBF7
:10DA0800D0F1010038BF002010BD022010BD022057
:10DA180010BD00BFD618002008B50DF033FCC0B209
:10DA280008BD00002DE9F047634B644C1A7899460D
:10DA380012F0010F624D65D02078FFF7D1FF614ADF
:10DA48002B181178604F93F8A831604E442938702C
:10DA5800336090460AD12D2B08D038B995F8A91112
:10DA680001233B7031602078FFF7D6FF98F800302B
:10DA7800552B10D133682D2B0DD03B785BB1013B72
:10DA8800514ADBB21370EB1893F8A8114F4B20786A
:10DA98001960FFF7C1FF98F80030232B19D14C4BC0
:10DAA80020781B689B7C013B984212DA434B01307B
:10DAB800C0B21870FFF794FF3870281890F8A83192
:10DAC8003360444B9B7803F00203DBB20BB1FAF7E7
:10DAD800A5FD98F800302A2B14D1207890B1374B47
:10DAE8000138C0B21870FFF77BFF3870281890F81B
:10DAF800A8313360374B9B7803F00203DBB20BB1DC
:10DB0800FAF78CFD344EFCF7E1FC237832789A4220
:10DB180088BF337032780F32934202DD2E4A0F3BB2
:10DB28001370DFF8C480002730783818C0B2FFF7C8
:10DB380057FF281890F8A8310137102F08F8013F2F
:10DB480007D0254B1A78224BBA181B689B7C9A423F
:10DB5800EADB99F8003013F0010F13D01F4B1A7845
:10DB68001F4B02F08002D2B22AB1227831781032EB
:10DB7800521A5F2105E0227831781032521A13497F
:10DB880009689954134DAB7803F00203DBB25BB11B
:10DB98002078E91D652246F66153FAF78FFD0520C6
:10DBA8000B212A46FAF7F6FD21780E4801310222A8
:10DBB800BDE8F047FAF75CBE09190020D318002029
:10DBC800344C0208041800201C180020E01800201B
:10DBD8003C18002018190020CB180020C031002064
:10DBE800F4010020F50100200302002038B50546A5
:10DBF80000240123A3402A78E0B29A4205D10E49B5
:10DC0800102246F6A553FAF759FD0134042CF0D139
:10DC1800043C0A4BE0B2E3189A782B78934206D179
:10DC28002BB10549102246F6C553FAF747FD0134D2
:10DC3800042CEED138BD00BF06180020D6180020ED
:10DC48002DE9F041074610460D461446F2F7F2FD5D
:10DC5800C3B28046B3B1AB4214D80B4E20212A463A
:10DC6800F019F2F797FB2046F2F7E4FDC8EB05053B
:10DC78006D08EDB2EF1902462146F019BDE8F041F2
:10DC8800F2F7E0BABDE8F081F4010020F0B5154BD9
:10DC98000C781A1895781F46FDB100233A18927827
:10DCA8001A4112F0010F4FF001020DD0AC420E786C
:10DCB80003D09A4042EA060604E09A40C2F10F02F5
:10DCC80002EA06060E7005E09A400E78C2F10F02CD
:10DCD80032400A700133042BE0D10B7803B90C7081
:10DCE800F0BD00BFD6180020312200230178194169
:10DCF80011F0010F02D00449C9188A7501330132A5
:10DD0800042BD2B2F2D17047F401002070B57D4BDC
:10DD1800044631B11B78532B40F0F280533B03701B
:10DD280070BD1A78302A35D1774A53785BB1774B72
:10DD380077491B78172000FB03135B7913F0100F4A
:10DD480001D001235370734B20781978014013D008
:10DD58009278002A40F0D4801978114111F0010F0F
:10DD680006D0012191402078C1F10F0101402170B6
:10DD78000132042AF0D143E01A780A4112F0010F67
:10DD880004D001228A4020780243227001310429FC
:10DD9800F2D135E0A2F13101C9B203293AD85A4982
:10DDA8004A785AB1594A5A481278172505FB02028F
:10DDB800527912F0100F01D001224A701B78554A8F
:10DDC800313B1278DBB21A4112F0010F00F0988053
:10DDD800227852FA03F010F0010F0BD0897800294D
:10DDE80040F08E80013111FA03F3C3F10F0303EA07
:10DDF800020204E0012111FA03F343EA020222704D
:10DE0800002112224448F2F7C5FA2046BDE87040C6
:10DE1800FFF7ECBE132A0CD0552A17D13B4B3C4ACE
:10DE28001B78172101FB03235B7913F0200F03D123
:10DE380070BD354B01225A7000202146FFF726FF9E
:10DE4800344B9B78002B5BD0002051E0142A0CD077
:10DE58002A2A17D12D4B2E4A1B78172101FB0323A1
:10DE68005B7913F0200F03D170BD274B01225A7044
:10DE780001202146FFF70AFF264BDB78002B3FD015
:10DE8800012035E0152A0CD0232A17D11F4B204A30
:10DE98001B78172101FB03235B7913F0200F03D1B3
:10DEA80070BD194B01225A7002202146FFF7EEFE81
:10DEB800184B1B79002B23D0022019E0162A0CD00E
:10DEC800442A1DD1114B124A1B78172101FB032349
:10DED8005B7913F0200F03D170BD0B4B01225A70F0
:10DEE80003202146FFF7D2FE0A4B5B7943B103209A
:10DEF8000949102246F6C553BDE87040FAF7DEBB63
:10DF080070BD00BF04180020670E0020CC18002048
:10DF18008D320020D6180020061800202DE9F04F79
:10DF280087B09DF840508046072D0E4605929A46C8
:10DF380037D1002427463378234113F0010F2CD022
:10DF4800012523B24FF000080293512029462A46A2
:10DF58002B460095CDF8048002F08CFF1B2041462B
:10DF680062194346CDF80080F4F7C6FB37B9112093
:10DF780039463A462B460097F4F7BEFB534B2046EA
:10DF880013F8242001276FF3000203F824201199C5
:10DF9800F5F722FA2046F5F723FC0134042CCAD100
:10DFA800F7E1012D03780CD10BB90B7823B3FF23CC
:10DFB80000930021464B01911B780C2001330293FA
:10DFC80016E0022D09D10BB90B78ABB10021FF2364
:10DFD80000930191029134200AE0062D0CD10BB96F
:10DFE8000B784BB10021FF2300930191029165202A
:10DFF80004220B4602F03EFFBAF1010F98F80030F8
:10E008002BD13BB1334B0020D979024653460090BF
:10E01800F4F772FB33783BB12E4B0120D9790022FB
:10E0280003460092F4F768FB0020F5F7C7F998F863
:10E038000030002B5BD0284B1978002957D1274B8B
:10E04800DB78002B53D0FF2300933A2001220B46A4
:10E058000191029102F00EFF49E063B1052D4FF0E6
:10E06800000102D100910F2001E000910B200A4627
:10E078000123F4F741FB337883B1052D4FF00001FC
:10E0880006D110200A4601230091F4F735FB12E06F
:10E098000C200A4601230091F4F72EFB022D25D00F
:10E0A800032D01D10E4B02E0042D02D10D4B1F7838
:10E0B8001DE0052D01D10C4BF9E7012D01D1044BD1
:10E0C800F5E7062D0CBFFF27002710E010150020EC
:10E0D800DD150020D6180020FE140020670E002051
:10E0E800E01A002037390020DF330020FF2798F896
:10E0F8000030002B00F09D80914C237803F0200322
:10E10800DBB26BB18F4B197811F0010108D1FF23F5
:10E118000093282001220B460191029102F0AAFEE9
:10E12800237803F01003DBB273B1864B197801F042
:10E138000201C9B241B9FF230093292001220B46ED
:10E148000191029102F096FEE37813F0010F0ED0D0
:10E158007C4B197801F00401C9B241B9FF2300933F
:10E168002A2001220B460191029102F083FEE378F6
:10E1780003F00203DBB273B1724B197801F00801A6
:10E18800C9B241B9FF2300932B2001220B4601910C
:10E19800029102F06FFEE37803F00403DBB273B17F
:10E1A800684B197801F01001C9B241B9FF230093F7
:10E1B8002C2001220B460191029102F05BFEE378CC
:10E1C80003F00803DBB273B15E4B197801F020014C
:10E1D800C9B241B9FF2300932D2001220B460191BA
:10E1E800029102F047FE0FF017FB70B1554B1978FA
:10E1F80001F04001C9B241B9FF230093492001222F
:10E208000B460191029102F035FEE37803F04003DA
:10E21800DBB273B14B4B197801F08001C9B241B937
:10E22800FF2300934E2001220B460191029102F038
:10E2380021FE119B444A1978444B51B198F80010BB
:10E24800117032781A7033780BB1542005E05220DF
:10E2580003E01170327853201A7003F0E7F9119B2C
:10E2680000241A783A4B1A7098F80030234113F0BA
:10E27800010F2DD02146059814F01BFA0122014602
:10E2880028B923B2019000920293104605E00021BC
:10E2980023B200920191029324200B4602F0EAFD7A
:10E2A800BAF1010F05D12B4B8020DA790521013213
:10E2B80008E0022D07F1010202D18020072101E0C8
:10E2C800802006212346F5F79DFD2046F5F75CFAE8
:10E2D8003378234113F0010F57D000214FF0010B81
:10E2E80023B2029302205A460B46CDF800B00191A2
:10E2F80002F0C0FDDA45DFF868900CD119F8243037
:10E3080013EA0B0334D1134A0520D17900935944F9
:10E3180004EB0B022AE019F8243013F0010327D18B
:10E32800022D1FD10C4B1B7803F02403042B04BFD0
:10E338000A4B83F800B000230093072014E000BFC5
:10E34800C03100209F1600204815002049150020E4
:10E35800BC160020D6180020C6160020600E00202B
:10E368001015002000930620791C621CF4F7C4F9EC
:10E3780011992046F5F730F82046F5F731FA19F8E3
:10E3880024306FF3000309F824300134042C7FF49F
:10E398006BAF07B0BDE8F08F2DE9F04180460E461F
:10E3A800174646F28B7500243846214614F081F949
:10E3B80088B1294608220B4802F0EFFC094841467B
:10E3C80014F024F9074814F047F920B90123A340B1
:10E3D80032781343337001340835042CE4D1BDE896
:10E3E800F08100BFB41600202DE9F04387B08046C5
:10E3F800894604A847F2B511082202F0CEFC002491
:10E4080040462146E7B214F054F9002843D0384674
:10E41800F3F7AEFE0025661C0246314611202B4656
:10E428000095F4F769F9012321462A460420FF08DC
:10E438000095F4F761F94AF2B340381802F09CFCF1
:10E4480004F00703C1B2194111F001014FF00202B3
:10E458004FF001030AD00092019336B27720294683
:10E4680092182B46029602F005FD14E000920193E3
:10E4780036B2232004220B46029602F0FBFCB9F1C7
:10E48800000F08D004A8214614F013F918B1054864
:10E49800214614F0F8F80134402CB1D107B0BDE89A
:10E4A800F08300BF251500202DE9F74F1746984641
:10E4B8003B7805460C469DF830909DF834B09DF8A1
:10E4C8003820DFF8B4A043B102EA03033B700978AF
:10E4D8009AF800208A18D31A0370237883B1214848
:10E4E8002146F5F729F920491E4814F08FF81D48F0
:10E4F8000121FFF779FF1B4841462246FFF74CFFF1
:10E508001A4B00261E70297843F6F72002F02AFCE1
:10E51800494646F2C96002F025FC204639464A467B
:10E52800F4F710FF124B39461E7142464B462046FF
:10E53800CDF800B00195FFF7F1FC2846F7F7A2FDEA
:10E548002B780C480C498AF80030F5F7F5F888F86C
:10E5580000603E7026702E7003B0BDE8F04F02F0E8
:10E5680075BF00BFBD160020401500200819002007
:10E57800670E0020A0160020FE14002010B50B4BDB
:10E588000B4C024603CB206061600A48114614F028
:10E598005EF82146074814F039F8064814F05CF88C
:10E5A800D0F1010038BF002010BD00BF7825002041
:10E5B800AA160020B416002010B50A4C637C4BB193
:10E5C80000200949FAF72EF9084B1B78432B01D193
:10E5D800433B6374607C20B90549BDE81040FAF7F5
:10E5E80021B910BD06180020CDD402080418002057
:10E5F800ACD40208034B1A7801321A700123037055
:10E60800704700BF0819002010B50C48FAF7B0F899
:10E618000B4A002414700B4A0B4B14700B4A5C71A4
:10E6280014700B4A1C7114700A4A5C7014700A4A00
:10E638001470FAF7BBF9094B1C6010BD18190020BB
:10E64800D618002005180020670E00200A1900209F
:10E658001619002040180020081900203C18002036
:10E668002DE9F04F934B944E93F800903368DFF800
:10E6780094829C7C914BF0221A7098F800308BB0F1
:10E688000C2B354647463DD18D4B93F805C0BCF160
:10E69800010F02D900208B492FE01AD100245C71A8
:10E6A800894A8A4B8A498B488B4D04701C701470B8
:10E6B8000C70CDF800C001942D780295FFF7F4FE98
:10E6C800FAF774F9854834600BB0BDE8F04FFAF7F3
:10E6D8004FB883487E49F5F72FF8824B824A03CB1F
:10E6E800824B10601B785160532B57D198F800303B
:10E6F8007F49013388F8003000200BB0BDE8F04FA7
:10E70800FAF790B8082B0FD1784B1B78532B3DD1D3
:10E71800784B00221A700C2388F80030764B1A7850
:10E7280042F006021A707FE20D2B37D16F4B1B782F
:10E73800532B2BD171496A4813F068FF6848FFF7DB
:10E748001DFF044640B198F800300522013B88F8C7
:10E7580000305B4B5A7167E2082246F2CA61624890
:10E7680002F01BFB6049664813F071FF0123009318
:10E77800594B01941B78574802935549524A534BB9
:10E78800FFF792FEFAF712F934604DE2232B40F0BE
:10E798004B820BB0BDE8F04FFFF736BF631E48BF92
:10E7A800A31DDB10013303FB09F91FFA89F909F5E9
:10E7B800CC46A9F5B649A9F14D094F4BCDF81C90A7
:10E7C8001A78CA3612F0010F4A4C00F01E81474BE6
:10E7D8001A789946432A40F0C7803B780C2B40F0C2
:10E7E800C3803F48217813F064FF002800F0BC8004
:10E7F8003D48217813F05DFF002840F0B580079967
:10E8080020780FFA81FB0BEBD00002F0B5FA2378E1
:10E818004FF0010A03F007020AFA02FADFF8E8806B
:10E828005FFA8AFA10EA0A0FC8F8000027D0244BCA
:10E83800DB78002B40F09880274BD879F7F780FBDE
:10E84800002800F09180D8F80010CAF1FF0A20785B
:10E858000AEA0101C8F800100BEBD00002F082FAB6
:10E8680020780FFA86FB0BEBD00002F085FA00EA5D
:10E878000A012078C8F800100BEBD0005FE032B234
:10E8880002EBD300059202F077FA10EA0A0FC8F8F3
:10E8980000003BD140EA0A01059B2078C8F8001027
:10E8A80003EBD00002F05EFA2178154813F0EBFE76
:10E8B8005AE000BFC91800203C1800201519002094
:10E8C800670E002072D502080A19002005180020DA
:10E8D8001619002040180020D6180020181900200A
:10E8E800BD16002078250020F4140020041800200C
:10E8F80038D60208D3180020091900203515002041
:10E908004015002008190020E0180020924BDB7801
:10E9180023B9924BD879F7F713FBB8B92078DDF80B
:10E9280014C0CAF1FF0A0CEBD00002F025FA8C4A99
:10E9380000EA0A01059B2078116003EBD00002F081
:10E9480011FA2178874813F0A9FE0DE020780BEB27
:10E95800D00002F011FA40EA0A012078C8F8001045
:10E968000BEBD00002F0FEF999F80030232B10D100
:10E978002A682378927C013A93420ADA7A4A013368
:10E9880013707A4B9B7803F00203DBB20BB1F9F7F3
:10E9980045FE99F800302A2B0CD1237853B1724ADE
:10E9A800013B1370714B9B7803F00203DBB20BB190
:10E9B800F9F734FE99F80030552B12D129682278DE
:10E9C800897C694B08398A4201DA083200E0002262
:10E9D8001A70664B9B7803F00203DBB20BB1F9F7B0
:10E9E8001DFE99F80030442B0FD122785E4B072A80
:10E9F8009CBF2A68927C083A1A705C4B9B7803F09B
:10EA08000203DBB20BB1F9F709FEFBF75FFD584AC9
:10EA1800237811789246994288BF137012780F3282
:10EA2800934202DD524A0F3B13702B684FF0000BE4
:10EA380093F81280CDF818B0B8F10F0F9ABFC8F14B
:10EA480020085FFA88F84FF0100839784FFA8BF3EE
:10EA58000C2905D19AF800209B18DB10454A04E0E0
:10EA68009AF800209B18444ADB10D35C9AF80020DF
:10EA780005934FFA8BF39A180C2902F007094FEA0D
:10EA8800E20202D13D49895C0691DDF81CC004937D
:10EA98000FFA8CF0101802F06FF9C0B2049B0890BE
:10EAA8009AF8000032B2181802EBE00002F064F99C
:10EAB80039789AF80020049BC0B209919A1846E068
:10EAC800059BDDF824C043FA09F12D4B01F0010143
:10EAD80000290CBFA521DB21BCF10C0F03F808109D
:10EAE80014D128494FEAE20C11F80C1041FA09F147
:10EAF80011F0010F08D0DDF818C04CFA09F111F037
:10EB0800010F03D0582110E02D210EE0DDF820C0C0
:10EB18004CFA09F111F0010F01D0502105E040FA3B
:10EB280009F111F0010F02D0542103F8081009F17E
:10EB380001095FFA89F90BF1010B08F101080132AB
:10EB4800B9F1080F5FFA8BFB5FFA88F81CD0B8F1AF
:10EB5800200FB5D125E000BF670E0020D618002091
:10EB6800E018002040150020D318002018190020B4
:10EB7800CB1800203515002095150020F41400202E
:10EB8800F4010020BD160020B8F1200F09D09AF832
:10EB980000304FFA8BF2D2182B689B7C9A42FFF612
:10EBA80054AF23490B7813F0010F17D02B68214A73
:10EBB8009B7C12780F2B02F0800298BFC3F11003E0
:10EBC800D2B294BFDBB2002342B122789AF8001087
:10EBD8001032521A1849CB185F219954174EB3783E
:10EBE80003F00203DBB293B1F11D652246F66143DF
:10EBF8002078F9F763FD2B689B7C102B02D9052040
:10EC08000B2101E0002007213246F9F7C3FD2B68EC
:10EC18009B7C102B08D921780948013102220BB0BE
:10EC2800BDE8F04FF9F724BE0BB0BDE8F08F00BF88
:10EC380009190020C0310020F40100201819002013
:10EC4800F50100202DE9F043002387B08DF8173037
:10EC5800754B1B78012B00F06082744B1A7898462C
:10EC680072B1734BDB78002B40F05782714C2378DC
:10EC7800002B40F0A780F9F799FE08232370A1E044
:10EC88006C4B19781C46072900F29C806A49097860
:10EC9800232913D11A70F9F789FE6849684A0B7855
:10ECA80053B16848013B0478DBB244F006040470B1
:10ECB8000B70654951F8233013609FE2614B1A7855
:10ECC80012F0010F04D101210A438DF817101A70B0
:10ECD800F4F744F928B923781BB90DF11700FFF7A9
:10ECE80089FCF4F749F930B92378012B03D10DF1E8
:10ECF8001700FFF77FFCF4F74DF930B92378022BA2
:10ED080003D10DF11700FFF775FCF4F74FF930B98F
:10ED18002378032B03D10DF11700FFF76BFCF4F7F1
:10ED280053F948B9F4F76CF930B92378042B03D1B7
:10ED38000DF11700FFF75EFCF4F7A0F930B923785E
:10ED4800052B03D10DF11700FFF754FCF4F78AF9EE
:10ED580030B92378062B03D10DF11700FFF74AFCD1
:10ED6800F4F740F930B92378072B03D10DF11700D8
:10ED7800FFF740FC9DF8173023B32378072B1FD8E3
:10ED8800DFE803F004070C0F1215181B00202F49A9
:10ED980001E02F490020F9F745FD13E000202D4937
:10EDA800F9E700202C49F6E700202C49F3E700207A
:10EDB8002B49F0E700202B49EDE700202A49EAE734
:10EDC800F9F7F4FD1B4F3B783D46082B40F0B08027
:10EDD8001C4E194F317811F0010151D1234C1222E8
:10EDE8002046F1F7D7FA01236374214A98F80030D6
:10EDF800137003B96374637C13B11E4B00221A703D
:10EE0800FFF7DAFB1A48617CFEF780FF337803F0DE
:10EE1800FD0343F001033370174B1A7872B33A704D
:10EE280000221A702CE000BF15190020FE140020E3
:10EE3800670E00200819002004180020F718002089
:10EE48003C18002009190020F81800201EDB0208D1
:10EE5800FDDA02083FDB020860DB020881DB0208FA
:10EE6800A2DB0208C3DB0208E4DB02080618002064
:10EE780040180020600E0020CD18002030233B7081
:10EE88003B78884E13B97378102B4DD1DFF8649214
:10EE9800854CFFF791FB844899F81110FEF736FF6F
:10EEA800237823B1002010214A46FEF7C9FE98F8BE
:10EEB800003024787D4A24EA030111707C4A23EA51
:10EEC800040111703A78A2F15200C0B2012803D9A6
:10EED8007078744F10280CD1002373701CB911B1CD
:10EEE8000133009311E1042373712B7801332B70E4
:10EEF8001AE0432A18D1BBB9FC78ACB96D4BD87964
:10EF0800F7F71EF838B96C49F9F78CFC05237B71C3
:10EF180007332B7004E020466849F9F783FC7C71BD
:10EF2800674A684B1A6069E15F48FEF7DDFE65E1F4
:10EF3800092B31D15D4808F0BFF9C6B2594C36B338
:10EF48006379042B02D100205F4903E0022B04D12E
:10EF58005E490020F9F766FC02E00BB904336371DF
:10EF6800314602225A48F9F783FC5A4B1E78232E61
:10EF780000F0D3803046F9F711FD002800F03E81FB
:10EF8800312E40F03B812B7801332B7002E03B7827
:10EF980001333B70042332E00A2B32D1434808F096
:10EFA80071F9C6B23F4C36B36379042B02D1002005
:10EFB800494903E0022B04D148490020F9F732FC03
:10EFC80002E00BB904336371314602224048F9F775
:10EFD8004FFC404B1E78232E00F09F803046F9F7F7
:10EFE800DDFC002800F00A81312E40F007812B78E3
:10EFF80001332B7002E03B7801333B7008236371C7
:10F00800FCE00B2B40F0FA80284808F021F9002199
:10F01800C4B2264808F0F2F8002C6DD0214E33799E
:10F028002BB9BE2014F032F9337901333371737977
:10F038001C4A092B02D900201F4915E010D11D4B8D
:10F0480000241C705471264B194A1849164801258A
:10F058001C7014700C7004700095019402949EE06A
:10F06800082B04D11F490020F9F7DCFB11E0062B1F
:10F0780002D100201C49F7E7042B02D100201B49CC
:10F08800F2E7022B02D100201949EDE70BB908334A
:10F0980053717379082B3CD80D4821460222F9F7A1
:10F0A800E7FB36E0670E0020401800201619002004
:10F0B8000A190020D618002072D50208EED40208DA
:10F0C800E04D02083C180020F6D5020817D60208C1
:10F0D800F401002004180020B4D50208D5D5020890
:10F0E800051800200FD5020830D5020851D50208AE
:10F0F80093D5020806180020012542484249434A90
:10F108002B460095F4F7CAFC0095414B01941B78F7
:10F1180040E0404F3C78232C02D1FFF775FA6DE0B0
:10F128002046F9F73BFC002868D0303CE4B2631E67
:10F13800DBB2012B3C7039D8022C354D1ED1E87951
:10F14800F6F7FEFE002838D02E48FFF717FA0028F9
:10F1580033D1082246F2CA612F4801F01EFE294920
:10F168002D4813F05EFA2C49082246F2CA6001F0D5
:10F178000EFE2949294813F06AFA06E001232148BE
:10F188002149224A0093F4F789FC012300240093C3
:10F1980001942B78029322481C49224A1A4BFFF704
:10F1A80083F9F9F703FC204B1C6027E0032C25D1D9
:10F1B800174BD879F6F7C4FE10B90C2373711DE00C
:10F1C80000241048214613F074FA28B1E02014F006
:10F1D8005DF8204614F096F80134402CF1D1134A1A
:10F1E8000023137073712B78114A01332B700E4B67
:10F1F8001A60104B1A7842F006021A7007B0BDE880
:10F20800F08300BFBD160020051800201619002045
:10F21800D618002004180020F414002040150020FF
:10F22800401800200A1900203C180020D31800209C
:10F23800E04D0208091900201FB5044611B100204D
:10F248000B4901E008460B49F9F7ECFA217810223E
:10F258000139C9B201EB011101F5C24144316846D7
:10F2680001F09BFD102001466A46FEF7E9FC1FBD30
:10F2780074AC0208B6AC02080B4B1B78442B06D0C2
:10F28800552B037801D013B17047013B01E0037897
:10F298000133037003780BB9203302E0212B01D12D
:10F2A800203B0370FFF7C8BF041800202DE9F74F73
:10F2B800DFF8C881DFF8D4A198F80030554643F04C
:10F2C800010388F800309AF80130624C23F07F037C
:10F2D8009B46D3B100206049F9F7A4FA5F482A2178
:10F2E800F1F7D6F818B121788222F9F7C1FA227815
:10F2F800002A40F0AB802B6862F3CF332B60584B69
:10F308001A7842F003021A70A0E0DFF854912370D3
:10F3180099F800304E4603F00202D2B20192514FE2
:10F32800002A40D013F0010813D058464E49F9F787
:10F3380079FA3B78232B20D14C4B4D4A4D481A6023
:10F348000121FFF779FF337803F0FE036BF34103E4
:10F3580012E040464849F9F765FA3B78232B0CD16F
:10F36800424B434A43481A600121FFF765FF33784F
:10F3780068F3000368F3410333703B782A2B65D1A7
:10F38800337803F0FE036FF3410333702B6843F4C3
:10F3980000432B600F232370364B187803B0BDE869
:10F3A800F04F0DF0C7BC0DF009FC054600282DD024
:10F3B80001213048FFF760FF3B78532B12D1337897
:10F3C800019A03F0FD0362F300033370DAF80030AA
:10F3D80043F40043CAF800300F232370254B1878F4
:10F3E8000DF0A8FC3B78232B30D13378002203F0B2
:10F3F800FD036FF3000333701E4B1A70F9F7D6FA4A
:10F408001E4A137843F00603137015E01C49F9F7F8
:10F4180009FA3B78232B19D199F8003065F3410399
:10F4280065F3000389F80030F9F7C0FA98F800305E
:10F4380043F0060388F80030124A1378013BDBB228
:10F448001370114A52F82320084B1A6003B0BDE824
:10F45800F08F00BF423A0020F8AC0208F401002007
:10F46800633300200418002019AD02083C1800205E
:10F47800FC4D0208D31800203AAD020809190020F3
:10F488005BAD0208F7180020F8180020C0310020F2
:10F498002DE9FF412C4D2D4C2B7843F001032B70A7
:10F4A800217801F00401C9B211B92948FFF7E4FE37
:10F4B800284E3378232B21D12378274F13F00408C3
:10F4C8000AD0224A6FF382031370244B20483B6012
:10F4D8000021FFF7B1FE11E0F9F768FA2B78204A0E
:10F4E80043F006032B701378013BDBB213701D4AFF
:10F4F80052F823303B60164B83F800803378532B47
:10F508001FD12378052243F004032370104B1649BA
:10F518001C78013CE4B204EB840000F5CA40843056
:10F5280001F035FC00201149F9F77CF9FF2300218F
:10F5380000930134162004220B460191029401F035
:10F5480099FCBDE8FF8100BF091900206333002042
:10F55800D3180020041800203C180020184E020878
:10F56800F7180020F8180020344E0208D7AC02081B
:10F578002DE9F041984B04469A7812F0010F00F0FB
:10F5880017811B88002B40F01381944D95F820308B
:10F598003F2B40F2D780012C14D1914B1B7803F0FC
:10F5A8000203DBB2002B00F0C48095F820208B4BBF
:10F5B800402A03D1013283F82020FBE0482283F857
:10F5C8002020B6E0022C03D1482385F82030B0E093
:10F5D800844E337803F02002D2B28AB195F8202005
:10F5E800402A0DD1032C0BD07F4B804A03F1100128
:10F5F80053F8040B8B4242F8040BF9D1412395E0F0
:10F6080003F01003DBB28BB195F82030412B0DD1FC
:10F61800032C0BD0764B754A03F1100153F8040BF9
:10F628008B4242F8040BF9D142237FE0F37813F0C0
:10F63800010F0FD095F82020422A0BD16D4B6B4A51
:10F6480003F1100153F8040B8B4242F8040BF9D173
:10F6580043236BE003F00202D2B27AB195F820207E
:10F66800432A0BD1644B614A03F1100153F8040B90
:10F678008B4242F8040BF9D1442357E003F004020B
:10F68800D2B27AB195F82020442A0BD15B4B574A65
:10F6980003F1100153F8040B8B4242F8040BF9D123
:10F6A800452343E003F00803DBB28BB195F8203023
:10F6B800452B0DD1032C0BD0514B4C4A03F11001B3
:10F6C80053F8040B8B4242F8040BF9D146232DE082
:10F6D8000EF0A2F8A0B14B4B1B788BB195F82030F7
:10F6E800462B0DD1032C0BD0474B404A03F1100198
:10F6F80053F8040B8B4242F8040BF9D1472315E069
:10F70800F37803F04003DBB29BB195F82030472B28
:10F718000FD1032C0DD03D4B344A03F1100153F89F
:10F72800040B8B4242F8040BF9D1482385F82030AA
:10F7380078E095F820300133DBB2472B85F820308C
:10F748007FF629AF95F82060472E04D9234B002671
:10F7580083F8206001E00136F6B206F14007FFB2F7
:10F7680012E02B48314612F0A4FF08B1032C04D153
:10F77800284B9B5D23B1032C02D185F820600FE054
:10F788000136F6B2BE4203D03F2EEAD9402E07D149
:10F79800214B1E221A70402385F82030BDE8F081E5
:10F7A80095F820001149652246F66143F8F786FF6F
:10F7B800012C37D1194B0D4A03F1100153F8040BF2
:10F7C8008B4242F8040BF9D1044B93F820303F2BBD
:10F7D8003CD9002012493EE018190020F40100200D
:10F7E800FF140020C0310020ACB302081F1900200C
:10F7F800CDB30208EEB302080FB4020830B4020811
:10F8080051B402084035002072B40208B4B40208AA
:10F81800951500204B150020D4180020AC160308BD
:10F828006AB30208104BD87800F02000C0B220B1AB
:10F83800022C06D000200D490DE0032C01D10C4903
:10F8480009E00C4B93F820303F2B02D800200A49DE
:10F8580001E00A490020F8F7E5FF1020084A0146B0
:10F86800BDE8F041F8F796BFC031002085AA02082C
:10F878008BB30208F401002028B3020893B40208ED
:10F888001819002010B5F9F791F8084B1B7803F008
:10F898000403DBB22BB106490020BDE81040F8F79D
:10F8A800C1BF0220BDE81040FFF762BEFF14002070
:10F8B8005AB1020870B5224B06461B78214CF3B9A1
:10F8C800257819E02048294612F0F3FE78B123681C
:10F8D8009D4202D9FF2E02D007E0FF2E02D19D42A1
:10F8E80008D202E036B91DB913B9256012E00EB985
:10F8F800013500E0AD19EDB23F2DE3D90AE0013B37
:10F908002021124810222360F0F744FD00201049FE
:10F91800F8F788FF0F48F8F72BFF46F66143207881
:10F928000D496522F8F7CAFE084D216805F1100057
:10F9380001310222F8F79CFF2D23AB7470BD00BF84
:10F94800C9180020E018002042180020F401002007
:10F9580028F50208181900201F190020F8B5544B83
:10F96800F02254481A700378044613F00E0518D193
:10F97800514A43F00203156000F8013B12F03EFEC5
:10F988002C464E4BE35C1BB14D48214612F07BFEE2
:10F998000134402CF5D14B4B1A7842F001021A7011
:10F9A800F8BD13F00C0543D12E464548294612F000
:10F9B80080FE08B10136F6B20135402DF5D11EB9E9
:10F9C800237843F0040331E000253F482946EFB28D
:10F9D80012F06FFE68B1394BEB5C53B13B4B01370A
:10F9E8001F700020FFF766FF237843F00803237099
:10F9F80002E00135402DE8D1354D3A212846F0F78F
:10FA080047FD38B1401BC0B20130281831460222E8
:10FA1800F8F72EFF2F4B1B78532B47D12B4B002089
:10FA28001870FFF747FF237843F008032370F8BDE9
:10FA38006FF34103037003F00403DBB2254D23B1D8
:10FA480000202549F8F7EEFE0EE02B78552B01D162
:10FA5800FF2002E0442B02D10120FFF72BFF1320E7
:10FA68000D211E4AF8F796FE2B78232B1ED12278FB
:10FA780002F00204D4B90F4902F0FB0264F3C30296
:10FA88000A700D4A1460F8F791FF0E4B1A7842F08D
:10FA980006021A70124A1378013BDBB21370114A3E
:10FAA80052F82320104B1A60084B1C70F8BD00BF99
:10FAB8001519002041180020E0180020E823002034
:10FAC800421800200919002000150020C91800203C
:10FAD800F4010020041800206E06030818190020FD
:10FAE800F7180020F81800203C18002070B50546CB
:10FAF8000C4616463BB143004AF28D3018184018A0
:10FB0800114601F02FF9054B172202FB0535F309C1
:10FB18002C1906F07F066370E67070BD8D320020E8
:10FB280038B510B3A0F14103DBB2432B1FD9C50987
:10FB380000F07F040BD0052C19D90021601E0A465D
:10FB48000AF042FCD0F1010038BF002038BD082C73
:10FB58000FD9601EC0B229462A460AF09FF850B94C
:10FB6800202C8CBF0020012038BD012038BD00208A
:10FB780038BD284638BD284638BD0000F7B5614C69
:10FB880031232374604F01332376053B6374637616
:10FB98003B784AF28D305B00181801F0EDF8C0B2DE
:10FBA80020F07F0200F07F01D2B28DF804108DF8AA
:10FBB800002004F1120359B9544A04F115001188C0
:10FBC800927861829A7020210222F0F7E3FB0CE020
:10FBD800D20904EB8202526A10886082927804F19A
:10FBE80015009A700222F8F743FE3878400000F5B5
:10FBF800224000F5C77001F0BFF8C0B220F07F03C3
:10FC080000F07F01DBB28DF805108DF80130404817
:10FC180051B93E4B20311A889B7862838370022247
:10FC28000330F0F7B7FB0BE0DB0904EB83035B6AF7
:10FC38001A8862839B78022283700330F8F718FED3
:10FC4800344B1B7813F0010F5AD0334D02A92A7890
:10FC58008B1813F8041C13F8086C304B1B78232BF3
:10FC680004D1002A41D1223B2B703EE02A2B04D13B
:10FC7800002A3AD0013A2A7037E0552B46EA0106A5
:10FC880011D10DE02B7802AAD318013E13F8081CF5
:10FC9800F6B23046C90913F8042CFFF741FF98B9AA
:10FCA800002EEFD121E0442B19D115E02B7802A9C1
:10FCB800CB18013613F8081CF6B23046C90913F8F8
:10FCC800042CFFF72DFF38B1134B387819783246DA
:10FCD8000123FFF70BFF08E0872EE7D905E0532B38
:10FCE80003D1533B2B70FAF7F1FB0D4B1B7803F054
:10FCF8008003DBB223B12B782022023304F83320AF
:10FD0800FEBD00BFF4010020C91800206B120308D3
:10FD18000E02002009190020D31800200418002022
:10FD2800C0310020024800210922F0F733BB00BF90
:10FD3800E518002070B50A46002405E01B19811A51
:10FD48002A2501345D54E4B20E4D0F4B295D09B1EB
:10FD58009442F3D1801A001918182021121BF0F7C9
:10FD680019FB0A4B1E785EB1432E04D10CB1013C3D
:10FD7800E4B200232B553046F8F710FE00B12E559B
:10FD880070BD00BFE5180020F40100200418002011
:10FD980038B5184C184DA07800F01000C0B250B912
:10FDA8001649F8F73FFDFFF7BDFF236843F48013BA
:10FDB80023600F232B702A782AB92368FF2062F367
:10FDC8001453236038BD0E48C5792DB91C2008216D
:10FDD800FFF7B0FF284638BD23680A496FF314536C
:10FDE80008222360F0F756FD00280CBF0120FF20F1
:10FDF80038BD00BFC031002017190020BDB102086E
:10FE0800E5180020AA310308F0B55B4C85B0667888
:10FE180006F01006F6B2002E3ED1584B1A78584B11
:10FE2800013A53F82230574A934204D1564B1A7874
:10FE380042F0020207E002F11C018B4208D1524B4A
:10FE48001A7842F00402022161F3C7021A7019E01D
:10FE58003832934216D1FFF79BFF002800F08A80C2
:10FE68000128494D06D12B78022243F0010362F3A1
:10FE7800C70306E030464549F8F7D4FC2B7866F30B
:10FE8800C7032B70424B1A7842F001021A7023689C
:10FE980043F4805323606DE03B4D2B7813F0F80654
:10FEA80006D03C49002005B0BDE8F040F8F7BABCE0
:10FEB80013F0070F3FD003F00202D7B24FB1122060
:10FEC80031460EF03DFEFF23009301960296432033
:10FED80028E003F00406F6B296B1394638460EF02B
:10FEE8002FFE0EF079F809F003FD0CF08FFEFF23CA
:10FEF8000093019702974420394604223B4614E0B8
:10FF080013F0010F13D0012143F61C600EF018FE08
:10FF18003046F6F77FF8204B45201E80FF230093DC
:10FF28000196029631460422334600F0A3FF0020D2
:10FF38001A49F8F777FC2B7803F0FA036FF34103BB
:10FF48002B70174B1B78232B14D123686FF30C33BA
:10FF58002360F8F72BFD0E4B1A7842F006021A7050
:10FF6800064A1378013BDBB21370054A52F8232086
:10FF78000C4B1A6005B0F0BDC0310020F718002006
:10FF8800F81800203C4E0208C5370020DEB10208F0
:10FF9800091900200A0A03081A180020E9090308A9
:10FFA800041800203C1800201FB50446F6F71EF977
:10FFB800A8B14B2001F03AFBFF2300930121FF3B3E
:10FFC8000193392004220B460134029400F052FFB9
:10FFD800064B01205A7842F004025A7004E0044BA0
:10FFE8001888003818BF012004B010BD5033002015
:08FFF800583A0020F0B5204E3C
:020000040801F1
:100000000024337A0546013385B00F463372102041
:100010002146012223460094F2F772FB55B9FF23D3
:1000200000934F20294604222B460195029700F0A9
:1000300025FF0EE0012D0CD1FF2300935020234615
:10004000214604220194029700F018FF337A013B05
:100050003372337A052B11D1FA3301210024009336
:1000600027200B4604220194029400F007FF044B62
:100070001C7205B0BDE8F04001F0AEBA05B0F0BDAD
:10008000D6180020074B172202FB00335B7913F0D0
:10009000100F05D0044B163A9A715A7009329A70B3
:1000A000704700BF8D320020670E00202DE9F04F11
:1000B0009A4B87B01A78074699461AB1012A40F040
:1000C000E68130E0964B1A68964B9A4200F0E18147
:1000D000F5F716FD944B5B7803F00203DBB253B9DE
:1000E000924B5B7803F08003DBB223B901F09AFAFC
:1000F00008B909F001FC8E4B1A686FF310421A60C0
:100100008C4B1878F8F74EFC002800F0C281FFF7FE
:100110000DFE894B3C221A70F8F790FA99F80030DE
:10012000013389F80030844B1C7874B9834B791CF7
:100130001A78204664F3C30264F304121A70C9B239
:10014000FFF75CFF89F80040A3E17D4D384609F0D8
:10015000F3FBF8F767FA00207A49F8F767FBDFF856
:10016000F4812B78AA46434413F8313C23B91B2071
:100170000621FFF7E3FD8CE1704A0B21137804A8F8
:10018000C3F3C004C3F3001603F0F7036FF30413C3
:100190001370002389F80030062200F002FE2A784E
:1001A000414604A8303AF0F71FF8804628B14FF0D6
:1001B00000084FF0120945462AE049F23F6000F07E
:1001C000DFFD0028F3D0604D85F80880F5F7F8FDD5
:1001D0000446002840F05D815C4A514B21461A607C
:1001E000FF2300930190029004220820234600F090
:1001F00045FE012223460E2021460094F2F780FAA4
:10020000534B1A7842F004021A700123AB7140E19B
:100210004946062204A800F0C4FD9AF8002004A86C
:100220004C49303AEFF7E0FF002840F021812846A2
:10023000FFF7BEFE002840F02C81DFF80CB1012151
:100240008BF808002846F5F7C9FD8146F5F7B8FD9B
:10025000DA46002840F0B58048463F49F0F7A2F959
:10026000B0B901F0F7F82E4B14B916B93B4A23E0A8
:1002700036B13B4A1A603B4B1A786FF3410205E0F6
:10028000394A1A60374B1A7866F341021A70D7E080
:1002900048463649F0F786F920B148463449F0F728
:1002A00081F970B9002C40F0F480002E40F0F1800C
:1002B00001F0D0F82F4A1A4B1A603846FFF7E2FED9
:1002C000BEE048462C49F0F76DF950B949F23D605F
:1002D000012100F04BFD164A136843F400531360EC
:1002E000E0E748462549F0F75DF938B9002C40F0C1
:1002F000D080002E40F0CD80214A0CE048462149B4
:10030000F0F750F9002841D1002C40F0C280002EB7
:1003100040F0BF801C4A024B1A6091E03818002060
:100320003C180020904E0208AA2B00205F330020CA
:10033000C03100200418002017190020E418002004
:100340002018002064AA0208D6180020AC4E02082B
:1003500021210020E518002035330308F850020859
:1003600080520208091900209C520208B132030889
:1003700041350308B8520208EC320308EE32030894
:10038000F0520208FE34030844530208484642492A
:10039000F0F708F9002853D101F05CF83CB13F4A6E
:1003A0003F4B1A603F4B1A786FF3410270E0002E0A
:1003B0006FD03D4A3A4B1A603A4B1A7864F34102C7
:1003C00066E048463449F0F7EDF8064620B901F0FA
:1003D00041F8002C5DD01BE048463449F0F7E2F8C4
:1003E000002856D048463249F0F7DCF838B9002CDE
:1003F0004FD1304A2A4B8BF807501A6049E04846E3
:100400002D49F0F7CFF8064650B9A4B101F022F813
:10041000224A234B1A60234B1A7866F3410237E0D5
:1004200048462649F0F7BEF820B148462449F0F77F
:10043000B9F800B96CBB234A194B1A6001F00AF8ED
:1004400008F56A5078308AF8075000F099FC8AF86D
:1004500000009AF8070000F5D640353000F090FC17
:100460008AF801001848F5F7F1FD202D11D108E0B8
:100470000135EDB2202D08F1010809F107097FF4DB
:10048000C7AE791C0020C9B2FFF7B8FD01E0002219
:100490001A7007B0BDE8F08FF03203089C520208D2
:1004A0003C1800200919002080520208EE3203088F
:1004B000FE3403084453020835330308B1320308FD
:1004C000EC32030860530208D618002010B521480A
:1004D000214903680A789C7B944203D99C8914F0D3
:1004E000200F18D09A8912F0800F01D105E01C3B33
:1004F0009A8912F0400FFAD000E01C330360002309
:100500000B7003689B8913F0200F16D0134BDA7918
:10051000114B1A7011E00132D2B20A70986843F69A
:100520000553984209D101E00132D2B2162A03D80C
:100530000B4853B29840F7D40A700A4A136843F440
:1005400080731360F8F77AF8074B1A7842F00602C6
:100550001A7010BD3C180020C9180020D6180020C1
:1005600000060088C03100200919002010B5234979
:10057000234A0B78D3B11068848914F0200F15D169
:10058000013BDBB20B70846843F60552944228D1DC
:1005900004E013B1013BDBB200E0837B162B03D8F0
:1005A000184C5AB29440F4D40B701AE0136898892E
:1005B00010F0400F01D106E01C33988910F0800F35
:1005C000FAD0136002E00E481C3B036013689A7B6C
:1005D0000A709B8913F0200F03D00B4BDA79074B7D
:1005E0001A700A4A136843F480731360F8F726F808
:1005F000074B1A7842F006021A7010BDC918002085
:100600003C18002000060088D6180020C0310020C9
:1006100009190020084B1A68084B9A4204D003F5C8
:1006200080630C339A4205D1054B1878003818BF07
:1006300001207047002070473C180020904E0208AF
:10064000FE140020074B084A1B68934202D0383240
:10065000934205D1054B1878003818BF0120704728
:10066000002070473C18002044530208FE1400206C
:100670002DE9F04F804B814D1970A0F11103DBB2D1
:10068000012B87B00E46287006D8122801D11138E8
:1006900000E00020F5F720FD2B78522B0DD1F2F76A
:1006A0003DFD28B9F2F72EFD10B9F2F74FFD20B14C
:1006B000734B1A7842F008021A70724B724C1B7816
:1006C000002B2DD12168714A914229D0704A2360B4
:1006D0001370704A70481178037063F3C30163F3B9
:1006E000000163F3071111706C4A117863F3010183
:1006F00011706B4A117863F3C5011170694A137068
:10070000694A117863F3410163F3000163F38201E5
:100710001170664A116863F30C311160644A1370FA
:100720002368002B40F05F81604F7B7803F020034B
:10073000DBB273B15F4B93F80080B8F1000F08D1C2
:1007400049F23D60414600F011FB3B6868F34D33D0
:100750003B60594B187810F01E0002D0002057491A
:1007600007E0574B93F807909846B9F1000F05D072
:10077000544907B0BDE8F04FF8F758B8524F97F812
:1007800001B0BA46BBF1000F2DD0BBF1070F15D950
:100790004E48F7F7F1FF4E49B878652246F66153A7
:1007A000F7F790FF3878072310F003007B700EBF37
:1007B000484948464849F8F739F80CE0BBF1020FC0
:1007C00009D84248437823B1F7F7D6FF87F801905C
:1007D000ABE202237B7010203C4A014607B0BDE823
:1007E000F04FF7F7DBBF3D4FBB795BB187F806B041
:1007F00000F028FC8E20594601225B46CDF800B05F
:10080000F1F77EFF0020F2F7DDFD224A2049137840
:10081000334843F00603137000230B703149236003
:100820000B7088F8033088F801300370173303FB2E
:1008300006FC2D49934611F80CC089461CF0080FA0
:1008400004D130460593FFF731FC059B03FB06936B
:100850005B7913F0100F04D02A78133AD2B2032A2E
:1008600046D913F0200F79D02B78442B40D03DD8B7
:10087000232B3DD02A2B3AE0CC180020041800206E
:100880003D150020151900203C180020E04D0208FD
:10089000F718002009190020D31800201D18002087
:1008A000CE180020D5180020E4180020C031002008
:1008B00014190020FE140020413A0020C7AA0208A3
:1008C000670E002026DC0208D0180020181900202E
:1008D0001F190020CFAB0208AEAB0208D6180020CB
:1008E000CD180020C91800208D320020552B35D19D
:1008F0008C4B1B78002B31D18B4B93F80090B9F1C6
:10090000000F2BD143F6DB2000F03AFA012825D165
:100910001F23FB7188F8030043F6173000F030FA0C
:100920003870F87900F5D640353000F029FA787043
:100930007E48F5F78BFB9BF80030304669F34103A6
:100940008BF8003008F0F8FFF8F734F8784B794866
:100950002360794BC3F800902B7803702B78432BDE
:100960000AD1714B1B783BB9013388F80330734BC4
:100970003046236008F0E0FF28781738C3B2072B11
:1009800027D86F49FF220AF0D7FC9AF800106D4B68
:1009900060F301018AF8001001F00301022918D068
:1009A0000122032041B1009001929B7868309B188E
:1009B00002930021033206E0009001929B786C20A4
:1009C0000133029304220B4600F058FAFF238AF801
:1009D000013098F80630002B00F0A78152232B70CD
:1009E000594B00229A712268544B9A4250D1287870
:1009F000A0F14303DAB2122A22D8544A5BB29A40D9
:100A00001ED5432840F09181464B1B78002B40F0C7
:100A10008C8100F029FD4E4B48B11A780320110952
:100A2000013191FBF0F000EB4000091A04E01A7864
:100A30001109013101F0070161F307121A7074E125
:100A4000F7F7B0FF002823D0414F3A7812F0F003B7
:100A500008D163F307123A7023603E4B1A7842F0D4
:100A600008020EE0102B13D100F0FEFC80B13B78A1
:100A70006FF307133B7000232360364B1A7842F064
:100A8000100230461A7007B0BDE8F04FFFF70EBBFA
:100A9000314B1E211A78264F61F346021A702B78CB
:100AA000232B1CD12368BB4219D12C4B172202FBEC
:100AB0000636737913F0100F11D0294B1B7873B1E0
:100AC0001A4EF7F777FFFDF7A3FDF07900F56A50AE
:100AD000783000F055F93070AA20F2F773FC1C4E04
:100AE000337813F0010F43D02368BB420BD01D4A6B
:100AF000934208D0FFF78EFD28B9FFF7A3FD10B988
:100B0000AA30F2F75FFC2268174B9A4202D100200C
:100B1000F2F758FC2B78522B40F0CC80134B532229
:100B20001A70C7E0FE14002038180020D6180020E4
:100B300060530208CD180020F8180020904E0208DB
:100B4000D2180020D0180020670E0020002000C01E
:100B500009190020E4180020861900208D32002099
:100B6000F7180020E04D02089853020804180020EE
:100B70002368BB420BD06E4A934208D0FFF74AFD70
:100B800028B9FFF75FFD10B9AA30F2F71BFC2B78EC
:100B9000552B1ED1FFF7EAFC3378664843F0060375
:100BA00033708378644F03F00203DBB24BB1F7F785
:100BB000E3FD23681868FBF70BFD3B786FF34103F7
:100BC0003B705E48837803F00203DBB20BB1F7F7AA
:100BD000D3FD2B78442B1ED1FFF778FC3378554892
:100BE00043F0060333708378534F03F00203DBB204
:100BF0004BB1F7F7C1FD23681868FBF7E9FC3B78B8
:100C00006FF341033B704D48837803F00203DBB27E
:100C10000BB1F7F7B1FD2B78522B09D133780022B5
:100C200043F001033370464B1A70464B45321A703D
:100C3000454B00271F702B78232B3BD1434B3D485E
:100C40001F70434B1F70F7F797FD3C48F7F794FD73
:100C50003378404943F0060333700B78364A1BB3B0
:100C60003D4A013B17703D4ADBB20B7052F823300E
:100C70003B4A23609B68934202D109F0EDFD19E0E5
:100C800002F59A718B4203D002F5E0718B4204D1D8
:100C90000120014606F0CAFF0CE002F5EE72934215
:100CA00008D1304B1F7005E0117863F30711117004
:100CB00023603AE02C4BDB7813B10020F2F782FB83
:100CC00023681F7B17F00F0702D1FCF765FE1BE0BE
:100CD000012F02D1F9F7B0FD16E0022F02D1FAF789
:100CE0002BFD11E0082F05D84FF09C53BB4001D5D8
:100CF000FAF7E8FF042F03D123689B69984703E0C4
:100D0000052F01D1FAF796FA337803F00203DBB22C
:100D10001BB123681868FBF75BFC33786FF3410362
:100D200033702B780BB1084A137007B0BDE8F08F11
:100D3000E04D020818190020091900204C18002065
:100D4000D3180020041800201E180020D5180020F9
:100D500014190020F7180020C9180020F8180020E6
:100D6000B45302084B180020670E002007B502ABF1
:100D700003F8011D19460122002305F0AFFB0EBD4B
:100D800007B5002302A901F8013D012205F00EFC80
:100D90009DF807000EBD08B5002305F09FFB00205D
:100DA00008BD034610B508461446194605F0FEFB7B
:100DB000E0B210BD10B5034600248454084619461D
:100DC00005F0F4FB204610BD37B50546002400E0D1
:100DD0001446012260190DF1070105F0E7FB9DF8AB
:100DE0000730621C203BDBB25A2BF1D920463EBDB6
:100DF000F8B500252C461E4B1C21585D01FB043123
:100E0000400000F574506230043102220134FFF7D3
:100E1000C2FF1C355C2CEED14FF46F5420B204227B
:100E200005341449FFF7B7FFA4B243F6D4339C420C
:100E3000F4D1002548F63C472C4615E007EB460068
:100E400004EB440100B259180222FFF7A4FF013657
:100E5000F6B2094B5A199278B242EFD80134803772
:100E60000335142CBFB201D00026F2E7F8BD00BF55
:100E7000587E0208B3320308688802082DE9F34758
:100E8000044615468A46022243F61A610DF1060011
:100E90001E46BDF930909DF828809DF82C70FFF714
:100EA00080FF2F4B2F499A78BDF906008A705A7837
:100EB00000EBC000CA701A7900F578500A715A79AF
:100EC0001C304A719A791B7845EAC6158A710C70F4
:100ED00081F80190CB710D7200B20922FFF75BFF20
:100EE0001EB1214B1A8801321A80BDF80630013339
:100EF0009BB2B3F57A7FADF8063002D30023ADF88C
:100F0000063002220DF1060143F61A60FFF743FF97
:100F1000BDF80600154B188000B200EBC00000F5CC
:100F2000785000F11C05243000B2FFF729FF10F0C3
:100F3000800F03D00C4B1A88013A1A8028B2002186
:100F4000FFF714FF0A4B03F8148003EB44046770A7
:100F5000BAF1000F02D00120F5F760F8BDE8FC8778
:100F6000CC370020EE1800201A180020A82B0020F3
:100F70003D2900202DE9F743314B1D78303DEDB27E
:100F8000C5F10606F6B23EB305F11207202413E0C0
:100F900008F101080FFA89F000215FFA88F8FFF7DD
:100FA000E5FE09F10109B0451FFA89F9F0D1013CCC
:100FB0000737E4B2BFB21CB1B9464FF00008E7E70B
:100FC0000B35013428B20021E4B20135FFF7CEFE23
:100FD000B442ADB2F5D131E0122425B268462946BB
:100FE0000622FFF7DEFE9DF8003043B19DF8053084
:100FF0002BB99DF803308DF804308DF80530073497
:10100000062228466946A4B2FFF7C5FEF22CE4D1B9
:1010100068460B210622FFF7C4FE9DF8003043B15D
:101020009DF805302BB99DF803308DF804308DF80C
:1010300005300B2069460622FFF7ADFEBDE8FE83B2
:101040002018002070B509F007FC0BF08BFE05F0AE
:10105000E3FF05F009FFF2F715FCA648F5F710F8D5
:1010600043F6D120FFF78CFEA34BA44C187043F637
:10107000D020FFF785FEA24B187043F6DC20FFF767
:101080007FFEA04B187043F60350FFF779FE9E4B8E
:10109000187043F60450FFF773FE9C4B187043F62C
:1010A000DA20FFF76DFE9A4B187043F6D920FFF750
:1010B00067FE984B187043F6CF20FFF761FE964B02
:1010C000187043F6CC20FFF75BFE944B187043F684
:1010D000D220FFF755FE924B187043F6DF20FFF742
:1010E0004FFE904B187043F6E820FFF749FE8E4BF9
:1010F000187043F6DD20FFF743FE237801280CBF6C
:1011000043F001036FF30003237043F6E020FFF781
:1011100037FE237801280CBF43F080036FF3C71319
:10112000237043F6E720FFF72BFE804B01281A6857
:1011300043F6ED200CBF42F000526FF35D721A606F
:10114000FFF71EFE7A4B18B91A7860F3000202E02E
:101150001A7842F001021A7043F6EA20FFF710FEF7
:10116000637801280CBF43F001036FF30003637041
:10117000704843F66E210822FFF713FE6E4B0024E1
:101180001C705C706B48235C312B03D110302146FE
:1011900011F07DFA0134082CF4D1224643F6F61101
:1011A0006448FFF7FEFD224643F63A216348FFF705
:1011B000F8FD47F2D71104226148FFF7F2FD47F22C
:1011C000DB1104225F48FFF7ECFD0DF093F9F5F712
:1011D0005FFA43F6E120FFF7D3FD5B4C237860F321
:1011E0000003237043F6E220FFF7CAFD237860F383
:1011F0004103237043F6E420FFF7C2FD237860F338
:10120000C303237043F6E620FFF7BAFD237860F3AB
:101210004513237043F6E920FFF7B2FD237860F30E
:101220008613237043F6E520FFF7AAFD237860F3C9
:101230000413237043F6EB20FFF7A2FD237860F33D
:10124000C713237043F6E320FFF79AFD237860F37A
:10125000820323703D48FFF793FD3D4B3D49052236
:1012600018703D48FFF79DFD3C48FFF789FD3C4B5A
:1012700018703C48FFF784FD3B4B18703B48FFF764
:101280007FFD3B4B18703B48FFF77AFD3A4B1870D7
:101290003A48FFF775FD3A4B18703A48FFF770FD72
:1012A000394B18703948FFF76BFD394B1870FFF751
:1012B00061FE3848FFF764FD374B18703748FFF779
:1012C0005FFD374B18703748FFF75AFD364B1870E3
:1012D0003648FFF755FD364B18703648FFF750FD7E
:1012E000354B18703548FFF74BFD354B002869D159
:1012F000187069E034180020620E00208619002062
:10130000610E0020640E002071140020DE10002009
:101310005A3A002000000020B21600201F180020BA
:10132000630E00205332002009320020C03100201B
:1013300020290020ED320020FD320020F53200206F
:10134000D0310020E83100209F160020328CFFFFB2
:1013500040350020AEA4FFFFA0120020358CFFFF17
:101360003E350020368CFFFF71340020388CFFFFA3
:10137000E5330020398CFFFFB41A00204096FFFFB0
:10138000391700209EA3FFFFBA1700203E96FFFFEB
:10139000201800208AA3FFFFA831002007A3FFFF29
:1013A0009F2B002004A3FFFF332A002006A3FFFF8A
:1013B000A72B002005A3FFFFA12B00203A8CFFFFE5
:1013C0000218002001221A704AF28D35002428B23A
:1013D000FFF7D6FC002102460B462046FEF78AFBAB
:1013E000681C00B2FFF7CCFC012102460023204616
:1013F00001340235FEF77EFB042CADB2E7D10E4876
:10140000FFF7BEFC0D4B18700D48FFF7B9FC0D4BF4
:1014100001281A780C480CBF42F020026FF34512E5
:101420001A70FFF7ADFC094B18700948FFF7A8FCCC
:10143000BDE8704010F06ABBEA8BFFFF5E3300200E
:1014400020A4FFFF78400020E98BFFFF5C210020F3
:10145000ADA4FFFF034B1E211A7861F346021A70F8
:10146000704700BF86190020024B187800F0010079
:10147000704700BF86190020014B1878C0097047DB
:101480008619002008B5FFF7F7FF38B9044B1B7821
:1014900013F07E0F0CBF0020012008BD012008BD05
:1014A00086190020F8B547F2CD042046FFF768FC06
:1014B0002D2803DD20462D21FFF758FCA4F55C56AE
:1014C000353E3046FFF75CFC414FC0B207EBC00031
:1014D0000579C5F30015A5B90DE03D4B3D4953F81D
:1014E0003500EFF75FF820B930462946FFF73EFC9C
:1014F00007E00135EDB207EBC5031B7913F0080FC8
:10150000EBD0013447F20D139C42CED143F6C424F4
:101510002046FFF735FC2D2803DD20462D21FFF75F
:1015200025FC013443F6C8239C42F1D1012143F646
:10153000E120FFF71BFC012143F6E220FFF716FC38
:10154000012143F6E420FFF711FC012143F6E620D8
:10155000FFF70CFC012143F6E920FFF707FC01210E
:1015600043F6E520FFF702FC012143F6E320FFF7F5
:10157000FDFB012143F6EB20FFF7F8FB002143F6CA
:10158000E020FFF7F3FB002143F6EA20FFF7EEFB34
:10159000002143F6EC20FFF7E9FB012143F6DC20B4
:1015A000FFF7E4FB002149F23F60FFF7DFFB48F65D
:1015B000A8300121FFF7DAFB47F2B5142046FF21DE
:1015C000FFF7D4FB013447F2BD139C42F6D1F8BDBE
:1015D000140400206215030810B508F06DF90BF033
:1015E00085FB074B4FF416721A80012147F2C51094
:1015F000FFF7BCFB4C20BDE8104000F01BB800BF5B
:10160000583A002010B508F077F90BF003FB044BB3
:10161000002147F2C5101980BDE81040FFF7A6BBB6
:10162000583A0020024B1888003818BF0120704734
:10163000583A0020542873B5044663D83D4BDB78F4
:1016400003F02003DBB2002B72D13F2801D811F048
:1016500049FE394D35F81460002E69D1E10001F5DD
:10166000DA416846D5310822FFF79BFB3348214613
:1016700011F023F850B1F3B2072B07D03F2C05D857
:101680000122B240D243D2B22D4B27E01DF80630E2
:101690000122542B08D0562B03D0532B284B1AD1A0
:1016A00000E0284BB24007E0B240254BD2B2195DB2
:1016B00042EA01011955234B195D0A431A55FFF7F8
:1016C000D3FE98B1204B1B7883B13F2C0ED81E332C
:1016D00025F814300AE0B240D243D2B2195D02EAD2
:1016E00001011955174B195D0A401A550136082E8C
:1016F000BCD1134B1A5D134B1B5D134318D125F856
:10170000143015E0C10001F5DA416846D5310822F0
:10171000FFF747FB00231DF803202D2A05D00121E8
:101720009940074A105D014311550133082BF2D14E
:101730007CBD00BFC03100208A1900207025002028
:10174000561E0020B11C0020301700201FB501F0EC
:1017500015F910B901F026F948B10021FF230093D3
:101760000B2004220B4601910291FFF787FBAD226B
:101770000023D9B24D2909D0012A07D90D480021EB
:1017800019540D4819540D4820F813100133013233
:10179000552BD2B2EDD1074B002183F85510084BE1
:1017A00008481970084B0822197005B05DF804EB61
:1017B000EEF7F4BD561E0020B11C00208A1900204F
:1017C000151B0020F41A00208819002059B1064B7F
:1017D0000C2202FB0030437AC918837A4172083028
:1017E0000BB93C3383707047BC250020072813B524
:1017F000044624D9124B1B5C022B20D10DF10701AA
:101800000DF1060208F04EFA58B19DF806100120BD
:1018100010FA01F19DF807300A4AD05C0143D15417
:101820000DE0083CE4B2E308012104F0070411FADA
:1018300004F4054A0133D15C41EA0404D4541CBDCC
:10184000E82300202432002020320020044B0C2208
:1018500002FB00330C3A5A729A72FFF7C7BF00BFFF
:10186000BC25002010B50446FFF7F0FF034B0C2207
:1018700002FB0434FF23637210BD00BFBC250020AF
:1018800070B5104D002410482146E6B210F015FF47
:1018900098B96B7A8BB10D4AA318A25C93F880308B
:1018A000022A0AD0413BDAB2122A06D8084A5BB2B1
:1018B0009A4002D53046FFF7C9FF01340C35402C61
:1018C000E1D170BDBC250020A0160020E823002037
:1018D0000020008810B50A4B0C2203EBD00393F8CC
:1018E0008011084B02FB00331C7A3CB900F0070062
:1018F00051FA00F010F0010F18BF1A7210BD00BFAE
:10190000E8230020BC250020044B0C2202FB0033FE
:101910001A7AFF2A01D1FF3A1A727047BC250020BB
:10192000104B1B7813F0010F02D10F4B187818B130
:101930000E4B03F540720CE00C4B03F54072197A24
:101940000C330139C9B2FD2998BF01209342F6D169
:101950007047197A09B1FF2119720C339342F8D1FB
:1019600000207047C616002030170020BC2500203C
:1019700030B504461048007800F00200C0B2C8B18B
:101980000C2060430D4D285C904201D1994207D054
:10199000984201D1914203D0052A0BD1052B09D1E0
:1019A0000C2303FB0455064821462B72BDE830404A
:1019B00010F078BE30BD00BF41180020BC250020CB
:1019C000421800201FB504462146144810F075FE49
:1019D000002821D00122022300210093A3180293A2
:1019E0005C200B460192FFF749FA21460B4810F0A4
:1019F00059FE21460A4810F055FE2146094810F0CC
:101A000046FE074BE40804F5CC40195DCA3004B02B
:101A1000BDE81040FFF7AAB904B010BD251500209D
:101A200040150020A016002010B50D4C0021082202
:101A30002046EEF7B3FC43F6F120FFF7A1F9207141
:101A400043F6F220FFF79CF943F6F421607102227D
:101A50002046FFF7A6F9A37943F00203A37110BD56
:101A6000341A00200A4B1B781D2B0A4B0BD89A798D
:101A700012F0010F03D05A880AB1013A5A809A79BC
:101A80006FF3000202E09A7942F001029A71704706
:101A9000CC370020341A00202DE9F0436F4885B080
:101AA00010F0B0FDDFF8D0816D4E0024E5B228467D
:101AB00005F050FB18F8019F074618F8403C13B199
:101AC000022B3ED10FE02846FFF7C0FE21466548B5
:101AD00010F0E8FD2146644810F0E4FD214663481B
:101AE00010F0E0FDDAE028464946F3F715FE10B1A4
:101AF0002846FFF79FFD737AFF2B01D1FF3B7372DE
:101B0000737A4B4501D2F37A9BB15448214610F0C9
:101B1000BEFDF37A002B40F0C180204605F080FE28
:101B2000052128460A460B46FFF722FF2846FFF705
:101B30008DFEF37A002B40F0B1802846FFF742FF7C
:101B4000ACE090B92846FFF781FE2146434810F0EB
:101B50009EFD28463946F2F77FF9002800F097806D
:101B60003378002B00F093803AE0022814D13B48F0
:101B7000214610F08CFD3378012B01D0737A1BB90C
:101B800028460121FFF722FE28464946F3F7C4FD07
:101B900000287CD0284626E003280FD12846FFF7EE
:101BA00055FE21462D4810F072FD28460121F2F71E
:101BB00053F900286BD03378032B10E0042815D19B
:101BC0002846FFF743FE2146244810F060FD2846D2
:101BD0000221F2F741F9002859D03378042B56D06E
:101BE000052B54D04520FFF725FD50E001284ED1AC
:101BF000737A4B4502D32846FFF728FE2146194841
